:020000040800F2
:1000000000060020E1020008E3020008E302000805
:10001000E3020008E3020008E3020008E30200082C
:10002000E3020008E3020008E3020008992C00083C
:10003000E3020008E3020008E3020008E30200080C
:10004000E3020008E3020008E3020008E3020008FC
:10005000E3020008E3020008E3020008E3020008EC
:10006000E3020008E3020008E3020008811200082E
:10007000A9120008D5120008011300082D1300086A
:100080005513000881130008E3020008E30200088A
:10009000E3020008E3020008E3020008E3020008AC
:1000A000E3020008E3020008E3020008E30200089C
:1000B000E3020008E3020008E3020008E30200088C
:1000C000E3020008E3020008E3020008E30200087C
:1000D000E3020008E3020008E3020008E30200086C
:1000E000E3020008E3020008E3020008E30200085C
:1000F000E3020008E3020008E3020008AD13000871
:10010000E3020008E30200087D440008E30200085F
:10011000E3020008E3020008E3020008E30200082B
:10012000D9130008011400082D1400085914000800
:1001300085140008E3020008E3020008E302000857
:10014000E3020008E3020008E3020008E3020008FB
:10015000AD140008D914000805150008E3020008D2
:10016000E3020008E3020008E3020008E3020008DB
:10017000E302000885380008E3020008E3020008F3
:10018000E3020008E3020008E3020008E3020008BB
:10019000E3020008E3020008E3020008E3020008AB
:1001A000E3020008E3020008E3020008E30200089B
:1001B000E3020008E3020008E3020008E30200088B
:1001C000E3020008E3020008E3020008E30200087B
:1001D000E302000871380008E3020008E3020008A7
:1001E000E3020008E3020008E3020008E30200085B
:1001F000E3020008E3020008E3020008E30200084B
:10020000E3020008E3020008E3020008E30200083A
:10021000E3020008E3020008E3020008E30200082A
:10022000E3020008E3020008E3020008E30200081A
:10023000E3020008E3020008E3020008E30200080A
:10024000E3020008E3020008E3020008E3020008FA
:10025000E3020008E3020008E3020008E3020008EA
:10026000E3020008E3020008E3020008E3020008DA
:10027000E3020008E3020008E3020008E3020008CA
:10028000E3020008E3020008E3020008E3020008BA
:10029000E3020008E3020008E3020008E3020008AA
:1002A000E3020008E3020008E3020008E30200089A
:1002B000E3020008E3020008E3020008E30200088A
:1002C000E3020008E3020008E3020008E30200087A
:1002D000E3020008E3020008E3020008E30200086A
:1002E00002E000F000F8FEE772B6374880F30888B5
:1002F000364880F3098836483649086040F20000E5
:10030000CCF200004EF63471CEF200010860BFF36B
:100310004F8FBFF36F8F40F20000C0F2F0004EF637
:100320008851CEF200010860BFF34F8FBFF36F8F8B
:100330004FF00000E1EE100A4EF63C71CEF20001E3
:100340000860062080F31488BFF36F8F02F006FD6B
:1003500003F04EFE4FF055301F491B4A91423CBFFF
:1003600041F8040BFAE71D49184A91423CBF41F895
:10037000040BFAE71A491B4A1B4B9A423EBF51F83D
:10038000040B42F8040BF8E700201849184A914280
:100390003CBF41F8040BFAE702F01EFD03F0ACFE8F
:1003A000144C154DAC4203DA54F8041B8847F9E7A6
:1003B00000F0D2F8114C124DAC4203DA54F8041B91
:1003C0008847F9E702F006BD000600200022002061
:1003D0000000000808ED00E00000002000060020FA
:1003E00040490008002200205C22002060220020FA
:1003F00004440020E0020008E0020008E0020008D7
:10040000E00200082DE9F04F2DED108AC1F80CD064
:10041000D0F80CD0BDEC108ABDE8F08F002383F338
:1004200011882846A047002001F0E6FEFEE701F013
:100430006BFE00DFFEE70000032A70B515D940EA25
:10044000010C1CF0030F04460B4621D1194620462F
:100450000E680568B54204F1040403F1040317D1E2
:10046000043A032A20461946F0D8541EA2B100F1DE
:10047000FF3C013901E0C3180CD01CF801EF11F862
:10048000012F9645A4EB0C03F5D0AEEB020070BD36
:10049000541EECE7184670BD104670BD80EA01029C
:1004A000844612F0030F4FD111F0030F32D14DF8F3
:1004B000044D11F0040F51F8043B0BD0A3F10132AD
:1004C0009A4312F0803F04BF4CF8043B51F8043BC0
:1004D00016D100BF51F8044BA3F101329A4312F038
:1004E000803FA4F101320BD14CF8043BA24312F03F
:1004F000803F04BF51F8043B4CF8044BEAD023463C
:100500000CF8013B13F0FF0F4FEA3323F8D15DF8ED
:10051000044B704711F0010F06D011F8012B0CF8B5
:10052000012B002A08BF704711F0020FBFD031F82D
:10053000022B12F0FF0F16BF2CF8022B8CF80020B4
:1005400012F47F4FB3D1704711F8012B0CF8012B37
:10055000002AF9D1704700BF38B500F0C5FC00F0A3
:1005600067FE02F055FB054602F088FB0446C0B961
:100570000E4B9D4217D001339D4241F2883512BF88
:10058000044600250124002002F04CFB0CB100F0D1
:1005900073F800F021FE284600F01CF900F06CF81A
:1005A000F9E70025EFE70546EDE700BF010007B0DA
:1005B00008B500F06BFCA0F120035842584108BD7B
:1005C00007B5042101900DEB010000F07DFC03B0A4
:1005D0005DF804FB38B5302383F3118817480368AE
:1005E0000BB101F0D5FE0023154A4FF47A71134880
:1005F00001F0C4FE002383F31188124C236813B169
:100600002368013B2360636813B16368013B636047
:100610000D4D2B7833B963687BB9022000F03CFDA7
:10062000322363602B78032B07D163682BB9022038
:1006300000F032FD4FF47A73636038BD6022002011
:10064000D50500088023002078220020084B187070
:1006500003280CD8DFE800F008050208022000F0AB
:1006600009BD022000F0F4BC024B00225A60704722
:100670007822002080230020F8B5504B504A1C46B9
:100680001968013100F0998004339342F8D162680F
:100690004C4B9A4240F291804B4B9B6803F10063B4
:1006A00003F500339A4280F08880002000F042FC7D
:1006B0000220FFF7CBFF454B0021D3F8E820C3F819
:1006C000E810D3F81021C3F81011D3F81021D3F893
:1006D000EC20C3F8EC10D3F81421C3F81411D3F8AC
:1006E0001421D3F8F020C3F8F010D3F81821C3F880
:1006F0001811D3F81821D3F8802042F00062C3F813
:100700008020D3F8802022F00062C3F88020D3F844
:100710008020D3F8802042F00072C3F88020D3F804
:10072000802022F00072C3F88020D3F8803072B6A7
:100730004FF0E023C3F8084DD4E90004BFF34F8F16
:10074000BFF36F8F224AC2F88410BFF34F8F5369F3
:1007500023F480335361BFF34F8FD2F8803043F6D8
:10076000E076C3F3C905C3F34E335B0103EA060C1D
:1007700029464CEA81770139C2F87472F9D2203BDC
:1007800013F1200FF2D1BFF34F8FBFF36F8FBFF381
:100790004F8FBFF36F8F536923F4003353610023EE
:1007A000C2F85032BFF34F8FBFF36F8F302383F304
:1007B0001188854680F308882047F8BD00000208AC
:1007C00020000208FFFF0108002200200044025818
:1007D00000ED00E02DE9F04F95B0DFF8D89220222F
:1007E000FF21029004A8D9F8085000F09FFCA84A05
:1007F0001378A3B90121A74811700360302383F354
:10080000118803680BB101F0C3FD0023A24A4FF425
:100810007A71A04801F0B2FD002383F31188029B96
:1008200013B19E4B029A1A609D4A1378032B03D092
:1008300000231370994A53604FF0000B029C5E46F0
:10084000DA46CDF804B0012000F014FC24B1934B3B
:100850001B68002B00F02882002000F017FBB0F18D
:100860000008F3DB012000F0F3FBA8F121031F2BAC
:10087000E9D801A252F823F0F90800081509000888
:10088000A3090008470800084708000847080008AF
:100890002D0A00081F0C0008110B00086D0B000842
:1008A000930B0008B90B000847080008CB0B0008A1
:1008B000EF0B0008670C00088109000847080008D2
:1008C000AF0C000805090008810900084708000866
:1008D0006D0B000847080008470800084708000893
:1008E00047080008470800084708000847080008AC
:1008F00047080008A30900080220FFF759FE002856
:1009000040F0FF81029B02216648BBF1000F08BF47
:100910001C4640E04FF47A7000F0B8FA071EF1DB95
:100920000220FFF745FE0028ECD0013F052F00F222
:10093000EA81DFE807F003070A0D10330520FFF70F
:100940003FFE14E0D9F80000F9E7D9F80400F6E713
:10095000D9F80800F3E74FF01C08404608F10408F6
:1009600000F0EAFAFFF72CFEB8F12C0FF5D10120C8
:10097000019B4FF0000A00FA07F71F43FBB20193F7
:1009800000F020FC2EB1019B03F00B030B2B08BFE2
:1009900000240221444800F097FA54E7D9F80C00EB
:1009A000CDE7002EAED0019B03F00B030B2BA9D19A
:1009B0000220FFF7FDFD07460028A3D001200026F6
:1009C00000F0B8FA0220FFF741FE1FFA86FB5846F6
:1009D00000F0C0FA044688B1A8F14002584601363A
:1009E0005142514100F0C6FA0028EED1BB46044600
:1009F00002212E483E4600F067FA24E725460120F2
:100A0000FFF724FED9F80830AB4207D9284600F09A
:100A100093FA013040F07A810435F3E70025204B4A
:100A2000BB463E461D701D4B5D60A9E7002E3FF49E
:100A300069AF019B03F00B030B2B7FF463AF022024
:100A4000FFF704FE322000F021FAB0F10008FFF6B3
:100A500059AF18F003077FF455AF08EB0503D9F839
:100A6000082093423FF64EAFB8F5807F3FF74AAF7C
:100A70000F4BB84503931FDD4FF47A7000F006FA70
:100A80000028FFF63FAF039B013703F8010BF0E7A7
:100A90007C23002060220020D50500088023002050
:100AA00078220020E4440008DC440008E044000808
:100AB0007C22002000220020C820FFF779FD074695
:100AC00000283FF41FAF1F2D11D8C5F1200204AB41
:100AD00025F003008F494245184428BF424603923F
:100AE00000F0FEFA039AFF218A4800F01FFB4FEA4C
:100AF000A803C8F3870287492846039300F01EFB2A
:100B0000064600283FF474AF039B05EB830537E7E7
:100B10000220FFF74DFD00283FF4F4AE00F048FA44
:100B200000283FF4EFAE0027B846D9F80830BB42A2
:100B300018D91F2F11D8049B01330ED027F00303BF
:100B400050336B4453F8403C0C93404604220CA9AC
:100B5000043700F07FFB8046E7E7384600F0ECF909
:100B60000C90F2E74046FFF72BFD09E700236421D4
:100B70000CA80C9300F09EF900287FF4C3AE02206D
:100B8000FFF716FD00283FF4BDAE0C9800F006FA02
:100B9000E9E7002364210CA80C9300F08BF90028EE
:100BA0007FF4B0AE0220FFF703FD00283FF4AAAEA9
:100BB0000C9800F0F5F9D6E70220FFF7F9FC0028C1
:100BC0003FF4A0AE00F004FACDE70220FFF7F0FCFE
:100BD00000283FF497AE0CA9142000F0FFF9039011
:100BE000FFF7EEFC03990CA800F06EF9C8E60220AE
:100BF000FFF7DEFC00283FF485AE474B0CAF03F156
:100C0000100C1868083353F8041C3A46634503C2B5
:100C10001746F6D11020FFF7D3FC1021E3E732206E
:100C200000F034F9071EFFF66DAEBB077FF46AAE25
:100C300007EB0A03D9F8082093423FF663AE02207F
:100C4000FFF7B6FC00283FF45DAE27F003075744DA
:100C5000BA453FF495AE50460AF1040A00F06CF92B
:100C6000FFF7AEFCF4E74FF47A70FFF7A1FC002821
:100C70003FF448AE00F09CF9002849D0049B0133B2
:100C80000BD0082204A9002000F058FA00283FD019
:100C90002022FF2104A800F049FA2048022100F098
:100CA00013F91F4801F0AEFA15B0BDE8F08F002E21
:100CB0003FF428AE019B03F00B030B2B7FF422AE15
:100CC000002364210CA80C9300F0F4F807460028D8
:100CD0007FF418AE0220FFF76BFC804600283FF43B
:100CE00011AE02210D4800F0EFF841F2883001F01A
:100CF00089FA0C9800F09AFA46463C4600F062FAEF
:100D0000A1E506463CE64FF0000AFBE5BB466FE670
:100D100037466DE67C220020C8440008DC44000809
:100D2000A08601000F4B70B51B780C460133DBB277
:100D3000012B11D80C4D4FF47A732968A2FB0332B2
:100D400022460E6A01462846B047844204D1074B2A
:100D5000002201201A7070BD4FF4FA7001F052FAAF
:100D60000020F8E710220020B0260020B423002045
:100D700000232DE9F0471A4605468846012019460A
:100D800000F068FC0446802001F0D2FE07460028EF
:100D900061D0002C5FD03B4E28464FF0800A73692B
:100DA00043F0C0637361D6F8143143F0C063C6F8F2
:100DB000143101F041FD05EB080200FB05F34FF48F
:100DC000D06C50434FF03D0E834233D23269520112
:100DD00043D4D6F8102151013FD4216803F10062B9
:100DE0008A602268D7602268C2F804A02268C2F82C
:100DF00000C0D4F80090D9F8002042F00102C9F8F0
:100E00000020D4F80090D9F8002022F01E02C9F882
:100E10000020D4F80090D9F80020D207FBD494F831
:100E20000C90803361680EFA09F20A60CCE700206A
:100E300001F0E0FD204600F04DFC384601F0AEFE2A
:100E4000104B5A6942F0C0625A61D3F8142142F043
:100E5000C062C3F81421BDE8F0870B4B9A6A42F4D4
:100E600000729A629A6A42F400429A6261B600265F
:100E7000012001F0BFFDB045D9D9A819013601F014
:100E8000F3FCF8E70020005200ED00E0002307B576
:100E9000024601210DF107008DF80730FFF742FFF0
:100EA00020B19DF8070003B05DF804FB4FF0FF3060
:100EB000F9E700000A46042108B5FFF733FF80F088
:100EC0000100C0B2404208BD30B4054C0A4601469C
:100ED00023682046DD69034BAC4630BC604700BF49
:100EE000B0260020A086010070B5104C0025104EE1
:100EF00001F0A6FC20803068238883420CD80025AE
:100F00002088013801F098FC23880544013BB5F5A1
:100F1000802F2380F4D370BD01F08EFC336805442C
:100F20000133B5F5003F3360E5D3E8E7B623002091
:100F30008823002001F05EBD00F1006000F5003064
:100F40000068704700F10060920000F5003001F089
:100F5000D3BC0000054B1A68054B1B889B1A8342C3
:100F600002D9104401F068BC00207047882300209B
:100F7000B623002038B50446074D29B1286820441F
:100F8000BDE8384001F070BC2868204401F05AFCEC
:100F90000028F3D038BD00BF882300200020704710
:100FA00000F1FF5000F58F10D0F8000870470000E6
:100FB000064991F8243033B100230822086A81F8E9
:100FC0002430FFF7BFBF0120704700BF8C230020F3
:100FD000014B1868704700BF0010005C194B0138C6
:100FE0000322084470B51D68174BC5F30B042D0C84
:100FF0001E88A6420BD15C680A46013C8242134619
:101000000FD214F9016F4EB102F8016BF6E7013A05
:1010100003F10803ECD181420B4602D22C2203F8E3
:10102000012B0424094A1688AE4204D1984284BF99
:10103000967803F8016B013C02F10402F3D1581ACF
:1010400070BD00BF0010005C142200201445000891
:10105000022804D1054B4FF400429A6170470128E1
:10106000FCD1034B4FF40062F7E700BF00040258C5
:10107000000C0258022804D1054B4FF000429A613F
:1010800070470128FCD1034B4FF00062F7E700BF27
:1010900000040258000C0258022805D1064A536980
:1010A00083F40043536170470128FCD1034A53691C
:1010B00083F40063F6E700BF00040258000C0258F6
:1010C00070B504464FF47A764CB1412C254628BFC2
:1010D000412506FB05F0641B01F094F8F4E770BDB0
:1010E000002310B5934203D0CC5CC4540133F9E71C
:1010F00010BD0000013810B510F9013F3BB191F966
:1011000000409C4203D11AB10131013AF4E71AB10F
:1011100091F90020981A10BD1046FCE703460246DC
:10112000D01A12F9011B0029FAD170470244034674
:10113000934202D003F8011BFAE770472DE9F84308
:101140001F4D14460746884695F8242052BBDFF809
:1011500070909CB395F824302BB92022FF2148468B
:101160002F62FFF7E3FF95F824004146C0F1080223
:1011700005EB8000A24228BF2246D6B29200FFF7BC
:10118000AFFF95F82430A41B17441E449044E4B2EA
:10119000F6B2082E85F82460DBD1FFF709FF00289E
:1011A000D7D108E02B6A03EB82038342CFD0FFF74D
:1011B000FFFE0028CBD10020BDE8F8830120FBE72B
:1011C0008C230020024B1A78024B1A70704700BF24
:1011D000B42300201022002010B5114C114800F05B
:1011E0002BFB21460F4800F053FB24684FF47A7024
:1011F000D4F89020D2F8043843F00203C2F804383F
:10120000FFF75EFF0849204600F050FCD4F890201C
:10121000D2F8043823F00203C2F8043810BD00BF2E
:10122000D0460008B0260020D846000870470000CD
:1012300008B571B6054B1988054B1888FFF798FD5E
:1012400002210E20FFF794FD61B608BDB6230020F1
:101250008823002030B50A44084D91420DD011F882
:10126000013B5840082340F30004013B2C4013F09D
:10127000FF0384EA5000F6D1EFE730BD2083B8EDDC
:1012800008B5074B074A196801F03D01996053689A
:101290000BB190689847BDE8084001F035BD00BF2C
:1012A00000000240B823002008B5084B19688909DE
:1012B00001F03D018A019A60054AD3680BB11069BB
:1012C0009847BDE8084001F01FBD00BF0000024084
:1012D000B823002008B5084B1968090C01F03D013E
:1012E0000A049A60054A53690BB190699847BDE8B2
:1012F000084001F009BD00BF00000240B8230020F3
:1013000008B5084B1968890D01F03D018A059A60FE
:10131000054AD3690BB1106A9847BDE8084001F04F
:10132000F3BC00BF00000240B823002008B5074B03
:10133000074A596801F03D01D960536A0BB1906AC0
:101340009847BDE8084001F0DFBC00BF0000024044
:10135000B823002008B5084B5968890901F03D0100
:101360008A01DA60054AD36A0BB1106B9847BDE871
:10137000084001F0C9BC00BF00000240B8230020B3
:1013800008B5084B5968090C01F03D010A04DA6000
:10139000054A536B0BB1906B9847BDE8084001F0CC
:1013A000B3BC00BF00000240B823002008B5084BC2
:1013B0005968890D01F03D018A05DA60054AD36B51
:1013C0000BB1106C9847BDE8084001F09DBC00BF10
:1013D00000000240B823002008B5074B074A1968EF
:1013E00001F03D019960536C0BB1906C9847BDE8DA
:1013F000084001F089BC00BF00040240B82300206F
:1014000008B5084B1968890901F03D018A019A6005
:10141000054AD36C0BB1106D9847BDE8084001F048
:1014200073BC00BF00040240B823002008B5084B7D
:101430001968090C01F03D010A049A60054A536DD0
:101440000BB1906D9847BDE8084001F05DBC00BF4E
:1014500000040240B823002008B5084B1968890D24
:1014600001F03D018A059A60054AD36D0BB1106EFB
:101470009847BDE8084001F047BC00BF00040240A7
:10148000B823002008B5074B074A596801F03D0111
:10149000D960536E0BB1906E9847BDE8084001F0DB
:1014A00033BC00BF00040240B823002008B5084B3D
:1014B0005968890901F03D018A01DA60054AD36E55
:1014C0000BB1106F9847BDE8084001F01DBC00BF8C
:1014D00000040240B823002008B5084B5968090CE5
:1014E00001F03D010A04DA60054A536F0BB1906FB9
:1014F0009847BDE8084001F007BC00BF0004024067
:10150000B823002008B5084B5968890D01F03D014A
:101510008A05DA60054AD36F13B1D2F88000984784
:10152000BDE8084001F0F0BB00040240B8230020F1
:1015300000230C4910B51A460B4C0B6054F82300DD
:10154000026001EB430004334260402BF6D1074AAE
:101550004FF0FF339360D360C2F80834C2F80C3404
:1015600010BD00BFB8230020244500080000024041
:101570000F28F8B510D9102810D0112811D0122832
:1015800008D10F240720DFF8C8E00126DEF800505C
:10159000A04208D9002653E00446F4E70F240020B7
:1015A000F1E70724FBE706FA00F73D424AD1264C53
:1015B0004FEA001C3D4304EB00160EEBC000CEF8D2
:1015C0000050C0E90123FBB273B12048D0F8D830F5
:1015D00043F00103C0F8D830D0F8003143F00103E4
:1015E000C0F80031D0F8003117F47F4F0ED0174803
:1015F000D0F8D83043F00203C0F8D830D0F800312A
:1016000043F00203C0F80031D0F8003154F80C0068
:10161000036823F01F030360056815F00105FBD183
:1016200004EB0C033D2493F80CC05F6804FA0CF43F
:101630003C6021240560446112B1987B00F054F8AD
:101640003046F8BD0130A3E72445000800440258A5
:10165000B823002010B5302484F31188FFF788FFE9
:10166000002383F3118810BD10B50446807B00F081
:1016700051F801231549627B03FA02F20B6823EA51
:101680000203DAB20B6072B9114AD2F8D81021F015
:101690000101C2F8D810D2F8001121F00101C2F8FE
:1016A0000011D2F8002113F47F4F0ED1084BD3F86C
:1016B000D82022F00202C3F8D820D3F8002122F06B
:1016C0000202C3F80021D3F8003110BDB823002076
:1016D0000044025808B5302383F31188FFF7C4FF94
:1016E000002383F3118808BD090100F16043012242
:1016F00003F56143C9B283F8001300F01F039A4059
:1017000043099B0003F1604303F56143C3F8802163
:101710001A60704700F01F0301229A40430900F14C
:1017200060409B0000F5614003F1604303F56143B5
:10173000C3F88020C3F88021002380F8003370476D
:10174000026843681143016003B118477047000005
:1017500013B5406B00F58054D4F8A4381A6811789A
:10176000042914D1017C022911D11979012312898C
:101770008B4013420BD101A94C3002F0B5F9D4F8DB
:10178000A4480246019B2179206800F0DFF902B0ED
:1017900010BD0000143002F037B900004FF0FF33E5
:1017A000143002F031B900004C3002F009BA0000E8
:1017B0004FF0FF334C3002F003BA0000143002F057
:1017C00005B900004FF0FF31143002F0FFB80000FF
:1017D0004C3002F0D5B900004FF0FF324C3002F02F
:1017E000CFB900000020704710B500F58054D4F840
:1017F000A4381A681178042917D1017C022914D160
:101800005979012352898B4013420ED1143002F0D2
:1018100097F8024648B1D4F8A4484FF44073617970
:101820002068BDE8104000F07FB910BD406BFFF7A5
:10183000DBBF0000704700007FB5124B0125042676
:10184000044603600023057400F1840243602946C6
:10185000C0E902330C4B0290143001934FF44073F3
:10186000009602F049F8094B04F69442294604F127
:101870004C000294CDE900634FF4407302F010F97C
:1018800004B070BD244600082D1800085117000848
:101890000A68302383F311880B790B3342F8230055
:1018A0004B79133342F823008B7913B10B3342F891
:1018B000230000F58053C3F8A4180223037400200A
:1018C00080F311887047000038B5037F044613B1D8
:1018D00090F85430ABB90125201D0221FFF730FFED
:1018E00004F114006FF00101257700F0B3FC04F15E
:1018F0004C0084F854506FF00101BDE8384000F00E
:10190000A9BC38BD10B5012104460430FFF718FF0B
:101910000023237784F8543010BD000038B5044606
:101920000025143002F000F804F14C00257702F095
:10193000CFF8201D84F854500121FFF701FF204605
:10194000BDE83840FFF750BF90F8803003F06003E7
:10195000202B06D190F881200023212A03D81F2AAA
:1019600006D800207047222AFBD1C0E91D3303E0CE
:10197000034A426707228267C3670120704700BF9E
:101980002C22002037B500F58055D5F8A4381A6808
:10199000117804291AD1017C022917D11979012360
:1019A00012898B40134211D100F14C04204602F001
:1019B0004FF958B101A9204602F096F8D5F8A4488D
:1019C0000246019B2179206800F0C0F803B030BDC9
:1019D00001F10B03F0B550F8236085B004460D46C5
:1019E000FEB1302383F3118804EB8507301D0821F5
:1019F000FFF7A6FEFB6806F14C005B691B681BB194
:101A0000019002F07FF8019803A902F06DF80246F8
:101A100048B1039B2946204600F098F8002383F341
:101A2000118805B0F0BDFB685A691268002AF5D02C
:101A30001B8A013B1340F1D104F18002EAE7000068
:101A4000133138B550F82140ECB1302383F31188BD
:101A500004F58053D3F8A4281368527903EB82036A
:101A6000DB689B695D6845B104216018FFF768FE7B
:101A7000294604F1140001F06DFF2046FFF7B4FE83
:101A8000002383F3118838BD7047000001F03ABA93
:101A900001234022002110B5044600F8303BFFF737
:101AA00045FB0023C4E9013310BD000010B530230D
:101AB000044683F311882422416000210C30FFF793
:101AC00035FB204601F040FA02230020237080F30A
:101AD000118810BD70B500EB8103054650690E46B4
:101AE0001446DA6018B110220021FFF71FFBA0692D
:101AF00018B110220021FFF719FB31462846BDE836
:101B0000704001F027BB000083682022002103F011
:101B1000011310B5044683601030FFF707FB204621
:101B2000BDE8104001F0A2BBF0B4012500EB810438
:101B300047898D40E4683D43A469458123600023C3
:101B4000A2606360F0BC01F0BFBB0000F0B40125EF
:101B500000EB810407898D40E4683D436469058199
:101B600023600023A2606360F0BC01F035BC00007C
:101B700070B5022300250446242203702946C0F8CC
:101B800088500C3040F8045CFFF7D0FA204684F807
:101B9000705001F073FA63681B6823B12946204630
:101BA000BDE87040184770BD0378052B10B504469A
:101BB0000AD080F88C300523037043681B680BB192
:101BC000042198470023A36010BD00000178052977
:101BD00006D190F88C20436802701B6803B1184747
:101BE0007047000070B590F87030044613B10023C0
:101BF00080F8703004F18002204601F05BFB6368DE
:101C00009B68B3B994F8803013F0600535D000219B
:101C1000204601F04DFE0021204601F03DFE6368A4
:101C20001B6813B1062120469847062384F87030BC
:101C300070BD204698470028E4D0B4F88630A26FE3
:101C40009A4288BFA36794F98030A56F002B4FF0AC
:101C5000300380F20381002D00F0F280092284F825
:101C6000702083F3118800212046D4E91D23FFF75B
:101C70006DFF002383F31188DAE794F8812003F0E5
:101C80007F0343EA022340F20232934200F0C58010
:101C900021D8B3F5807F48D00DD8012B3FD0022B3F
:101CA00000F09380002BB2D104F188026267022217
:101CB000A267E367C1E7B3F5817F00F09B80B3F5CE
:101CC000407FA4D194F88230012BA0D1B4F88830A1
:101CD00043F0020332E0B3F5006F4DD017D8B3F5EF
:101CE000A06F31D0A3F5C063012B90D86368204664
:101CF00094F882205E6894F88310B4F88430B0477A
:101D0000002884D0436863670368A3671AE0B3F5CB
:101D1000106F36D040F6024293427FF478AF5C4BAE
:101D200063670223A3670023C3E794F88230012B83
:101D30007FF46DAFB4F8883023F00203A4F8883044
:101D4000C4E91D55E56778E7B4F88030B3F5A06FB6
:101D50000ED194F88230204684F88A3001F0ECF9F4
:101D600063681B6813B10121204698470323237041
:101D70000023C4E91D339CE704F18B03636701234F
:101D8000C3E72378042B10D1302383F31188204636
:101D9000FFF7BAFE85F311880321636884F88B503E
:101DA00021701B680BB12046984794F88230002BB5
:101DB000DED084F88B300423237063681B68002B0B
:101DC000D6D0022120469847D2E794F884302046A6
:101DD0001D0603F00F010AD501F05EFA012804D0B8
:101DE00002287FF414AF2B4B9AE72B4B98E701F0B6
:101DF00045FAF3E794F88230002B7FF408AF94F8AB
:101E0000843013F00F01B3D01A06204602D501F03A
:101E100067FDADE701F058FDAAE794F88230002B8A
:101E20007FF4F5AE94F8843013F00F01A0D01B06B8
:101E3000204602D501F03CFD9AE701F02DFD97E721
:101E4000142284F8702083F311882B462A462946F1
:101E50002046FFF769FE85F31188E9E65DB115229A
:101E600084F8702083F3118800212046D4E91D23D3
:101E7000FFF75AFEFDE60B2284F8702083F31188E9
:101E80002B462A4629462046FFF760FEE3E700BFBF
:101E9000544600084C4600085046000838B590F8F3
:101EA00070300446002B3ED0063BDAB20F2A34D8FD
:101EB0000F2B32D8DFE803F03731310822323131CD
:101EC0003131313131313737856FB0F886309D424D
:101ED00014D2C3681B8AB5FBF3F203FB12556DB92C
:101EE000302383F311882B462A462946FFF72EFE1E
:101EF00085F311880A2384F870300EE0142384F8E7
:101F00007030302383F31188002320461A46194687
:101F1000FFF70AFE002383F3118838BDC36F03B1B6
:101F200098470023E7E70021204601F0C1FC00218B
:101F3000204601F0B1FC63681B6813B106212046FE
:101F400098470623D7E7000010B590F87030044694
:101F5000142B29D017D8062B05D001D81BB110BDE2
:101F6000093B022BFBD80021204601F0A1FC0021F7
:101F7000204601F091FC63681B6813B106212046DE
:101F80009847062319E0152BE9D10B2380F8703010
:101F9000302383F3118800231A461946FFF7D6FD34
:101FA000002383F31188DAE7C3689B695B68002B21
:101FB000D5D1C36F03B19847002384F87030CEE7C2
:101FC00000238268037503691B6899689142FBD2FC
:101FD0005A6803604260106058607047002382684E
:101FE000037503691B6899689142FBD85A680360BE
:101FF000426010605860704708B50846302383F38C
:1020000011880A7D0023052A06D8DFE802F00B05B7
:102010000503120E826913604FF0FF338361FFF7EF
:10202000CFFF002383F3118808BD826993680133D1
:102030009360D0E9003213605A60EDE7FFF7C0BF4C
:1020400038B50A4B1C68DD682875226853601A6031
:102050000122DC60A3682275934201D100F018FED2
:1020600029462046BDE83840FEF7CCB94024002080
:102070000C4B30B5DD684B1C87B004460FD02B46A7
:10208000094A684600F07AF92046FFF7D9FF009B1D
:1020900013B1684600F07CF9A86907B030BDFFF7BE
:1020A000CFFFF9E740240020F91F000870B50F4E5C
:1020B00004468161F36881689A68914203D8BDE85B
:1020C0007040FFF77DBF1846FFF788FF836805461D
:1020D000012B01D100F0DEFD012329462046F460EA
:1020E0002375BDE87040FEF78DB900BF4024002085
:1020F000044B1A68DB6890689B68984294BF002084
:10210000012070474024002038B50B4B1C68DD6867
:10211000226853601A600122DC602275AB6893422A
:1021200001D100F0B7FD2846FFF758FF01462046D1
:10213000BDE83840FEF766B94024002038B50123D9
:10214000084C00252370656001F0BEFD01F0E4FD40
:102150000549064801F0B8FE0223237085F3118873
:1021600038BD00BFA82600205C460008402400209F
:1021700000F044B9034A516853685B1A9842FBD88F
:10218000704700BF001000E08B6002230861084622
:102190008B8270478368A3F1840243F8142C026990
:1021A00043F8442C426943F8402C094A43F8242C54
:1021B000C268A3F1200043F8182C022203F80C2C6B
:1021C000002203F80B2C034A43F8102C704700BF81
:1021D0001D0400084024002008B5FFF7DBFFBDE820
:1021E0000840FFF72BBF0000024BDB6898610F200F
:1021F000FFF726BF40240020302383F31188FFF728
:10220000F3BF000008B50146302383F3118808208E
:10221000FFF72EFF002383F3118808BD064BDB6810
:1022200039B1426818605A60136043600420FFF7B8
:102230001FBF4FF0FF3070474024002003689842D2
:1022400006D01A680260506018469961FFF7F6BE22
:102250007047000038B504460D462068844200D11E
:1022600038BD036823605C608561FFF7E7FEF4E733
:10227000036810B59C68A2420CD85C688A600B6049
:102280004C602160596099688A1A9A604FF0FF3358
:10229000836010BD121B1B68ECE700000A2938BFE1
:1022A0000A2170B504460D460A26601901F006FDA4
:1022B00001F0EEFC041BA54203D8751C04462E4613
:1022C000F3E70A2E04D90120BDE8704001F03CBEBE
:1022D00070BD0000F8B5144B0D460A2A4FF00A07EE
:1022E000D96103F11001826038BF0A224160196987
:1022F0001446016048601861A81801F0CFFC01F095
:10230000C7FC431B0646A34206D37C1C281927465C
:10231000354601F0D3FCF2E70A2F04D90120BDE8CD
:10232000F84001F011BEF8BD40240020F8B5064683
:102330000D4601F0ADFC0F4A134653F8107F9F4243
:1023400006D12A4601463046BDE8F840FFF7C2BF35
:10235000D169BB68441A2C1928BF2C46A34202D964
:102360002946FFF79BFF224631460348BDE8F84067
:10237000FFF77EBF4024002050240020C0E9032343
:10238000002310B45DF8044B4361FFF7CFBF00009A
:1023900010B5194C236998420DD08168D0E90032FC
:1023A00013605A609A680A449A60002303604FF0F1
:1023B000FF33A36110BD0268234643F8102F53601A
:1023C0000022026022699A4203D1BDE8104001F068
:1023D0006FBC936881680B44936001F059FC2269DB
:1023E000E1699268441AA242E4D91144BDE8104060
:1023F000091AFFF753BF00BF402400202DE9F04722
:10240000DFF8BC8008F110072C4ED8F8105001F00E
:102410003FFCD8F81C40AA68031B9A423ED81444DB
:102420004FF00009D5E90032C8F81C4013605A602B
:10243000C5F80090D8F81030B34201D101F038FC53
:1024400089F31188D5E9033128469847302383F36F
:1024500011886B69002BD8D001F01AFC6A69A0EBD7
:10246000040982464A450DD2022001F06DFD00228A
:10247000D8F81030B34208D151462846BDE8F0479D
:10248000FFF728BF121A2244F2E712EB0909294686
:10249000384638BF4A46FFF7EBFEB5E7D8F81030AC
:1024A000B34208D01444C8F81C00211AA960BDE842
:1024B000F047FFF7F3BEBDE8F08700BF50240020CF
:1024C0004024002000207047FEE700007047000015
:1024D0004FF0FF307047000002290CD0032904D0D0
:1024E0000129074818BF00207047032A05D805486E
:1024F00000EBC2007047044870470020704700BFDF
:10250000344700083C220020E846000870B59AB025
:1025100005460846144601A900F0C2F801A8FEF7D6
:10252000FDFD431C0022C6B25B001046C5E9003425
:1025300023700323023404F8013C01ABD1B202340E
:102540008E4201D81AB070BD13F8011B013204F895
:10255000010C04F8021CF1E708B5302383F311885D
:102560000348FFF70FFA002383F3118808BD00BF6B
:10257000B026002090F8803003F01F02012A07D116
:1025800090F881200B2A03D10023C0E91D3315E008
:1025900003F06003202B08D1B0F884302BB990F8F9
:1025A0008120212A03D81F2A04D8FFF7CDB9222A77
:1025B000EBD0FAE7034A426707228267C36701202C
:1025C000704700BF3322002007B5052917D8DFE880
:1025D00001F0191603191920302383F31188104ACA
:1025E00001210190FFF776FA019802210D4AFFF7C9
:1025F00071FA0D48FFF792F9002383F3118803B0B5
:102600005DF804FB302383F311880748FFF75CF97A
:10261000F2E7302383F311880348FFF773F9EBE700
:1026200088460008AC460008B026002038B50C4D9E
:102630000C4C2A460C4904F10800FFF767FF05F12E
:10264000CA0204F110000949FFF760FF05F5CA72DC
:1026500004F118000649BDE83840FFF757BF00BF36
:10266000883F00203C22002068460008724600088F
:102670007D46000870B5044608460D46FEF74EFD3F
:10268000C6B22046013403780BB9184670BD3246F5
:102690002946FEF72FFD0028F3D10120F6E70000C0
:1026A0002DE9F84F05460C46FEF738FD2C49C6B219
:1026B0002846FFF7DFFF08B10336F6B2294928465E
:1026C000FFF7D8FF08B11036F6B2632E0DD8DFF849
:1026D0009080DFF89090244FDFF894A0DFF894B05A
:1026E0002E7846B92670BDE8F88F29462046BDE809
:1026F000F84FFDF7D3BE252E2ED10722414628469E
:10270000FEF7F8FC70B9DBF8003007350A3444F8FE
:102710000A3CDBF8043044F8063CBBF8083024F8E7
:10272000023CDDE7082249462846FEF7E3FC98B95B
:10273000A21C0E4B197802320909C95D02F8041C6B
:1027400013F8011B01F00F015345C95D02F8031C8A
:10275000F0D118340835C3E7013504F8016BBFE741
:10276000544700087D4600086747000800E8F11F4D
:102770000CE8F11F5C470008BFF34F8F044B1A6948
:102780005107FCD1D3F810215207F8D1704700BF90
:102790000020005208B50D4B1B78ABB9FFF7ECFFDA
:1027A0000B4BDA68D10704D50A4A5A6002F1883225
:1027B0005A60D3F80C21D20706D5064AC3F8042183
:1027C00002F18832C3F8042108BD00BFE6410020B1
:1027D000002000522301674508B5114B1B78F3B95F
:1027E000104B1A69510703D5DA6842F04002DA60EB
:1027F000D3F81021520705D5D3F80C2142F040023E
:10280000C3F80C21FFF7B8FF064BDA6842F001026B
:10281000DA60D3F80C2142F00102C3F80C2108BDA4
:10282000E6410020002000520F289ABF00F580608A
:1028300040040020704700004FF400307047000053
:10284000102070470F2808B50BD8FFF7EDFF00F5F3
:1028500000330268013204D104308342F9D10120EF
:1028600008BD0020FCE700000F2838B505463FD81A
:10287000FFF782FF1F4CFFF78DFF4FF0FF33072854
:102880006361C4F814311DD82361FFF775FF03029B
:1028900043F02403E360E36843F08003E3602369CB
:1028A0005A07FCD42846FFF767FFFFF7BDFF4FF438
:1028B000003100F0C5F92846FFF78EFFBDE838402B
:1028C000FFF7C0BFC4F81031FFF756FFA0F10803AF
:1028D0001B0243F02403C4F80C31D4F80C3143F04C
:1028E0008003C4F80C31D4F810315B07FBD4D9E76E
:1028F000002038BD002000522DE9F84F04460D4657
:10290000104644EA0203DE0602D00020BDE8F88F3C
:1029100020F01F00DFF8D4B0DFF8D4A0FFF73AFFB3
:1029200005EB0008454503D10120FFF755FFEDE712
:10293000202229462046FDF77FFD10B9203420359E
:10294000F0E7234604F120021F68791CDDD104332F
:102950009342F9D104F178432048214EB3F5801F0A
:10296000204B38BF184603F1F80332BFD946D14691
:102970001E46FFF701FF0760A4EB050C336805F165
:102980001C0143F0020333602B1FD9F8007017F0CD
:102990000507FAD153F8042F8B424CF80320F4D1E9
:1029A000BFF34F8FFFF7E8FE4FF0FF33036033684C
:1029B00023F002033360BFF34F8F0B4BC3F85C422D
:1029C000BFF34F8FBFF36F8F202229462046FDF7BC
:1029D00033FD0028B2D03846A7E700BF14210052CB
:1029E0000C2000521420005200ED00E01020005294
:1029F0001021005210B5084C237828B11BB9FFF7FD
:102A0000C9FE0123237010BD002BFCD02070BDE84F
:102A10001040FFF7E1BE00BFE64100202DE9F04F76
:102A20000D4685B0814658B111F00D0614BF202225
:102A3000082211F00803019304D0431E03426AD018
:102A4000002435E0002E37D009F11F0121F01F09C5
:102A50004FF00108324F05F00403DFF8D0A005EA7B
:102A6000080BBBF1000F32D07869C0072FD408F1F2
:102A700001080C37B8F1060FF3D19EB9294D49462C
:102A8000A819019201F06AF9044600283AD11836D3
:102A9000019A782EF3D1494601F060F904460028E6
:102AA00030D1019A4946204801F058F9044668BBE4
:102AB000204605B0BDE8F08F0029C9D1014628465F
:102AC000029201F04BF90446E0B9029AC0E713B153
:102AD00078694107CBD5AC0702D578698007C6D5A0
:102AE000019911B178690107C1D51820494600FB49
:102AF00008A0CDE9022301F031F90446DDE9022303
:102B00000028B4D04A460021204601E04A46002170
:102B1000FEF70CFBCCE70246002E95D198E700BFEC
:102B20007847000818420020E841002000420020B9
:102B30000121FFF773BF0000F8B500231A461A60A1
:102B40000433B3F5806FFAD1114D01241827114ECB
:102B500007FB046001342A6955F80C1F01F0EAF8FC
:102B6000062CF5D137254FF4C0542046FFF7E0FF7F
:102B7000014628B122460848BDE8F84001F0DAB81D
:102B8000C4EBC404013D4FEAD404EED1F8BD00BF4C
:102B90007847000800420020E841002008B101F019
:102BA0004FB970470244074BD2B210B5904200D1E2
:102BB00010BD441C00B253F8200041F8040BE0B2F1
:102BC000F4E700BF504000580E4B30B51C6F240492
:102BD00005D41C6F1C671C6F44F400441C670A4C2E
:102BE00002442368D2B243F480732360074B9042BF
:102BF00000D130BD441C51F8045B00B243F82050B2
:102C0000E0B2F4E70044025800480258504000582F
:102C100007B5012201A90020FFF7C4FF019803B006
:102C20005DF804FB13B50446FFF7F2FFA04205D0A0
:102C3000012201A900200194FFF7C6FF02B010BDD8
:102C40000144BFF34F8F064B884204D3BFF34F8F2D
:102C5000BFF36F8F7047C3F85C022030F4E700BF0A
:102C600000ED00E0034B1A681AB9034AD2F8D024E9
:102C70001A607047904200200040025808B5FFF7E4
:102C8000F1FF024B1868C0F3806008BD904200203D
:102C90007047000070470000EFF30983054968336F
:102CA0004A6B22F001024A6383F30988002383F30D
:102CB0001188704700EF00E0302080F3118862B681
:102CC0000D4B0E4AD96821F4E0610904090C0A434E
:102CD0000B49DA60D3F8FC2042F08072C3F8FC2084
:102CE000084AC2F8B01F116841F0010111602022AA
:102CF000DA7783F82200704700ED00E00003FA0560
:102D000055CEACC5001000E0302310B583F3118818
:102D10000E4B5B6813F4006314D0F1EE103AEFF33E
:102D200009844FF08073683CE361094BDB6B2366D9
:102D300084F30988FFF7DCF910B1064BA36110BDDD
:102D4000054BFBE783F31188F9E700BF00ED00E0D6
:102D500000EF00E02F0400083204000870B5BFF354
:102D60004F8FBFF36F8F1A4A0021C2F85012BFF382
:102D70004F8FBFF36F8F536943F400335361BFF339
:102D80004F8FBFF36F8FC2F88410BFF34F8FD2F80D
:102D9000803043F6E074C3F3C900C3F34E335B01E4
:102DA00003EA0406014646EA81750139C2F8605219
:102DB000F9D2203B13F1200FF2D1BFF34F8F5369AB
:102DC00043F480335361BFF34F8FBFF36F8F70BDF8
:102DD00000ED00E0FEE70000214B2248224A70B5DA
:102DE000904237D3214BC11EDA1C121A22F0030283
:102DF0008B4238BF00220021FEF798F91C4A0023BD
:102E0000C2F88430BFF34F8FD2F8803043F6E074BD
:102E1000C3F3C900C3F34E335B0103EA0406014662
:102E200046EA81750139C2F86C52F9D2203B13F1A0
:102E3000200FF2D1BFF34F8FBFF36F8FBFF34F8FD0
:102E4000BFF36F8F0023C2F85032BFF34F8FBFF331
:102E50006F8F70BD53F8041B40F8041BC0E700BF20
:102E60009C4900080444002004440020044400203D
:102E700000ED00E0074BD3F8D81021EA0001C3F8B9
:102E8000D810D3F8002122EA0002C3F80021D3F8B9
:102E9000003170470044025870B5D0E92443002245
:102EA0004FF0FF359E6804EB42135101D3F800093F
:102EB000002805DAD3F8000940F08040C3F8000983
:102EC000D3F8000B002805DAD3F8000B40F080405F
:102ED000C3F8000B013263189642C3F80859C3F8CF
:102EE000085BE0D24FF00113C4F81C3870BD00003D
:102EF000890141F02001016103699B06FCD4122085
:102F0000FFF738B910B50A4C2046FEF7C1FD094B52
:102F1000C4F89030084BC4F89430084C2046FEF7B3
:102F2000B7FD074BC4F89030064BC4F8943010BD81
:102F30009442002000000840E4470008304300208D
:102F400000000440F047000870B503780546012BE7
:102F50005CD1434BD0F89040984258D1414B0E2160
:102F60006520D3F8D82042F00062C3F8D820D3F807
:102F7000002142F00062C3F80021D3F80021D3F809
:102F8000802042F00062C3F88020D3F8802022F035
:102F90000062C3F88020D3F88030FEF7A5FB324BE7
:102FA000E360324BC4F800380023D5F89060C4F8D1
:102FB000003EC02323604FF40413A3633369002B46
:102FC000FCDA01230C203361FFF7D4F83369DB0707
:102FD000FCD41220FFF7CEF83369002BFCDA002670
:102FE0002846A660FFF758FF6B68C4F81068DB68D6
:102FF000C4F81468C4F81C6883BB1D4BA3614FF070
:10300000FF336361A36843F00103A36070BD194BF4
:103010009842C9D1134B4FF08060D3F8D82042F0CA
:103020000072C3F8D820D3F8002142F00072C3F830
:103030000021D3F80021D3F8802042F00072C3F8B9
:103040008020D3F8802022F00072C3F88020D3F8CB
:103050008030FFF70FFF0E214D209EE7064BCDE796
:103060009442002000440258401400400300200213
:10307000003C30C030430020083C30C0F8B5D0F8E8
:103080009040054600214FF000662046FFF730FFD4
:10309000D5F8941000234FF001128F684FF0FF30E5
:1030A000C4F83438C4F81C2804EB431201339F429F
:1030B000C2F80069C2F8006BC2F80809C2F8080B30
:1030C000F2D20B68D5F89020C5F8983063621023CF
:1030D0001361166916F01006FBD11220FFF74AF8AB
:1030E000D4F8003823F4FE63C4F80038A36943F42D
:1030F000402343F01003A3610923C4F81038C4F837
:1031000014380B4BEB604FF0C043C4F8103B094B35
:10311000C4F8003BC4F81069C4F80039D5F89830F9
:1031200003F1100243F48013C5F89820A362F8BDA0
:10313000C047000840800010D0F8902090F88A1016
:10314000D2F8003823F4FE6343EA0113C2F80038D2
:10315000704700002DE9F84300EB8103D0F8905050
:103160000C468046DA680FFA81F94801166806F0C5
:103170000306731E022B05EB41134FF0000194BFB1
:10318000B604384EC3F8101B4FF0010104F11003D0
:1031900098BF06F1805601FA03F3916998BF06F5CE
:1031A000004600293AD0578A04F1580137434901B3
:1031B0006F50D5F81C180B430021C5F81C382B188C
:1031C0000127C3F81019A7405369611E9BB3138AE6
:1031D000928B9B08012A88BF5343D8F898209818EF
:1031E00042EA034301F140022146C8F8980028460C
:1031F00005EB82025360FFF77BFE08EB8900C36892
:103200001B8A43EA845348341E4364012E51D5F887
:103210001C381F43C5F81C78BDE8F88305EB491737
:10322000D7F8001B21F40041C7F8001BD5F81C1883
:1032300021EA0303C0E704F13F030B4A2846214675
:1032400005EB83035A60FFF753FE05EB4910D0F8F6
:10325000003923F40043C0F80039D5F81C3823EABC
:103260000707D7E70080001000040002D0F8942080
:103270001268C0F89820FFF70FBE00005831D0F850
:10328000903049015B5813F4004004D013F4001F40
:103290000CBF0220012070474831D0F8903049011E
:1032A0005B5813F4004004D013F4001F0CBF02203D
:1032B0000120704700EB8101CB68196A0B6813602D
:1032C0004B6853607047000000EB810330B5DD6848
:1032D000AA691368D36019B9402B84BF40231360D7
:1032E0006B8A1468D0F890201C4402EB4110013C1A
:1032F00009B2B4FBF3F46343033323F0030343EA5B
:10330000C44343F0C043C0F8103B2B6803F00303F1
:10331000012B0ED1D2F8083802EB411013F4807F54
:10332000D0F8003B14BF43F0805343F00053C0F883
:10333000003B02EB4112D2F8003B43F00443C2F8D9
:10334000003B30BD2DE9F041D0F8906005460C46B9
:1033500006EB4113D3F8087B3A07C3F8087B08D57E
:10336000D6F814381B0704D500EB8103DB685B68D3
:103370009847FA071FD5D6F81438DB071BD505EB9D
:103380008403D968CCB98B69488A5A68B2FBF0F6D5
:1033900000FB16228AB91868DA6890420DD2121A18
:1033A000C3E90024302383F3118821462846FFF720
:1033B0008BFF84F31188BDE8F081012303FA04F246
:1033C0006B8923EA02036B81CB68002BF3D0214683
:1033D0002846BDE8F041184700EB81034A0170B56B
:1033E000DD68D0F890306C692668E66056BB1A44F8
:1033F0004FF40020C2F810092A6802F00302012AE3
:103400000AB20ED1D3F8080803EB421410F4807FFF
:10341000D4F8000914BF40F0805040F00050C4F8C8
:10342000000903EB4212D2F8000940F00440C2F850
:1034300000090122D3F8340802FA01F10143C3F86C
:10344000341870BD19B9402E84BF40202060206818
:103450001A442E8A8419013CB4FBF6F440EAC440B5
:1034600040F00050C6E700002DE9F843D0F8906026
:1034700005460C464F0106EB4113D3F8088918F0B6
:10348000010FC3F808891CD0D6F81038DB0718D50F
:1034900000EB8103D3F80CC0DCF81430D3F800E063
:1034A000DA68964530D2A2EB0E024FF000091A609E
:1034B000C3F80490302383F31188FFF78DFF89F35D
:1034C000118818F0800F1DD0D6F834380126A64098
:1034D000334217D005EB84030134D5F89050D3F86C
:1034E0000CC0E4B22F44DCF8142005EB0434D2F80D
:1034F00000E05168714514D3D5F8343823EA060644
:10350000C5F83468BDE8F883012303FA01F20389A2
:1035100023EA02030381DCF80830002BD1D098475E
:10352000CFE7AEEB0103BCF81000834228BF03468F
:10353000D7F8180980B2B3EB800FE3D89068A0F1F8
:10354000040959F8048FC4F80080A0EB09089844D6
:10355000B8F1040FF5D818440B4490605360C8E7E5
:103560002DE9F84FD0F8905004466E69AB691E40C3
:1035700016F480586E6103D0BDE8F84FFEF7F8BA34
:10358000002E12DAD5F8003E9B0705D0D5F8003E94
:1035900023F00303C5F8003ED5F80438204623F095
:1035A0000103C5F80438FEF711FB370505D52046A1
:1035B000FFF772FC2046FEF7F7FAB0040CD5D5F8F9
:1035C000083813F0060FEB6823F470530CBF43F474
:1035D000105343F4A053EB6031071BD56368DB68DD
:1035E0001BB9AB6923F00803AB612378052B0CD121
:1035F000D5F8003E9A0705D0D5F8003E23F0030326
:10360000C5F8003E2046FEF7E1FA6368DB680BB1BF
:1036100020469847F30200F1BA80B70226D5D4F8C5
:10362000909000274FF0010A09EB4712D2F8003BB7
:1036300003F44023B3F5802F11D1D2F8003B002BC7
:103640000DDA62890AFA07F322EA0303638104EBC5
:103650008703DB68DB6813B139462046984701379A
:10366000D4F89430FFB29B689F42DDD9F00619D59B
:10367000D4F89000026AC2F30A1702F00F0302F4B2
:10368000F012B2F5802F00F0CA80B2F5402F09D1B8
:1036900004EB8303002200F58050DB681B6A97422D
:1036A00040F0B0803003D5F8185835D5E90303D57C
:1036B00000212046FFF746FEAA0303D5012120463C
:1036C000FFF740FE6B0303D502212046FFF73AFEC9
:1036D0002F0303D503212046FFF734FEE80203D56C
:1036E00004212046FFF72EFEA90203D5052120461E
:1036F000FFF728FE6A0203D506212046FFF722FEC7
:103700002B0203D507212046FFF71CFEEF0103D54E
:1037100008212046FFF716FE700340F1A780E90755
:1037200003D500212046FFF79FFEAA0703D50121FC
:103730002046FFF799FE6B0703D502212046FFF7CD
:1037400093FE2F0703D503212046FFF78DFEEE06DB
:1037500003D504212046FFF787FEA80603D50521DF
:103760002046FFF781FE690603D506212046FFF7B4
:103770007BFE2A0603D507212046FFF775FEEB05E1
:1037800074D520460821BDE8F84FFFF76DBED4F888
:1037900090904FF0000B4FF0010AD4F894305FFA8C
:1037A0008BF79B689F423FF638AF09EB4713D3F87E
:1037B000002902F44022B2F5802F20D1D3F800294D
:1037C000002A1CDAD3F8002942F09042C3F80029FD
:1037D000D3F80029002AFBDB3946D4F89000FFF724
:1037E00087FB22890AFA07F322EA0303238104EB09
:1037F0008703DB689B6813B13946204698470BF175
:10380000010BCAE7910701D1D0F80080072A02F125
:1038100001029CBF03F8018B4FEA18283FE704EB35
:10382000830300F58050DA68D2F818C0DCF808206D
:10383000DCE9001CA1EB0C0C00218F4208D1DB68F5
:103840009B699A683A449A605A683A445A6029E7F0
:1038500011F0030F01D1D0F800808C4501F1010176
:1038600084BF02F8018B4FEA1828E6E7BDE8F88F1D
:1038700008B50348FFF774FEBDE80840FFF744BAF7
:103880009442002008B50348FFF76AFEBDE80840EF
:10389000FFF73ABA30430020D0F8903003EB4111E3
:1038A000D1F8003B43F40013C1F8003B704700001F
:1038B000D0F8903003EB4111D1F8003943F40013F4
:1038C000C1F8003970470000D0F8903003EB411187
:1038D000D1F8003B23F40013C1F8003B704700000F
:1038E000D0F8903003EB4111D1F8003923F40013E4
:1038F000C1F800397047000030B50433039C0172F1
:10390000002104FB0325C160C0E90653049B036347
:10391000059BC0E90000C0E90422C0E90842C0E9F3
:103920000A11436330BD00000022416AC260C0E951
:103930000411C0E90A226FF00101FEF78BBC000000
:10394000D0E90432934201D1C2680AB9181D704708
:1039500000207047036919600021C2680132C2600B
:10396000C269134482699342036124BF436A0361BD
:10397000FEF764BC38B504460D46E3683BB16269A6
:103980000020131D1268A3621344E36207E0237A48
:1039900033B929462046FEF741FC0028EDDA38BD50
:1039A0006FF00100FBE70000C368C269013BC36020
:1039B0004369134482699342436124BF436A43616C
:1039C00000238362036B03B11847704770B530233F
:1039D000044683F31188866A3EB9FFF7CBFF05469C
:1039E00018B186F31188284670BDA36AE26A13F8FD
:1039F000015B9342A36202D32046FFF7D5FF002369
:103A000083F31188EFE700002DE9F84F04460E46D6
:103A1000174698464FF0300989F311880025AA46C9
:103A2000D4F828B0BBF1000F09D141462046FFF77A
:103A3000A1FF20B18BF311882846BDE8F88FD4E9A7
:103A40000A12A7EB050B521A934528BF9346BBF108
:103A5000400F1BD9334601F1400251F8040B91424B
:103A600043F8040BF9D1A36A403640354033A362D2
:103A7000D4E90A239A4202D32046FFF795FF8AF33E
:103A80001188BD42D8D289F31188C9E730465A4619
:103A9000FDF726FBA36A5E445D445B44A362E7E74F
:103AA00010B5029C0433017203FB0421C460C0E919
:103AB00006130023C0E90A33039B0363049BC0E998
:103AC0000000C0E90422C0E90842436310BD0000C1
:103AD000026A6FF00101C260426AC0E9042200225A
:103AE000C0E90A22FEF7B6BBD0E904239A4201D10D
:103AF000C26822B9184650F8043B0B607047002397
:103B00001846FAE7C3680021C2690133C3604369FC
:103B1000134482699342436124BF436A4361FEF7C1
:103B20008DBB000038B504460D46E3683BB1236900
:103B300000201A1DA262E2691344E36207E0237ABF
:103B400033B929462046FEF769FB0028EDDA38BD77
:103B50006FF00100FBE7000003691960C268013AD9
:103B6000C260C269134482699342036124BF436AFD
:103B7000036100238362036B03B1184770470000A1
:103B800070B530230D460446114683F31188866ACA
:103B90002EB9FFF7C7FF10B186F3118870BDA36A75
:103BA0001D70A36AE26A01339342A36204D3E16900
:103BB00020460439FFF7D0FF002080F31188EDE79D
:103BC0002DE9F84F04460D46904699464FF0300ACD
:103BD0008AF311880026B346A76A4FB949462046A2
:103BE000FFF7A0FF20B187F311883046BDE8F88FBA
:103BF000D4E90A073A1AA8EB0607974228BF1746E6
:103C0000402F1BD905F1400355F8042B9D4240F885
:103C1000042BF9D1A36A40364033A362D4E90A23C6
:103C20009A4204D3E16920460439FFF795FF8BF3EC
:103C300011884645D9D28AF31188CDE729463A46FC
:103C4000FDF74EFAA36A3D443E443B44A362E5E7D8
:103C5000D0E904239A4217D1C3689BB1836A8BB120
:103C6000043B9B1A0ED01360C368013BC360C36959
:103C70001A4483699A42026124BF436A03610023A4
:103C800083620123184670470023FBE700F060BA07
:103C9000014B586A704700BF000C0040034B0022E4
:103CA00058631A610222DA60704700BF000C0040BE
:103CB000014B0022DA607047000C0040014B586352
:103CC000704700BF000C0040024B034A1A60034AD1
:103CD0005A607047E443002008440020000002209E
:103CE000074B494210B55C68201A08401968821ACF
:103CF0008A4203D3A24201D85A6010BD0020FCE7DB
:103D0000E443002008B5302383F31188FFF7E8FF70
:103D1000002383F3118808BD04480121044B03608C
:103D20000023C0E901330C3000F016B9EC43002049
:103D3000053D0008CB1D083A23F00703591A521A13
:103D4000012110B4D2080024C0E9004384600C3083
:103D50001C605A605DF8044B00F0FEB82DE9F84F86
:103D6000364ECD1D0F46002818BF0646082A4FEADA
:103D7000D50538BF082206F10C08341D914640468F
:103D800000F006F909F10701C9F1000E2246246886
:103D90006CB9404600F006F93368CBB308224946B7
:103DA000E8009847044698B340E9026730E004EB26
:103DB000010CD4F804A00CEA0E0C0AF10100ACF1DD
:103DC000080304EBC0009842E0D9A0EB0C0CB5EB63
:103DD000EC0F4FEAEC0BD9D89C421CD204F108023C
:103DE000AB45A3EB02024FEAE202626009D9691C0B
:103DF000ED43206803EBC1025D44556043F8310098
:103E000022601C465F60404644F8086B00F0CAF828
:103E10002046BDE8F88FAA45216802D111602346EB
:103E2000EFE7013504EBC50344F8351003F1080151
:103E3000401AC01058601360F1E700BFEC43002047
:103E4000F8B550F8043C044650F8085CA0F10806A8
:103E500007332F1D0C35DB0840F8043C284600F0E2
:103E600097F83B469F421A6801D0B34228D20AB164
:103E7000964225D244F8082C54F8042C1E600132D6
:103E800054F8081C06EBC200814206D1486802447F
:103E900044F8042C0A6844F8082C5868411C03EBC9
:103EA000C1018E4207D154F8042C013202445A60F9
:103EB00054F8082C1A602846BDE8F84000F072B8A3
:103EC0001346CFE7FEE7000070B51B4B0025044604
:103ED00086B058600E4685620163FEF7EDFE04F180
:103EE0001003A560E562C4E904334FF0FF33C4E971
:103EF0000044C4E90635FFF7CBFE2B46024604F129
:103F000034012046C4E9082380230C4A2565FEF7C6
:103F10003BF901230A4AE060009203756846726823
:103F20000192B268CDE90223064BCDE90435FEF7D4
:103F300053F906B070BD00BFA8260020FC4700085A
:103F400001480008C53E0008024AD36A1843D062FF
:103F5000704700BF40240020C0E900008160704726
:103F60008368013B002B10B583600CDA074BDC68DB
:103F70004368A061206063601C6044600520FEF718
:103F80005FF8A06910BD0020FCE700BF40240020BE
:103F900008B5302383F31188FFF7E2FF002383F392
:103FA000118808BD08B5302383F311888368013375
:103FB000002B836007DC036800211A6802605060F0
:103FC0001846FEF773F8002383F3118808BD00003C
:103FD0004B6843608B688360CB68C3600B69436147
:103FE0004B6903628B6943620B6803607047000092
:103FF00008B53C4B40F2FF713B48D3F888200A4398
:10400000C3F88820D3F8882022F4FF6222F0070248
:10401000C3F88820D3F88820D3F8E0200A43C3F8F7
:10402000E020D3F808210A43C3F808212F4AD3F827
:1040300008311146FFF7CCFF00F5806002F11C014A
:10404000FFF7C6FF00F5806002F13801FFF7C0FFFF
:1040500000F5806002F15401FFF7BAFF00F58060BF
:1040600002F17001FFF7B4FF00F5806002F18C01EE
:10407000FFF7AEFF00F5806002F1A801FFF7A8FF8F
:1040800000F5806002F1C401FFF7A2FF00F5806037
:1040900002F1E001FFF79CFF00F5806002F1FC01F6
:1040A000FFF796FF02F58C7100F58060FFF790FF37
:1040B00000F01AF90E4BD3F8902242F00102C3F837
:1040C0009022D3F8942242F00102C3F894220522F0
:1040D000C3F898204FF06052C3F89C20054AC3F8FB
:1040E000A02008BD004402580000025808480008FB
:1040F00000ED00E01F00080308B500F0D3F9FEF75B
:104100001DF8104BD3F8DC2042F04002C3F8DC204D
:10411000D3F8042122F04002C3F80421D3F804317B
:10412000094B1A6842F008021A601A6842F0040249
:104130001A60FEF797FDFEF7FFFCBDE80840FEF7AA
:1041400075BA00BF004402580018024870470000CA
:10415000114BD3F8E82042F00802C3F8E820D3F866
:10416000102142F00802C3F810210C4AD3F8103194
:10417000D36B43F00803D363C722094B9A624FF015
:10418000FF32DA6200229A615A63DA605A600122D1
:104190005A611A60704700BF004402580010005C6A
:1041A000000C0040094A08B51169D3680B40D9B228
:1041B0009B076FEA0101116107D5302383F3118852
:1041C000FDF7D6FF002383F3118808BD000C0040E3
:1041D000064BD3F8DC200243C3F8DC20D3F80421DB
:1041E0001043C3F80401D3F8043170470044025867
:1041F00008B53C4B4FF0FF31D3F8802062F000420D
:10420000C3F88020D3F8802002F00042C3F8802059
:10421000D3F88020D3F88420C3F88410D3F8842006
:104220000022C3F88420D3F88400D86F40F0FF4008
:1042300040F4FF0040F4DF4040F07F00D867D86FC3
:1042400020F0FF4020F4FF0020F4DF4020F07F004A
:10425000D867D86FD3F888006FEA40506FEA5050A3
:10426000C3F88800D3F88800C0F30A00C3F88800B8
:10427000D3F88800D3F89000C3F89010D3F89000DA
:10428000C3F89020D3F89000D3F89400C3F89410AA
:10429000D3F89400C3F89420D3F89400D3F898008E
:1042A000C3F89810D3F89800C3F89820D3F8980072
:1042B000D3F88C00C3F88C10D3F88C00C3F88C2092
:1042C000D3F88C00D3F89C00C3F89C10D3F89C1052
:1042D000C3F89C20D3F89C30FDF72AF9BDE80840CC
:1042E00000F0D4B80044025808B50122534BC3F87B
:1042F0000821534BD3F8F42042F00202C3F8F42013
:10430000D3F81C2142F00202C3F81C210222D3F888
:104310001C314C4BDA605A689104FCD54A4A1A6049
:1043200001229A60494ADA6000221A614FF4404241
:104330009A61444B9A699204FCD51A6842F48072DF
:104340001A603F4B1A6F12F4407F04D04FF4803252
:104350001A6700221A671A6842F001021A60384B85
:104360001A685007FCD500221A611A6912F0380247
:10437000FBD1012119604FF0804159605A67344ADE
:10438000DA62344A1A611A6842F480321A602C4B9D
:104390001A689103FCD51A6842F480521A601A68B0
:1043A0009204FCD52C4A2D499A6200225A63196363
:1043B00001F57C01DA6301F2E71199635A64284A36
:1043C0001A64284ADA621A6842F0A8521A601C4B32
:1043D0001A6802F02852B2F1285FF9D148229A6196
:1043E0004FF48862DA6140221A621F4ADA641F4A77
:1043F0001A651F4A5A651F4A9A6532231E4A13607E
:10440000136803F00F03022BFAD10D4A136943F02E
:1044100003031361136903F03803182BFAD14FF02B
:104420000050FFF7D5FE4FF08040FFF7D1FE4FF070
:104430000040BDE80840FFF7CBBE00BF0080005140
:10444000004402580048025800C000F00200000179
:104450000000FF010088900822204000630209014B
:10446000470E0508DD0BBF012000002000000110F1
:104470000910E000000101100020005208B5FFF70C
:1044800091FEBDE80840FEF73FBC000009217A20FC
:1044900008B5FDF729F907213220BDE80840FDF7EE
:1044A00023B9000008B5FFF7A3FE00F00BF8FDF7F5
:1044B000EDFAFDF7BFF9FFF749FEBDE80840FFF749
:1044C000E5BB0000704700003136366130353038CA
:1044D00061303438343435370000000012100000E9
:1044E000121100001213000053544D333248373F6D
:1044F0003F3F0053544D3332483733782F373278AB
:104500000053544D3332483734332F3735332F3738
:104510003530000001105A000310590001205800E6
:10452000032056001000024008000240000802402C
:1045300000000B002800024008000240040802406E
:1045400006010C004000024008000240080802403A
:1045500010020D0058000240080002400C08024002
:1045600016030E00700002400C00024010080240CA
:1045700000040F00880002400C00024014080240B2
:1045800006051000A00002400C000240180802407E
:1045900010061100B80002400C0002401C08024046
:1045A00016072F00100402400804024020080240B1
:1045B0000008380028040240080402402408024091
:1045C000060939004004024008040240280802405D
:1045D000100A3A0058040240080402402C08024025
:1045E000160B3B00700402400C04024030080240ED
:1045F000000C3C00880402400C04024034080240D5
:10460000060D4400A00402400C0402403808024099
:10461000100E4500B80402400C0402403C08024061
:10462000160F460000000000B11700089D17000893
:10463000D9170008C5170008D1170008BD170008D2
:10464000A917000895170008E517000800000000EA
:104650000100000000000000633000005846000820
:1046600098240020A82600204172647550696C6F60
:10467000740025424F415244252D424C002553459C
:104680005249414C250000000200000000000000DB
:10469000D1190008411A000840004000583F00208E
:1046A000683F00200200000000000000030000003E
:1046B00000000000891A000800000000100000003F
:1046C000783F002000000000010000000000000012
:1046D0009442002001010200C9250008D9240008E5
:1046E000752500085925000843000000F046000821
:1046F00009024300020100C0320904000001020265
:104700000100052400100105240100010424020217
:104710000524060001070582030800FF09040100C3
:10472000020A00000007050102400000070581029F
:1047300040000000120000003C4700081201100178
:10474000020000400912415700020102030100006B
:104750000403090425424F415244250049726F6EFB
:10476000436F72654837003031323334353637386D
:104770003941424344454600000000200000020049
:1047800002000000000000300000040008000000EB
:1047900000000024000008000400000000040000E5
:1047A00000FC000002000000000004300080000057
:1047B00008000000000000380000010001000000B7
:1047C00000000000E51B00089D1E0008491F0008AE
:1047D00040004000CC430020CC43002001000000FA
:1047E000DC430020800000004001000008000000C1
:1047F0000001000000100000080000006D61696EFB
:104800000069646C650000005000802A0000000010
:10481000AAAAAAAA50000024FFFF0000000000007E
:1048200000A00A000000004000000000AAAAAAAAF6
:1048300000000000FFFF000000000000000000007A
:104840001000000000000000AAAAAAAA10000000A0
:10485000FFFF00000000000000000000000040001A
:1048600000000000AAAAAAAA00000000FFFF0000A2
:104870000000000000000000000000000000000038
:10488000AAAAAAAA00000000FFFF00000000000082
:10489000000000000000000000000000AAAAAAAA70
:1048A00000000000FFFF000000000000000000000A
:1048B0000000000000000000AAAAAAAA0000000050
:1048C000FFFF0000000000000000000000000000EA
:1048D00000000000AAAAAAAA00000000FFFF000032
:1048E00000000000000000000000000000000000C8
:1048F000AAAAAAAA00000000FFFF00000000000012
:10490000000000000000000000000000AAAAAAAAFF
:1049100000000000FFFF0000000000000000000099
:104920000000000000000000AAAAAAAA00000000DF
:10493000FFFF000000000000000000000000000079
:10494000DB1B00000000000000001A000000000057
:10495000FF00000000000000E8440008830400009D
:10496000F3440008500400000145000800960000D0
:10497000000008009600000000080000040000008D
:104980005047000800000000000000000000000088
:10499000000000000000000000000000FFFFFFFF1B
:1049A000FFFFFFFFFFFFFFFFFFFFFFFFFFFFFFFF17
:1049B000FFFFFFFFFFFFFFFFFFFFFFFFFFFFFFFF07
:1049C000FFFFFFFFFFFFFFFFFFFFFFFFFFFFFFFFF7
:1049D000FFFFFFFFFFFFFFFFFFFFFFFFFFFFFFFFE7
:020000040801F1
:020000040802F0
:1000000000060030E90D02084D100D0881030208BA
:10001000D50F0D08CD0F0D08D10F0D08EB0D0208FF
:10002000EB0D0208EB0D0208EB0D02084168110808
:10003000EB0D0208EB0D0208EB0D0208EB0D0208B8
:10004000EB0D0208EB0D0208EB0D0208EB0D0208A8
:10005000EB0D0208EB0D0208D1771108FD771108AE
:100060002978110855781108817811083111110883
:100070005911110885111108B1111108DD1111086C
:100080000512110831121108410D1108EB0D02087B
:10009000EB0D0208EB0D0208EB0D0208AD7811081C
:1000A000EB0D0208257A1108EB0D0208397A1108C8
:1000B0003D7A1108517A1108EB0D0208CD1911088B
:1000C000FD191108EB0D0208EB0D0208A123110820
:1000D000EB0D020899791108AD791108C179110861
:1000E00011791108EB0D0208EB0D0208657A110871
:1000F000EB0D0208EB0D0208EB0D02085D12110872
:10010000EB0D020885791108EB0D0208B9231108DF
:10011000D5791108E9791108EB0D0208EB0D0208F9
:1001200089121108B1121108DD1211080913110802
:1001300035131108EB0D0208EB0D0208EB0D020858
:10014000EB0D0208EB0D0208EB0D0208EB0D0208A7
:100150005D13110889131108B5131108EB0D02087E
:10016000EB0D0208EB0D0208EB0D0208EB0D020887
:10017000EB0D02082D741108EB0D0208EB0D0208BF
:10018000EB0D0208EB0D0208FD791108117A110838
:10019000D1231108EB0D0208EB0D0208EB0D02084C
:1001A000EB0D0208EB0D0208EB0D0208EB0D020847
:1001B000EB0D0208EB0D0208EB0D02082D1A1108D9
:1001C0005D1A1108EB0D0208EB0D0208EB0D020899
:1001D000EB0D020819741108EB0D0208EB0D020873
:1001E000EB0D0208EB0D0208EB0D0208EB0D020807
:1001F000EB0D0208EB0D0208EB0D0208EB0D0208F7
:10020000EB0D0208EB0D0208EB0D0208EB0D0208E6
:10021000EB0D0208EB0D0208EB0D0208EB0D0208D6
:10022000EB0D0208EB0D0208EB0D0208EB0D0208C6
:10023000EB0D0208EB0D0208EB0D0208750D11081D
:10024000EB0D0208FD0E1108250F1108510F1108C2
:100250007D0F1108A90F1108D50F11080110110801
:100260002D101108EB0D0208EB0D0208EB0D020832
:10027000EB0D0208EB0D0208EB0D0208EB0D020876
:10028000EB0D0208EB0D0208EB0D0208EB0D020866
:10029000EB0D0208EB0D0208EB0D0208EB0D020856
:1002A000EB0D0208EB0D0208EB0D0208EB0D020846
:1002B000EB0D0208EB0D0208EB0D0208EB0D020836
:1002C000EB0D0208EB0D0208EB0D0208EB0D020826
:1002D000EB0D0208EB0D0208EB0D0208EB0D020816
:1002E000B1E702081518030835A9030899FF0308A8
:1002F000B59D0408794C0608A5500808DD56080885
:10030000FD92080811F80808410109088D04090840
:10031000BD7E09082D850908A1A3090879870A0867
:1003200045040B0801110B08E1010D0861070D08D8
:100330008D220D0869101008E9371008954E100835
:10034000C180100885861008000000000000000031
:10035000000000000000000000000000000000009D
:10036000000000000000000000000000000000008D
:10037000000000000000000000000000000000007D
:10038000EFF30383EFF30982EFF30881DFF814D072
:100390002DE9FE4F68460BF0E7F9BDE8FE4F8D46AC
:1003A00070470000D4310030F1EE101AA0EC200AA2
:1003B00001607047A0EC108A704700BF81F00041D7
:1003C00002E000BF83F0004330B54FEA41044FEA3A
:1003D000430594EA050F08BF90EA020F1FBF54EAD5
:1003E000000C55EA020C7FEA645C7FEA655C00F071
:1003F000E2804FEA5454D4EB5555B8BF6D420CDD42
:100400002C4480EA020281EA030382EA000083EAC4
:10041000010180EA020281EA0303362D88BF30BD64
:1004200011F0004F4FEA01314FF4801C4CEA1131BA
:1004300002D0404261EB410113F0004F4FEA033319
:100440004CEA133302D0524263EB430394EA050FA4
:1004500000F0A780A4F10104D5F1200E0DDB02FA13
:100460000EFC22FA05F2801841F1000103FA0EF2A7
:10047000801843FA05F359410EE0A5F120050EF16D
:10048000200E012A03FA0EFC28BF4CF0020C43FA9E
:1004900005F3C01851EBE37101F0004507D54FF0AB
:1004A000000EDCF1000C7EEB00006EEB0101B1F5FB
:1004B000801F1BD3B1F5001F0CD349085FEA300041
:1004C0004FEA3C0C04F101044FEA445212F5800F4C
:1004D00080F09A80BCF1004F08BF5FEA500C50F1E9
:1004E000000041EB045141EA050130BD5FEA4C0CCC
:1004F000404141EB0101013C28BFB1F5801FE9D229
:1005000091F0000F04BF01460020B1FA81F308BF4B
:100510002033A3F10B03B3F120020CDA0C3208DD17
:1005200002F1140CC2F10C0201FA0CF021FA02F1F2
:100530000CE002F11402D8BFC2F1200C01FA02F162
:1005400020FA0CFCDCBF41EA0C019040E41AA2BF87
:1005500001EB0451294330BD6FEA04041F3C1CDA4F
:100560000C340EDC04F11404C4F1200220FA04F06F
:1005700001FA02F340EA030021FA04F345EA030119
:1005800030BDC4F10C04C4F1200220FA02F001FADB
:1005900004F340EA0300294630BD21FA04F029465D
:1005A00030BD94F0000F83F4801306BF81F48011F6
:1005B0000134013D4EE77FEA645C18BF7FEA655C69
:1005C00029D094EA050F08BF90EA020F05D054EA3B
:1005D000000C04BF1946104630BD91EA030F1EBF40
:1005E0000021002030BD5FEA545C05D14000494144
:1005F00028BF41F0004130BD14F580043CBF01F537
:10060000801130BD01F0004545F0FE4141F470011C
:100610004FF0000030BD7FEA645C1ABF19461046F7
:100620007FEA655C1CBF0B46024650EA013406BFF8
:1006300052EA033591EA030F41F4002130BD00BFB7
:1006400090F0000F04BF0021704730B54FF4806474
:1006500004F132044FF000054FF0000150E700BFF5
:1006600090F0000F04BF0021704730B54FF4806454
:1006700004F1320410F0004548BF40424FF0000141
:100680003EE700BF42004FEAE2014FEA31014FEA84
:1006900002701FBF12F07F4393F07F4F81F06051D3
:1006A000704732F07F4208BF704793F07F4F04BF1E
:1006B00041F40021704730B54FF4607401F00045FB
:1006C00021F000411CE700BF50EA010208BF70475B
:1006D00030B54FF000050AE050EA010208BF70474C
:1006E00030B511F0004502D5404261EB41014FF4B5
:1006F000806404F132045FEA915C3FF4D8AE4FF0BD
:1007000003025FEADC0C18BF03325FEADC0C18BF9F
:10071000033202EBDC02C2F1200300FA03FC20FAF0
:1007200002F001FA03FE40EA0E0021FA02F114443D
:10073000BDE600BF80F0004002E000BF81F0004154
:1007400042001FBF5FEA410392EA030F7FEA226C77
:100750007FEA236C6AD04FEA1262D2EB1363C1BF07
:10076000D218414048404140B8BF5B42192B88BF76
:10077000704710F0004F40F4000020F07F4018BF99
:10078000404211F0004F41F4000121F07F4118BFB9
:10079000494292EA030F3FD0A2F1010241FA03FC61
:1007A00010EB0C00C3F1200301FA03F100F0004349
:1007B00002D5494260EB4000B0F5000F13D3B0F111
:1007C000807F06D340084FEA310102F10102FE2A80
:1007D00051D2B1F1004F40EBC25008BF20F00100F0
:1007E00040EA03007047490040EB0000013A28BF8F
:1007F000B0F5000FEDD2B0FA80FCACF1080CB2EB12
:100800000C0200FA0CF0AABF00EBC250524218438F
:10081000BCBFD0401843704792F0000F81F4000134
:1008200006BF80F400000132013BB5E74FEA410307
:100830007FEA226C18BF7FEA236C21D092EA030F73
:1008400004D092F0000F08BF0846704790EA010FED
:100850001CBF0020704712F07F4F04D1400028BF1A
:1008600040F00040704712F100723CBF00F50000FC
:10087000704700F0004343F0FE4040F40000704732
:100880007FEA226216BF08467FEA236301464202DE
:1008900006BF5FEA412390EA010F40F480007047F1
:1008A0004FF0000304E000BF10F0004348BF404297
:1008B0005FEA000C08BF704743F0964301464FF0D3
:1008C00000001CE050EA010208BF70474FF000032F
:1008D0000AE000BF50EA010208BF704711F0004370
:1008E00002D5404261EB41015FEA010C02BF844640
:1008F0000146002043F0B64308BFA3F18053A3F59F
:100900000003BCFA8CF2083AA3EBC25310DB01FAE5
:1009100002FC634400FA02FCC2F12002BCF1004F69
:1009200020FA02F243EB020008BF20F001007047FA
:1009300002F1200201FA02FCC2F1200250EA4C004E
:1009400021FA02F243EB020008BF20EADC70704794
:100950007BB972B90029BEBF00204FF0004106E00C
:1009600008BF00281CBF6FF000414FF0FF3000F0BF
:1009700039BAADF1080C6DE904CE002909DB002B72
:100980001ADB00F0C7F8DDF804E0DDE9022304B06B
:100990007047404261EB4101002B1BDB00F0BAF8CD
:1009A000DDF804E0DDE9022304B0404261EB4101DF
:1009B000524263EB43037047524263EB430300F040
:1009C000A9F8DDF804E0DDE9022304B0404261EB60
:1009D00041017047524263EB430300F09BF8DDF89E
:1009E00004E0DDE9022304B0524263EB43037047A5
:1009F00053B94AB9002908BF00281CBF4FF0FF3186
:100A00004FF0FF3000F0EEB9ADF1080C6DE904CE07
:100A100000F080F8DDF804E0DDE9022304B070475F
:100A200030B1012390FAA0F0B0FA80F0184470477A
:100A300008460029FBD02123F4E700BF430803F058
:100A40005533C01A830803F0333300F033301844B1
:100A500000EB101000F00F3000EB002000EB004026
:100A6000000E704708B502460B4643EC172BB5EE57
:100A7000C07BF1EE10FA03D4BDE8084000F02AB8BC
:100A8000B1EE477B51EC170B00F024F8404261EBCC
:100A9000410108BD9FED0B6B07EE900A9FED0B5BCC
:100AA000B7EEE77A27EE066BBCEEC66BB8EE464BA8
:100AB000A4EE457BFCEEC77B16EE101A17EE900AEB
:100AC000704700BF000000000000F03D0000000083
:100AD0000000F0419FED0B6B41EC170B9FED0B5BA2
:100AE00027EE066BBCEEC66BB8EE464BA4EE457B1C
:100AF000FCEEC77B16EE101A17EE900A704700BF87
:100B0000AFF30080000000000000F03D0000000096
:100B10000000F0412DE9F047089D04468E46002B69
:100B20004DD18A42944669D9B2FA82F252B101FAA1
:100B300002F3C2F1200120FA01F10CFA02FC41EAB1
:100B4000030E94404FEA1C48210CBEFBF8F61FFA36
:100B50008CF708FB16E341EA034306FB07F19942D1
:100B60000AD91CEB030306F1FF3080F01F81994284
:100B700040F21C81023E63445B1AA4B2B3FBF8F05E
:100B800008FB103344EA034400FB07F7A7420AD9E5
:100B90001CEB040400F1FF3380F00A81A74240F20D
:100BA00007816444023840EA0640E41B00261DB178
:100BB000D4400023C5E900433146BDE8F0878B42AD
:100BC00009D9002D00F0EF800026C5E9000130466C
:100BD0003146BDE8F087B3FA83F6002E4AD18B4246
:100BE00002D3824200F2F980841A61EB03030120F0
:100BF0009E46002DE0D0C5E9004EDDE702B9FFDEDC
:100C0000B2FA82F2002A40F09280A1EB0C014FEA86
:100C10001C471FFA8CFE0126200CB1FBF7F307FBE3
:100C2000131140EA01410EFB03F0884208D91CEB86
:100C3000010103F1FF3802D2884200F2CB80434623
:100C4000091AA4B2B1FBF7F007FB101144EA014402
:100C50000EFB00FEA64508D91CEB040400F1FF3191
:100C600002D2A64500F2BB800846A4EB0E0440EA7F
:100C700003409CE7C6F12007B34022FA07FC4CEA88
:100C8000030C20FA07F401FA06F31C43F9404FEA7B
:100C90001C4900FA06F3B1FBF9F8200C1FFA8CFE90
:100CA00009FB181140EA014108FB0EF0884202FAE4
:100CB00006F20BD91CEB010108F1FF3A80F08880A5
:100CC000884240F28580A8F102086144091AA4B262
:100CD000B1FBF9F009FB101144EA014100FB0EFEE3
:100CE0008E4508D91CEB010100F1FF346CD28E4512
:100CF0006AD90238614440EA0840A0FB0294A1EBA3
:100D00000E01A142C846A64656D353D05DB1B3EBFF
:100D1000080261EB0E0101FA07F722FA06F3F1402F
:100D20001F43C5E9007100263146BDE8F087C2F1D6
:100D30002003D8400CFA02FC21FA03F3914001434E
:100D40004FEA1C471FFA8CFEB3FBF7F007FB103687
:100D50000B0C43EA064300FB0EF69E4204FA02F433
:100D600008D91CEB030300F1FF382FD29E422DD986
:100D7000023863449B1B89B2B3FBF7F607FB1633BB
:100D800041EA034106FB0EF38B4208D91CEB01013B
:100D900006F1FF3816D28B4214D9023E6144C91ABB
:100DA00046EA004638E72E46284605E70646E3E6CB
:100DB0001846F8E64B45A9D2B9EB020864EB0C0ED5
:100DC0000138A3E74646EAE7204694E74046D1E7E4
:100DD000D0467BE7023B614432E7304609E7644492
:100DE000023842E7704700BF02E000F000F8FEE77B
:100DF00072B6374880F30888364880F30988364849
:100E00003649086040F20000CCF200004EF6347122
:100E1000CEF200010860BFF34F8FBFF36F8F40F237
:100E20000000C0F2F0004EF68851CEF200010860DA
:100E3000BFF34F8FBFF36F8F4FF00000E1EE100A4A
:100E40004EF63C71CEF200010860062080F3148853
:100E5000BFF36F8FF5F056FDF4F086FB4FF0553081
:100E60001F491B4A91423CBF41F8040BFAE71D4958
:100E7000184A91423CBF41F8040BFAE71A491B4A51
:100E80001B4B9A423EBF51F8040B42F8040BF8E7A3
:100E900000201849184A91423CBF41F8040BFAE778
:100EA000F5F06EFDF4F0E4FB144C154DAC4203DAA2
:100EB00054F8041B8847F9E70DF06AFC114C124DF9
:100EC000AC4203DA54F8041B8847F9E7F5F056BD45
:100ED00000060030002200300000020808ED00E0AB
:100EE0000000003000060030404A140800220030A4
:100EF000D42F0030D82F0030000B0230E00202085F
:100F00004803020848030208480302082DE9F04F8D
:100F10002DED108AC1F80CD0D0F80CD0BDEC108AA1
:100F2000BDE8F08F002383F311882846A0470020F6
:100F3000F4F08AF8FEE7F3F0F3FE00DFFEE70000CE
:100F400038B510EE104AC4F30A53B3F57D7FB7EEFF
:100F5000C07A1ED227EE077BB3F5667F6FD327EEEC
:100F6000071B634B93ED142B93ED125B93ED0E3B3C
:100F7000A7EE025B93ED0C0B93ED104BA7EE030B6A
:100F800027EE017BA1EE040BA5EE070BB7EEC00B1D
:100F900038BD40F22E42934254D8554991ED086B2A
:100FA00027EE066BFDEEC66B91ED0A5B16EE903AEE
:100FB00003F500031B1613F0020F06EE903A01F141
:100FC000700208BF0A46D807B8EEE66BA6EE457B6E
:100FD00027EE076B1AD503F0030301EBC30393ED70
:100FE000002B92ED1A4B92ED185B92ED163BA6EE9C
:100FF000045B27EE027B27EE064B26EE046BA4EE85
:10100000037BA5EE067BB7EEC70B38BD92ED142B24
:1010100092ED127B92ED0E3B92ED0C0B92ED104B8C
:1010200026EE065BA6EE027BA6EE030B26EE056B14
:10103000A5EE040BA7EE060BB7EEC00B38BDB7EE5E
:10104000000A38BDB3F5FF6F3DD22A4BC4F383626B
:1010500003EB820153F822200D69C4F31603C4F395
:10106000C25043F400038340086A03FB02F2A3FB6F
:101070000010E3FB050202F100518D0F01F0404129
:10108000511AFFF729FB1C4B9FED177B05EBD4741E
:1010900041EC160B14F0020FA3F1700208BF1346C7
:1010A000E90726EE077B27EE076B10D504F0030453
:1010B00002EBC40494ED002B93ED1A4B93ED185BF7
:1010C00093ED163B93E7BDE8384000F053B893ED3D
:1010D000142B93ED127B93ED0E3B93ED0C0B93EDE4
:1010E000104B9DE7AFF30080182D4454FB21193CB1
:1010F000C88B1108688B1108388C110810B582B0A4
:101100008DED010A044603F035FE9DED010A0460F1
:1011100002B010BD28B1F1EE407A27EE800A2220FD
:10112000ECE7F0EE407A27EE800A2220E6E700BFE7
:101130009FED010AEEE700BF000000109FED010ADD
:10114000E8E700BF0000201A9FED010AE2E700BFB8
:10115000000000709FED060AFFEE007AB7EE007AFD
:1011600000284FF0220047FE277A87EE800AC5E765
:101170000000000070EE407AB4EE400A87EEA77AD5
:10118000F1EE10FAB0EE470A01D62120B6E770471B
:10119000B0EE407B17EE903A1B4A23F00043934297
:1011A0001BDD1A4A934202DD30EE400B704700B55A
:1011B00085B0684601F0A2FA00F0030001289DED19
:1011C000021B9DED000B0CD0022812D070B1012043
:1011D00002F0C6FC05B05DF804FB9FED091B02F0B0
:1011E000CFB802F0BDFCB1EE400BF3E702F0C8F857
:1011F000F0E702F0C5F8B1EE400BEBE7AFF300808B
:101200000000000000000000FB21E93FFFFFEF7F2E
:10121000B0EE407B17EE903A1B4A23F00043934216
:101220001CDD1A4A934202DD30EE400B704700B5D8
:1012300085B0684601F062FA00F0030001289DEDD8
:10124000021B9DED000B0ED0022813D070B102F0EE
:1012500097F8B1EE400B05B05DF804FB9FED081B5D
:10126000002002F07DBC02F08BF8F4E7012002F0D0
:1012700077FCF0E7012002F073FCB1EE400BEAE7E7
:101280000000000000000000FB21E93FFFFFEF7FAE
:1012900038B510EE105A25F00044B4F1A14FF0EE2D
:1012A000407A0ADBB4F1FF4F57DCDFED517A9FED56
:1012B000510A002D37FE800A38BD4F4B9C425BDC43
:1012C000B4F1445F4CDB4FF0FF3267EEA76ADFED0D
:1012D0004B4ADFED4B5A9FED4B5A9FED4B4A26EEA2
:1012E000A67AB0EE666AE7EE245A531CDFED474A51
:1012F000DFED476AA5EE875AE7EE246ADFED455A2F
:10130000DFED454AE6EE875AA5EE074A9FED435AC0
:10131000DFED436AA5EE875AE4EE074ADFED415A56
:10132000E4EE876AE5EE075A66EE866A25EE877A6E
:1013300037D03D4B03EB820376EE876A93ED000ACC
:1013400093ED047A96EEA70A002D70EE677A37EED9
:10135000670AB1DAB1EE400A38BD30EE000A38BD96
:101360009FED327A30EE077AF7EE006AB4EEE67A55
:10137000F1EE10FAA7DD38BD00F036F92C4B9C4297
:1013800016DCA3F5D0039C4227DCF0EE007ABFEE1A
:10139000007AA0EE277A002230EE270AC7EE007A04
:1013A00093E776EE876AE6EEE77AB0EE670A38BD35
:1013B000204B9C420BDCF7EE087AB7EE007AA0EEE9
:1013C000277A022230EE670AC0EE077A7DE7BFEE89
:1013D000007AC7EE007A032277E7F7EE007A30EE64
:1013E000677A30EE270A0122C7EE007A6DE700BF68
:1013F000DB0FC93FDB0FC9BFFFFFDF3ED769853C6D
:1014000059DA4B3D356B883D6E2EBA3D21A215BD94
:101410006BF16EBD95879DBD2549123E388EE3BDAB
:10142000ABAAAA3ECDCC4CBE90861108CAF2497137
:10143000FFFF973FFFFF1B4082B08DED010A019A2D
:1014400022F00043B3F1FF4F3CD2BBB3B3F5000F22
:1014500006EE903A3ADADFED227A2249224B66EE26
:10146000A77A17EE900AA1FB000103EB510307EEE8
:10147000103A27EE076ADFED1D7ADFED1D4A9FED7A
:101480001D5AC6EE265A02F000429FED1B6ADFEDA0
:101490001B6AE7EE257AC4EEA75A77EE857A77EED7
:1014A000A57A86EE270A30EE260A20EE070A10EE0D
:1014B000103A134300EE103A02B070479DED010A56
:1014C00002B0704730EE000A02B0704705480C4980
:1014D000A0FB030301EB530307EE103AC9E700BF7B
:1014E0000000804BABAAAAAAF2195126B0F80A3F15
:1014F000F18E34BF5007B53FDBB6CD3F6EDBB63E55
:10150000F219512A10EE103A40F22A41C3F30A525E
:101510008A42B7EEC03A32D8B7EE000B2D4B93EDAE
:101520004A2B93ED481BB0EE417BA2EE037B17EEF6
:10153000100A37EE417B00F01F0203EBC20130B40A
:1015400092EE037B93ED4C4B53F832404D6893ED94
:101550004E6B93ED505BA4EE076B27EE074B00211B
:101560000A1905EBC033A5EE070B43EC172BA6EECB
:10157000040B30BC20EE070BB7EEC00B704713F521
:10158000000F20D0B2F5FF6F1AD2DFED137AB4EE60
:10159000E70AF1EE10FA10DCDFED107AB4EEE70A9C
:1015A000F1EE10FA12D4DFED0E7AB4EEE70AF1EEA6
:1015B00010FAB1D50020FFF7C1BD0020FFF7C4BD70
:1015C00030EE000A70479FED070A70470020FFF7D2
:1015D000AFBD00BFB08611081772B142B4F1CFC2DF
:1015E000CF8ECEC20000000010EE103A23F0004370
:1015F00000EE103A704700BF10EE102A22F00043B0
:1016000010B4B3F1FF4F4FF00004046017DAB3B128
:1016100012F0FF4F10EE101A09D1DFED0B7A60EED9
:10162000277A6FF0180417EE901A21F00043DB15AB
:101630007E3B234421F0FF42036042F07C5200EEE7
:10164000102A5DF8044B70470000004C10EE103A71
:10165000B3F17E5F10EE101A38D0A3F50002B2F19C
:10166000FE4F36D2BFEE000B01F14042264B02F591
:101670004D02C2F3C34003EB001093ED404B93EDDA
:10168000445B93ED467B93ED426BD30DDB0590ED10
:10169000002BCB1A03EE903A90ED021BD215B7EE59
:1016A000E33AA2EE030B03EE902A20EE002BA5EE08
:1016B000007BB8EEE33BA6EE027BA3EE041B30EE0C
:1016C000010BA2EE070BB7EEC00B70479FED0F0AA0
:1016D00070475A0014D0B3F1FF4F14D0002B0BDB2E
:1016E000B2F17F4F08D2DFED0A7A60EE277A17EE6B
:1016F000903AA3F13861B5E700EE103AFFF73ABD32
:101700000120FFF727BD704718891108000000006D
:101710000000004B10EE103AB3F17E5F3ED0A3F50F
:101720000001B1F1FE4F10EE102A3AD2BFEE002BAD
:1017300002F14043284903F54D03C3F3C34001EBD5
:10174000001091ED424B91ED447B91ED406B91ED9A
:10175000465BD90DC9052DED028B90ED021B90ED76
:10176000008B521ADB1500EE103A03EE902AB8EE09
:10177000C00BB7EEE33A30EE010BA8EE032BBDEC45
:10178000028B22EE023BA4EE027BA5EE020BA6EE3C
:10179000037BA3EE070BB7EEC00B70479FED0F0A5C
:1017A0007047590014D0B3F1FF4F14D0002B0BDB5E
:1017B000B1F17F4F08D2DFED0A7A60EE277A17EE9B
:1017C000903AA3F13862B1E700EE103AFFF7D2BCCD
:1017D0000120FFF7BFBC7047F88711080000000028
:1017E0000000004B10B485B08DED010A019BC3F3DE
:1017F000C751A1F17F021E2A2ADC501C23DB162AC6
:101800004FEAD3740BDDC3F3160040F400009639A1
:10181000884004B1404205B05DF8044B7047164B58
:10182000DDED017A03EB840393ED007A77EE277AFE
:10183000CDED037ADDED037A77EEC77A17EE903AB5
:1018400033F000420ED1002005B05DF8044B704724
:10185000DDED017AFDEEE77A17EE900A05B05DF84E
:10186000044B7047C3F31600C3F3C75340F40000A2
:10187000C3F19603D840CCE7388A11089FED010ADE
:10188000704700BF0000C07F30B410EE103A2DED5D
:10189000028BA3F5000110EE902AB1F1FE4F10EE7D
:1018A000104A82B04FEA42017ED201F1FF3C6FF054
:1018B0008070844580F0F980002004F1404303F5F6
:1018C0004D03C3F3C341DB0DDB05E21ADB1507EE65
:1018D000903ABFEE001BB24B03EB011191ED004BB0
:1018E00005EE102AB7EEC55AA4EE051B93ED444B46
:1018F00021EE012B93ED465B93ED403BA1EE045BA3
:1019000093ED426B93ED484BA1EE036B22EE023B4D
:10191000B8EEE78BB7EEE07A91ED020B38EE000BF4
:10192000A1EE040BA2EE050BA6EE030B27EE000BB7
:1019300010EE903A48F2BF02C3F3CF33934252D233
:10194000B7EE007B974B93ED402B30EE023B13EE4E
:10195000102A33EE423B02F01F01821803EBC10054
:1019600053F83140456830EE433B93ED465B93EDD1
:10197000424BA3EE057BB0EE470B93ED446B002387
:10198000181905EBC23141EC170BA3EE046B23EEE3
:10199000034BA6EE040B20EE070BB7EEC00B02B014
:1019A000BDEC028B30BC70474D1E6FF080708542DD
:1019B00080F0CE8059004D1E854280F09280002B31
:1019C00055DB0020B4F5000FBFF477AFDFED767A7A
:1019D00007EE103A67EE277A17EE904A24F000449B
:1019E000A4F1386469E79FED667BB4EEC70BF1EEB6
:1019F00010FA15DC9FED647BB4EEC70BF1EE10FA24
:101A000020DD4FF04C5388B10193DDED017ABFEE3C
:101A1000007A77EE677AF4EE477AF1EE10FA11D099
:101A200002B0BDEC028B30BCFFF78EBB0093DDED46
:101A3000007AB7EE007A77EE877AF4EE477AF1EE25
:101A400010FAEDD19FED527BB4EEC70BF1EE10FA18
:101A500057D99FED517BB4EEC70BF1EE10FA7FF52D
:101A60006FAF02B0BDEC028B30BCFFF767BBC2F3B7
:101A7000C7517E2911DD962954DC0120C1F1960160
:101A800000FA01F1481E104207D111EA020018BF06
:101A90004FF4803024F0004494E700EE103A02B096
:101AA000BDEC028B30BCFFF765BB002952D0B3F10F
:101AB0007E5F2CD06400B4F17F4F2ED8B1F17F4F00
:101AC0002BD1B4F1FE4F4BD0B4F1FE4F6FEA0202BE
:101AD00034BF00240124D20F94424CD09FED330A2E
:101AE0005DE7002B20EE000A1EDB002000293AD122
:101AF000002ABFF654AF02B0BDEC028B30BCFFF73A
:101B000029BB02B0BDEC028B30BCFFF711BB82F4E5
:101B10008002520012F5000F22D907EE903A37EEFC
:101B2000A00A3CE70020B5E7C2F3C753A3F17F004A
:101B30001728DAD8C3F19600012303FA00F0441EF7
:101B40001442D2D11040D1D0B1EE400A1846CDE7B0
:101B50000029AFD184F48002520012F5000FDCD8C6
:101B6000B7EE000A1BE7002ABFF619AFF7EE007ABE
:101B700087EE800A13E720EEA00A10E7AFF300809B
:101B800071D5D1FFFFFF5F40E2AAA3FFFFFF5F40D7
:101B90000000000000C062C00000000000A062C0A1
:101BA000408A1108B08611080000004B00000000B8
:101BB00010EE103A114A23F00043934218DDB3F1BE
:101BC000FF4F02DB30EE400A704700B583B0684635
:101BD00001F0A0FA400000F00200DDED010A9DEDE9
:101BE000000AC0F1010002F04DFB03B05DF804FBF8
:101BF000DFED030A012002F045BB00BFDA0F493FC9
:101C00000000000030B510EE104AC4F30A53B3F5DB
:101C10007D7FB7EEC06A83B01BD226EE065BB3F5BC
:101C2000667F70D326EE052B25EE021B754B93EDD8
:101C30001A3B93ED187B93ED164BA5EE037BA2EEBA
:101C4000046BB0EE460BA7EE010BB7EEC00B03B072
:101C500030BD40F22E42934260D86A4991ED087B34
:101C600026EE077BFDEEC77B91ED0A5B17EE903AFF
:101C700003F500031B1613F0020F07EE903A01F173
:101C8000700208BF0A46D807B8EEE77BA7EE456B9F
:101C9000B0EE460B26EE067B1BD403F0030301EBEC
:101CA000C30392ED1A5B93ED003B92ED186B20EEAF
:101CB000030B92ED164BA7EE056B20EE075B27EEAC
:101CC000057BA5EE040BA6EE070BB7EEC00B03B029
:101CD00030BD92ED142B27EE075B92ED126B92ED67
:101CE0000E3BA7EE026B92ED0C0B92ED104BA7EEA4
:101CF000030B27EE057BA5EE040BA6EE070BB7EE54
:101D0000C00B03B030BD220D12F4FF6FDFD1B7EE70
:101D1000C55B00EE104A8DED015AD8E7B3F5FF6FB1
:101D20004BD2394BC4F3836203EB820153F8222078
:101D30000D69C4F31603C4F3C25043F40003834097
:101D4000086A03FB02F2A3FB0010E3FB050202F1A9
:101D500000518D0F01F04041511AFEF7BDFC2B4B95
:101D60009FED267B05EBD47441EC160B14F0020FAB
:101D7000A3F1700208BF1346E90726EE077B27EEA2
:101D8000076B1FD404F0030402EBC40493ED1A4B59
:101D900094ED002B93ED185B27EE027B93ED163B41
:101DA000A6EE045B27EE064B26EE046BA4EE037B47
:101DB000A5EE067BB7EEC70B89E703B0BDE8304060
:101DC000FFF7D8B993ED142B26EE065B93ED127B4B
:101DD00093ED0E3BA6EE027B93ED0C0B93ED104BB7
:101DE000A6EE030B26EE056BA5EE040BA7EE060B85
:101DF000B7EEC00B6BE700BFAFF30080182D445463
:101E0000FB21193CC88B1108688B1108388C11080C
:101E100008B52DED048BB0EE408B00F027F9144B84
:101E2000B0EE409B93F9003001330FD0B4EE488BF5
:101E3000F1EE10FA0AD6B0EE480B02F007FCB7EE4E
:101E4000007BB4EEC70BF1EE10FA04DCB0EE490BE8
:101E5000BDEC048B08BD02F08DFFBDEC048B034686
:101E600021221A600348BDE8084002F07DBC00BF93
:101E7000002200301849140800F026BA08B52DEDEC
:101E8000048BB0EE409BB0EE418B00F0E9FA114BB1
:101E900093F9003001330BD0B4EE489BF1EE10FA09
:101EA00006D69FED0A9BB4EE498BF1EE10FA02D0F4
:101EB000BDEC048B08BD02F05DFF89EE090BBDECA3
:101EC000048B2123036008BDAFF3008000000000F5
:101ED000000000000022003008B52DED028BB0EEAE
:101EE000408A00F059FD144B93F900300133F0EEB5
:101EF000408A0FD0B4EE488AF1EE10FA0AD6B0EE5E
:101F0000480AFFF771FBF7EE007AB4EEE70AF1EE4C
:101F100010FA04DCB0EE680ABDEC028B08BD02F0DA
:101F200029FFBDEC028B034621221A600348BDE85D
:101F30000840FFF7A3BC00BF002200301849140876
:101F400008B52DED028BB0EE408A00F049FE144B2F
:101F500093F900300133F0EE408A0FD0B4EE488A96
:101F6000F1EE10FA0AD6B0EE480AFFF73DFBF7EEA5
:101F7000007AB4EEE70AF1EE10FA04DCB0EE680A7B
:101F8000BDEC028B08BD02F0F5FEBDEC028B0346F2
:101F900021221A600348BDE80840FFF76FBC00BF6C
:101FA000002200301849140800F020BF08B52DEDBC
:101FB000028BF0EE408AB0EE608A00F0BBFF0E4B61
:101FC00093F9003001330BD0F4EE488AF1EE10FAA9
:101FD00006D6DFED0A8AB4EE688AF1EE10FA02D076
:101FE000BDEC028B08BD02F0C5FE88EEA80ABDEC70
:101FF000028B2123036008BD002200300000000096
:1020000008B52DED028BB0EE408A01F023F8144B99
:1020100093F90030013314D0B4EE488AF1EE10FA8F
:102020000FD6B5EEC08AF1EE10FA0AD8B5EE408AA6
:10203000F1EE10FA08D102F09DFE22239FED090A6D
:102040000360BDEC028B08BD02F094FEBDEC028B78
:10205000034621221A600448BDE80840FFF70EBC81
:1020600000220030000080FF1849140838B510EE37
:10207000905A924B25F000449C422DED0A8B1DDDB9
:1020800010EE103A04F1404404F58014234308D0C4
:1020900030EE400B80EE007BBDEC0A8BB0EE470BC0
:1020A00038BDBDEC0A8B9FED677B9FED686B20EE22
:1020B000077BA0EE067BB0EE470B38BD804B9C4201
:1020C0000EDCB4F1795F80F28380B7EE006B9FED98
:1020D000617B30EE077BB4EEC67BF1EE10FA74DC68
:1020E000B6EE008B02F0B2FAB7EE007B9FED5B9B81
:1020F00037EE400B20EE088B9FED5AABB0EE480B4D
:102100009FED5A1B9FED5B3BA8EE0A1B9FED5B4BBF
:10211000A1EE083B9FED5B6BA3EE084B9FED5BCB05
:10212000A4EE086B9FED5B2BA6EE08CB2CEE08CB44
:102130009FED5A5BA8EE092B9FED5ABBA2EE085B00
:10214000A5EE08BBABEE087BB0EE479B00F020FC91
:102150005C4B9C422ADCB0EE004B8CEE093B53EC0E
:10216000102B9FED526B9FED377B002243EC122B1F
:1021700030EE025BA2EE428B30EE000B88EE051BC8
:10218000B0EE465BA1EE447BA2EE445B90EE037B97
:1021900037EE457B36EE477B002D3FF77DAFB1EE46
:1021A000477BB0EE470BBDEC0A8B38BD9FED417B02
:1021B0008CEE094BB0EE005B9FED246BA0EE040BA0
:1021C000A0EE057B36EE477BE6E7B0EE407B63E7AB
:1021D0009FED248B20EE006B9FED245B9FED253B54
:1021E000A6EE085B9FED254BA5EE063B9FED252B4C
:1021F000A3EE064BBDEC0A8BA4EE062B9FED237BD2
:102200009FED161BA2EE067B27EE067B9FED215B62
:102210009FED223BA6EE015B9FED224BA5EE063B18
:10222000B7EE005BA3EE064BA4EE065B87EE056BF4
:10223000B0EE407BA0EE067BB0EE470B38BD00BF92
:10224000AFF30080075C143326A6913C182D44544C
:10225000FB21F93F9C7500883CE4377E82922EB1C9
:10226000C5B8B33F09F7FD0DE13D023F88B20175E6
:10227000E0EF493F3B8F68B52882A4BF5544880EE4
:1022800055C1C93F7D6FEB0312D6D4BF5555555587
:102290005555C53F59018D1B6C06E6BFC88A599C30
:1022A000E52A00404B2D8A1C273A03C0182D4454C0
:1022B000FB21E93F075C143326A691BCFFFFEF3FEB
:1022C000FFFFDF3F3233EF3F2DE9F04151EC110BBF
:1022D0004342614C21F0004E03434EEAD37382B077
:1022E000A3428DED000B39D8DDE90067734233431B
:1022F00027F0004848EAD373A3422FD801F14043A6
:1023000003F5801303433ED08D1705F0020558EA0C
:10231000060345EAD7752AD05EEA000338D0A64501
:1023200044D0A04534D0A8EB0E0EBEF1747F4FEA26
:102330002E5338DA002945DA3C3343DA9FED380B67
:10234000012D53D0022D48D075B19FED376B9FED15
:10235000387B30EE460B30EE470B05E09DED006B11
:1023600041EC170B37EE060B02B0BDE8F081022DF1
:1023700016D09DED007B9FED300B032D00FE070B6B
:1023800002B0BDE8F08102B0BDE8F04102F05AB8F9
:102390009FED2B0B9FED2C7B002F20FE070BE3E71F
:1023A0009FED230BE0E79FED260BC9E7F04505F114
:1023B000FF3524D0022D2AD8284B03EBC50595ED17
:1023C000060BD1E79DED007B41EC160B87EE060B6B
:1023D00002F03CF902F036F8B2E79FED136B9FED87
:1023E000147B30EE460B37EE400BBDE710EE901A33
:1023F00053EC102B01F1004343EC102BB4E7022DFA
:1024000008D8164B03EBC50595ED000BACE79FED27
:10241000040BA9E79FED0E0BA6E700BFAFF300800A
:102420000000000000000000075C143326A6A13C59
:10243000182D4454FB210940182D4454FB2109C098
:10244000182D4454FB21F93F182D4454FB21F9BFAA
:10245000182D4454FB21E93F0000F07FA88C11089F
:102460002DE9F04385B08DED001BDDE9007C2CF0FB
:10247000004050EA07038DED020B2FD0039B994AD1
:1024800023F0004E964529DC7A4297493A4340EAC8
:10249000D2728A4222D8DDF8089086453C464A46E8
:1024A00003F0004606DCC0F2C880B945C0F0C58024
:1024B00000F0FE808C491940D9B9BEF1000F40F000
:1024C000E080B9F1000F4D4640F30981A1F21341BC
:1024D0006D00002D01F1FF31FADC0EE09DED027B75
:1024E0009DED006B27EE067B87EE070B05B0BDE880
:1024F000F0834FEA2E51A1F2FF317B4D0CEA050526
:1025000085B9002840F0AE80002FB84640F3E58042
:10251000A5F213454FEA4808B8F1000F05F1FF3561
:10252000F8DC02E00515A5F2FF35DFF8C081414572
:1025300073DBC3F3130343F48013DFF8B0E1754595
:1025400059DBCCF3130C4CF4801CD01B491B0BD172
:102550001DE050EA0E0345D04FEADE73013903EB6C
:1025600040034FEA4E0211D0A3EB0C00944288BF07
:1025700000F1FF300028A2EB040E4FEAD277E8DA30
:10258000013907EB43034FEA4202EDD1101BA3EBE5
:102590000C0C944288BF0CF1FF3CBCF1000FA4BFAF
:1025A0000246634653EA020105D11BE0D10F01EB5D
:1025B00043035200013DB3F5801FF7DB4B498D42C9
:1025C0006BDA491B142979DC05F21E40CA4003FA74
:1025D00000F043FA01F110430E433346024643EC48
:1025E000102B83E7424BF60F03EBC60696ED000B6C
:1025F00005B0BDE8F083AEEB050EBEF11F0F25DD83
:102600003C48491BA0EB050C07FA0CFC18BF002442
:10261000AAD1A3EB0C0C1046BFE7A8EB0108B8F158
:102620001F0F0DDC01F21E430EFA08FE29FA03F318
:1026300009FA08F243EA0E037FE79DED020B55E726
:102640002C4B5B1A09FA03F3002276E700FA0EFC22
:1026500005F21E4027FA00F007FA0EF440EA0C0CCF
:10266000101B73E74FEAC028B8F1000F1F4D7FF72A
:102670005CAF4FEA4808B8F1000F05F1FF35F8DC10
:1026800053E74FEACE25002D18497FF736AF6D008E
:10269000002D01F1FF31FADC2FE7A3F580131E4373
:1026A00005F2FF3546EA0551104641EC100B1DE7D7
:1026B0000F4B03EB167696ED000B17E71F2907DC8F
:1026C00005F21E4022FA01F1834043EA010084E74B
:1026D0000849491B43FA01F07FE7074D25E7064902
:1026E0000BE700BFFFFFEF7F0000F07F02FCFFFF62
:1026F000D88C1108E2FBFFFFEDFBFFFF70B553EC38
:10270000102B9C4923F000458D4288B004466ADDB9
:1027100099498D421E461BDC002B9FED867B40F3C2
:10272000EC8030EE477BA1F51B21A1F5F0618D42D5
:102730006AD09FED826B012037EE465B37EE457B1A
:1027400084ED005B37EE467B84ED027B08B070BD04
:102750008A498D4260DD8A498D424DDC2A1510EE92
:10276000100AA2F21642A5EB025141EC170B9FEDA5
:10277000755BBDEEC76BB8EEC66B37EE467B27EEDA
:10278000057BFDEEC74B8DED026BB8EEE46B37EECB
:10279000467B27EE057BB5EE407BF1EE10FA8DED22
:1027A000046B8DED067B40F0978014EE903A002B81
:1027B0000CBF01230223734901910221009102A859
:1027C000214600F075FE002EC0DA94ED006B94ED0A
:1027D000027BB1EE466BB1EE477B84ED006B84ED7E
:1027E000027B4042B2E700200021C4E90201002040
:1027F00084ED000B08B070BD30EE407B002084ED0E
:10280000027B84ED007BA1E79FED505B9FED516B58
:1028100037EE457B01208FE701F018FFB6EE007B15
:102820009FED4E5BA0EE057BFDEEC77B9FED413B30
:1028300017EE900A9FED416B1F28B8EEE75BB1EEF3
:10284000454BA5EE430B25EE067B1CDC4E4B421E92
:1028500053F82230AB4216D030EE476B84ED006B5C
:1028600030EE460B30EE470B002E84ED020BBFF628
:102870006DAFB1EE466BB1EE400B84ED006B84EDB5
:10288000020B404262E730EE476B16EE903AC3F31C
:102890000A532A15C3EB1555102DDFDDB0EE403B72
:1028A0009FED2A7B9FED2B6BA4EE073B30EE430B95
:1028B000A4EE070BB0EE407B95EE067B33EE476B44
:1028C00016EE903AC3F30A53D21A312A06DCB0EE60
:1028D000430B84ED006BC3E703236CE79FED216B93
:1028E000B0EE430B9FED212BA4EE060B33EE407BA5
:1028F000A4EE067B95EE027BAEE7244930EE077B23
:102900008D420ED09FED0D6B4FF0FF3037EE065B22
:1029100037EE457B84ED005B37EE067B84ED027B72
:1029200014E79FED0A5B9FED0B6B37EE057B4FF0D5
:10293000FF30EBE700004054FB21F93F3163621A9E
:1029400061B4D03D00000000000070410000601A3A
:1029500061B4D03D7370032E8A19A33B83C8C96D3F
:10296000305FE43F0000002E8A19A33BC1492025B7
:102970009A837B39FB21E93F7BD90240FB21394116
:10298000FFFFEF7F688D1108E88C1108FB21F93FEC
:10299000B1EEC00B704700BF08B510EE102A22F050
:1029A0000043B3F17E5F2DED028B12D00ADCB3F150
:1029B0007C5F18DAB3F10C5F6BDCBDEC028B9FED32
:1029C000770A08BD70EE407A87EEA70ABDEC028B4D
:1029D00008BDBDEC028B9FED720ADFED727A002A12
:1029E00030FE270A08BD002AC0F29080F7EE008A68
:1029F00038EEC00AB6EE008A20EE088AB0EE480A29
:102A000000F0BAFCDFED687A9FED687A9FED686AA6
:102A1000DFED685ADFED686AA8EE277ADFED677AA6
:102A2000A7EE086AE8EE257AE6EE086ADFED645A5A
:102A30009FED647AE7EE885AA6EE887ADFED627A37
:102A400010EE103AE5EE887A23F47F6323F00F034B
:102A5000B0EE476A9FED5D7AF0EE676AA6EE087AFF
:102A600007EE903AB0EE486AE6EE888AA7EEE76A8B
:102A700070EE276A27EE088A86EE267AC8EE286A64
:102A8000BDEC028BA0EE267A37EE870A30EE000A04
:102A900008BD20EE007ADFED447A9FED446ADFED59
:102AA000446A9FED445ADFED445AA7EE276ABDEC15
:102AB000028BE6EE076ADFED417A9FED416AE7EEB1
:102AC000057AE6EE875AA7EE876A9FED3E5ADFED5C
:102AD0003E7ADFED3E6AA5EE875AE6EE077AE5EE2E
:102AE000076AF7EE005AE7EE875A26EE877A9FEDDF
:102AF000386ADFED387AC7EE256AB0EE467AA0EE86
:102B0000667A30EE470A37EEC00A08BDB7EE007AA3
:102B100030EE070AF6EE007A60EE277ADFED226AE1
:102B20009FED226ADFED224ADFED225A9FED225A05
:102B30009FED268AA7EEA66ADFED206AE6EE274A19
:102B4000E7EEA56ADFED1E5A9FED1E6AA4EEA75AB6
:102B5000E6EEA75ADFED1C6AA5EE276AE5EEA76A46
:102B6000A6EE278AA6EEA77A28EE278AF0EE478AF5
:102B7000B0EE670A00F000FC88EE286ADFED167AF6
:102B8000B0EE407AE7EE067A9FED140A77EE877A88
:102B9000F0EE006AA7EEE60A18E700BFDB0FC93FB8
:102BA00000000000DB0F494008EF1138047F4F3A66
:102BB000461124BD2EC69D3DA80A4E3E613330BF4E
:102BC0002D57014090B0A6BE39D119C0ABAA2A3EFC
:102BD0006821A233DA0FC93F6821A2B3DA0F494056
:102BE00038B510EE105A25F00044B4F17E5F2DED9B
:102BF000048B00F085807ADCB4F17C5F0FDAB4F1ED
:102C0000485F80F29C80DFED697A70EE277AB7EE3C
:102C1000007AF4EEC77AF1EE10FA00F38D80FEF739
:102C2000E3FCF7EE007A37EEC00AB6EE008A20EE3B
:102C3000088A9FED5F7ADFED5F6A9FED5F6A9FED27
:102C40005F5ADFED5F5ADFED5F8AE8EE076A9FEDBE
:102C50005E7AA8EE067A9FED5D6AA6EE885AA7EE28
:102C6000086A9FED5B7ADFED5B6AE5EE085AA6EE37
:102C7000087AE5EE886AE7EE087AE6EE888AB0EE32
:102C8000480AB0EE679A00F077FB534B9C4268EE1F
:102C9000888A42DC10EE103A23F47F6323F00F039E
:102CA00006EE903AA6EEE68A70EE267A88EE895A0B
:102CB000C8EE274A9FED497ADFED497AB0EE006A07
:102CC000A4EEC67A30EE000AF0EE675AE6EEC65A77
:102CD00090EE057A37EE657A37EEC77A002D0ADC7A
:102CE000BDEC048BB1EE477AB0EE470A38BD70EE0A
:102CF000407A87EEA77ABDEC048BB0EE470A38BD68
:102D00009FED367ADFED377A20EE077ABDEC048B43
:102D1000A0EE277AB0EE470A38BD88EE896A9FEDAB
:102D2000327ADFED307AA0EE060AF0EE006AA0EE0D
:102D3000267A37EEC77AD1E7B0EE407ADBE760EE6D
:102D4000007A9FED1B7ADFED1B6A9FED1C6ADFEDB9
:102D50001A5A9FED1B5AE7EE876ABDEC048BA6EE6C
:102D6000A76A9FED197ADFED196AA7EEA57AA6EE9C
:102D7000275AE7EE276ADFED175A9FED156A9FED98
:102D8000117AE5EE275AA6EEA76AA5EEA77AF7EE26
:102D9000006AE6EE276A67EE277AB0EE407A87EEA1
:102DA000A66AA0EE067AB0EE470A38BDCAF24971AB
:102DB00008EF1138047F4F3A2EC69D3D461124BDC1
:102DC000A80A4E3EABAA2A3E613330BF2D570140C0
:102DD00039D119C090B0A6BE9999793F2EBD3BB3A9
:102DE000DB0F493FDB0FC93F2EBD3B3310B582B02F
:102DF000CDED010A019B23F00042B2F1FF4FF0EE4E
:102E0000407A30DC10EE100A20F00041B1F1FF4FA3
:102E100029DCB3F17E5F40D09C1704F0020444EA41
:102E2000D07431B372B3B2F1FF4F3ED0B1F1FF4F66
:102E300028D08A1AB2F1F45F4FEAE25132DA002B5D
:102E400040DA3C313EDA9FED330A012C4CD0022CA3
:102E500041D064B19FED307ADFED307A30EE070A71
:102E600030EE670A03E09DED017A37EE270A02B0E3
:102E700010BD022C0ED09FED2A0A032C00FE270A5B
:102E800002B010BD9FED270ADFED277A002820FE53
:102E9000270AECE79FED210AE9E702B0BDE8104000
:102EA000FEF7F6B99FED1F0ACFE7B1F1FF4F04F12E
:102EB000FF3420D0022C26D81C4B03EB840494ED65
:102EC000030AD4E79DED017A87EE870AFEF78CFBB3
:102ED000FEF7DEF9B9E79FED107ADFED107A30EEFC
:102EE000070A37EEC00AC2E710EE103A03F10043BA
:102EF00000EE103ABBE7022C08D80C4B03EB84041D
:102F000094ED000AB3E79FED030AB0E79FED080ACE
:102F1000ADE700BF000000002EBDBB33DB0F494012
:102F2000DB0F49C0DB0FC93FDB0FC9BF708E110833
:102F3000DB0F493F30B583B0CDED010A019D35F07F
:102F4000004041D010EE10EA2EF00043B3F1FF4FE5
:102F50003ADAB0F1FF4F37DC83423BDB0EF000443E
:102F60003AD01EF0FF4F56D1190200296FF07D02B2
:102F700004DD4900002902F1FF32FADC15F0FF4FB1
:102F800057D101026FF07D0C03D449000CF1FF3CD6
:102F9000FBD512F17E0F47DBCEF3160343F400039B
:102FA0001CF17E0F3ADBC5F3160040F40000B2EBD3
:102FB0000C0204D117E00FD04B00013A13D0191ABC
:102FC0000029F8DA5B00F8E7DDED017A60EE277A98
:102FD00087EEA70A03B030BD1D4B03EB547393ED8E
:102FE000000A03B030BD181A58BF03461BB9F3E7F7
:102FF0005B000CF1FF3CB3F5000FF9DB1CF17E0F19
:103000001CDBA3F500030CF17F0C234343EACC53F4
:1030100000EE103ADEE7DA157F3AAFE76FF07D0198
:10302000A1EB0C018840C2E76FF07D01891A8B404B
:10303000B6E74FEAE05CACF17F0CAAE76FF07D02E7
:10304000A2EB0C0C43FA0CF3234300EE103AC1E759
:10305000888E110808B510EE103A33F000422DEDBD
:10306000028B2BD0002B32DBB3F1FF4F41DAB3F5EB
:10307000000F35DB0021DA157F3A0A44D10FC1F188
:103080007F0102EBD272C3F3160307EE902A43EAE4
:10309000C15300EE103AB8EEE78AFEF7D7FADFED3B
:1030A000177A9FED177A20EE270ADFED167AA8EE41
:1030B000070AA8EE270ABDEC028B08BDBDEC028B07
:1030C0009FED117ADFED117A87EE270A08BDBDEC7E
:1030D000028B70EE407A9FED0D7A87EE870A08BD6D
:1030E000DFED0B7A60EE277A6FF0180117EE903A59
:1030F000C1E7BDEC028B30EE000A08BDD95BDE3EB5
:10310000DB27543580209A3E000000CC00000000F0
:103110000000004C70B510EE103A894A23F00044CC
:10312000944286B0054670DD864A944210EE106ADD
:1031300022DC002BDFED847A844A24F00F04B0EE09
:10314000407A40F3E480944270EE677A09BFDFED85
:10315000806A9FED807A9FED807A77EEE67A012093
:1031600077EEC76A77EEE67AC5ED006A77EEC77A42
:10317000C5ED017A06B070BD784A944254DDB4F1D1
:10318000FF4F49DAE215863AA4EBC25307EE903AB4
:10319000BDEEE77ADFED726AB8EEC77A77EEC77AEE
:1031A0008DED037A67EEA67ABDEEE77AB8EEC77AC0
:1031B00077EEC77A8DED047A67EEA67AF5EE407A5F
:1031C000F1EE10FACDED057A40F09080B5EE407A40
:1031D000F1EE10FA14BF022301236249019102218A
:1031E000009103A8294600F013FD002EC2DA95EDE8
:1031F000007AD5ED017AB1EE477AF1EE677A85ED86
:10320000007AC5ED017A4042B4E7002285ED000A5C
:103210004260002006B070BD70EE407A0020C5ED1F
:10322000017AC5ED007AA5E7FEF7DEF99FED4E7A4B
:103230009FED456AF6EE007AE0EE077A9FED457A5B
:10324000FDEEE77A17EE900AF8EEE76A1F28A6EE81
:10325000C60A66EE877AB1EE666A1EDC434A411EF4
:1032600024F0FF0352F82120934216D030EE677A03
:1032700085ED007A30EE470A002E30EE670A85EDC4
:10328000010ABFF677AFB1EE477AB1EE400A85ED9D
:10329000007A85ED010A40426CE730EE677AE2156C
:1032A00017EE103AC3F3C753C3EBD454082CDFDD39
:1032B000DFED277A9FED287AF0EE405AE6EE275AA6
:1032C00030EE650AA6EE270AF0EE407AD6EE877A4F
:1032D00035EEE77A17EE103AC3F3C753D21A192A1C
:1032E00006DCB0EE650A85ED007AC3E7032374E7D8
:1032F0009FED1F7A9FED1F5AB0EE650AA6EE070AF2
:1033000075EEC07AE6EE077AD6EE857AAEE794429D
:1033100070EE277A09BFDFED0E6A9FED0E7A9FED02
:103320000E7A77EEA67A4FF0FF3077EE876A77EE67
:10333000E67AC5ED006A77EE877AC5ED017A19E77E
:10334000D80F493FE3CB1640800FC93FD00FC93F8C
:10335000004435374344353708A3852E800F494351
:1033600000008043108F110884F9223F908E1108CD
:1033700000A3852E32318D24B1EEC00A704700BF04
:1033800010EE903A23F00043B3F1795F2DED028BFC
:103390002EDAFDEEC07B17EE903A002B65D020EEC2
:1033A000004B9FED358B9FED362B9FED373BA4EE09
:1033B000082B9FED375BA4EE023B9FED376BA4EE2D
:1033C000035B9FED377BA4EE056BA4EE067B24EE3A
:1033D000077B21EE400BB6EE006BA4EE070BBDECB5
:1033E000028BB7EE007B94EE060B37EE400B704776
:1033F0009FED218B20EE004B9FED212B9FED223B7B
:10340000A4EE082B9FED225BA2EE043B9FED226B06
:10341000A3EE045B9FED227BA5EE046B224AA6EE91
:10342000047B934227EE047BD3DD204A934217DCD2
:10343000B7EE006B0020A3F5001141EC150B36EE42
:10344000456BB6EE003B21EE400B94EE035BA4EE21
:10345000070BBDEC028B35EE400B36EE400B704790
:10346000B6EE076BB5EE025BEBE7B7EE000BBDEC1B
:10347000028B7047AFF30080D43888BEE9FAA8BD4C
:10348000C4B1B4BD9EEE213EAD529C804F7E92BE33
:103490009015CB19A001FA3E7751C1166CC156BFE9
:1034A0004C5555555555A53F3233D33F0000E93FA4
:1034B0002DE9F04F2DED088BADF5157D1C460493DD
:1034C0000791AD4BA69912F1140F53F82150824683
:1034D00004F1FF38C0F2A682A849D31E81FB030184
:1034E000DB17C3EBA10303930133A3EB8303DB00DF
:1034F000D3180693039B15EB0801A3EB08031AD41A
:1035000001319FED976BA79819441CAA0AE050F867
:10351000234007EE904A0133B8EEE77B8B42A2ECE2
:10352000027B08D0002BF2DAB0EE467B01338B42EF
:10353000A2EC027BF6D1002DC0F2D482049B1CAA1F
:1035400002EBC3046CAE4FEAC30C4046EF180AEB23
:10355000C301B8F1000F9FED827B09DB2246534681
:10356000B3EC025B32ED026B8B42A5EE067BF7D12A
:103570000130B842A6EC027B04F10804E9D107ABA4
:1035800008AF03EB85099FED789B07EB85039FED63
:10359000788B083BDDF818B005930AEB0C046CAE91
:1035A0002946019594AB03EBC103002913ED280BC9
:1035B00016DD06EBC1033A4620EE097B33ED025BD4
:1035C000B0EE406BBDEEC77BB342B8EEC77BA7EE53
:1035D000486BBDEEC66B37EE050BA2EC016AEBD172
:1035E0005846029101F0C8F8B0EE40ABB4EE000BC3
:1035F0002AEE000B01F034F8B2EE007BA0EE47ABF0
:10360000BDEECABBBBF1000FB8EECB7B02993AEE20
:1036100047AB75DD01F1FF3CCBF1180357F82C20C7
:1036200042FA03F000FA03F3D31ACBF117051BEEAD
:10363000102A43FA05F50244002D47F82C300BEE12
:10364000102A65DCB5EE40ABF1EE10FA40F0C78011
:10365000019B01F1FF3C63450EDC01F18042013A20
:1036600007EB8202002052F804394A4540EA030081
:10367000F9D1002840F0F580019B013B57F8233039
:10368000002B40F0E980059B012553F80429013502
:10369000002AFAD001F1010E0D447046049B194432
:1036A000039B03EB0E0C0CF1804CA79B0CF1FF3C31
:1036B00003EB8C0C1CAB06EBCE0E03EBC1019CEDB7
:1036C000017AB8EEC77BB8F1000F81ED007B0CF1F9
:1036D000040C0A469FED226B01F1080109DB5346F9
:1036E00001E032ED027BB3EC025BA342A5EE076B77
:1036F000F7D10130A842AEEC026BE0DD294651E77C
:1037000040F0A0804B1E57F82350ED15002D99DD99
:103710001BEE103A002903F101030BEE103A40F3BF
:1037200097813A68002A40F0858001292FD03B46D6
:10373000012053F8042F002A7FD0431CC2F180726D
:10374000994247F8202021DD57F8232007EB810C10
:1037500007EB83036FF07F4013E000BFAFF30080FF
:103760000000000000000000000000000000703EAB
:10377000000000000000704128921108ABAAAA2A9C
:103780001A68821A43F8042B6345F9D10122BBF170
:10379000000F0DDDBBF1010F00F03C81BBF1020F0A
:1037A00006D1481E57F82030C3F3150347F82030E0
:1037B000022D7FF447AFB7EE000B30EE4AAB002A84
:1037C0003FF440AF5846029100F0D6FF3AEE40ABCE
:1037D000B5EE40ABF1EE10FA02993FF439AF069C1A
:1037E000B0EE4A0B604202958B46019D00F0C4FF8B
:1037F0009FEDBF6BB4EEC60BF1EE10FA029AC0F269
:103800004D819FEDBD7B20EE077BBDEEC77B0BF1AD
:103810000103B8EEC75BA5EE460BBDEEC00B183436
:1038200010EE101A47F82B1017EE101A069447F8EE
:1038300023102DE00123002080E7013088427FF42F
:1038400078AFA4E7B6EE007BB4EEC7ABF1EE10FAAA
:1038500080F2ED800025F5E601F1010E7046754617
:103860001CE78B460699A1F1180057F82C1006901A
:103870002A466346019D59B90BF18041023907EB95
:10388000810151F80449013B1838002CF9D0069009
:103890000698B7EE000BCDE9012300F06DFF029B07
:1038A000019A002BC0F236816CA99FED936B01EB5E
:1038B000C30403F1010E07EB8E014FEAC30C04F1C0
:1038C000080031ED017AB942B8EEC77B27EE007BE4
:1038D00020EE060B20ED027BF3D19FED894B2746AE
:1038E00000260DF58878002D9FED877B10DBB0EE6C
:1038F000446B874C3846002103E08E4208DBB4EC71
:10390000026BB0EC025B01318D42A5EE067BF4DA6E
:1039100008EBC601B34281ED007BA7F1080706F171
:10392000010101D00E46DEE7A69902291EDC00291E
:1039300000F3908010D19FED747B0CF10803434499
:1039400033ED026B984537EE067BF9D10AB1B1EE43
:10395000477B079B83ED007B1BEE103A03F00700CB
:103960000DF5157DBDEC088BBDE8F08FA6990329F8
:10397000F2D1002B00F0EB8008EB0C0191ED006B15
:1039800008EBC30131ED027BB0EE465B884536EEB5
:10399000076B37EE467B81ED006B37EE057B81EDE3
:1039A000027BEFD1012B40F3D28003F10053C444DA
:1039B000013BDB009CED006B03F10801414446A88C
:1039C00031ED027BB0EE465B884236EE076B37EE98
:1039D000467B81ED006B37EE057B81ED027BEFD1FD
:1039E0009FED497B1033434408F1100133ED026B26
:1039F000994237EE067BF9D1002A57D1D8E9000168
:103A0000D8E90223079C84ED047BC4E90001C4E9E2
:103A10000223A1E7481E57F82030C3F3160347F8E6
:103A20002030C5E600216FF01703039160E51BEE1F
:103A3000103A002903F101030BEE103AC8BF02252A
:103A40003FF76FAEB7EE007B37EE4AAB0225F9E5E4
:103A500000229CE69FED2C7B08EBCE0E3EED026B28
:103A6000F04537EE067BF9D198ED006B82BB0799E4
:103A7000002B81ED007B36EE477B0BDD46A8012154
:103A8000B0EC026B01318B4237EE067BF8DA0AB1FB
:103A9000B1EE477B079B83ED027B5DE7BDEEC00B7C
:103AA00010EE103A47F82B305B46F1E698ED005BDC
:103AB000B1EE477B98ED026BB1EE455B079BB1EE33
:103AC000466B83ED005B83ED026B83ED047B43E784
:103AD0000799B1EE475B002B81ED005B36EE477B2B
:103AE000CCDCD5E7049B4FEAC30C48E5AFF300807C
:103AF0000000000000007041000000000000703E67
:103B000000000040FB21F93F000000000000000021
:103B100040921108A699022909DC002912DC7FF4E1
:103B20001BAF9FED0D7B002A3FF413AF0FE7A69B61
:103B3000032B7FF411AF9FED087B0DF58878002AE9
:103B4000B4D15BE79FED047B0DF588788CE79FEDA2
:103B5000027B002AAAD151E700000000000000000B
:103B600010EE903A23F00043B3F1795F04DAFDEEF2
:103B7000C07B17EE903A5BB320EE007B9FED162BD7
:103B80009FED173B9FED184BA7EE023B9FED185B97
:103B9000A3EE074B9FED186BA4EE075BA5EE076B3A
:103BA00020EE075B30B99FED164BA7EE064BA4EE57
:103BB000050B70479FED144B26EE456BB6EE003BB0
:103BC000A1EE036B96EE071BA5EE041B30EE410B36
:103BD000704700BFAFF300807CD5CF5A3AD9E53D9E
:103BE000EB9C2B8AE6E55ABE7DFEB157E31DC73E2E
:103BF000D561C119A0012ABFA6F810111111813F8A
:103C0000495555555555C5BF495555555555C53F48
:103C10002DE9F04F2DED048BDBB01C46039306918C
:103C2000A24B6899089253F82150111D824604F165
:103C3000FF38C0F2A382D31E48BF131DDB100293CE
:103C40000133DB000793DDE907239B1A0593029BF1
:103C500015EB0801A3EB080316D401319FED947A0C
:103C6000699819441EAA002BA4BF50F8234007EE00
:103C7000904A03F10103ACBFF8EEE77AF0EE477A21
:103C80008B42E2EC017AEED1002DC0F2E782039B79
:103C90001EAA02EB830446AE4FEA830C4046EF189F
:103CA0000AEB8301B8F1000FDFED817A09DB2246D0
:103CB0005346F3EC016A32ED017A8B42E6EE877AE5
:103CC000F7D10130B842E6EC017A04F10404E9D1FD
:103CD00009AB0AAF03EB850907EB8503083B9FEDB2
:103CE000769ADFED748A059804930AEB0C0446AECD
:103CF00000955AAB03EB8503002D13ED140A4FEA30
:103D0000850B16DD06EB85033A4660EE097AB0EEC8
:103D1000407AFDEEE77A73ED016AF8EEE77AB34296
:103D2000A7EEE87A37EEA60ABDEEC77AA2EC017AD2
:103D3000EBD1019000F0EAFDB0EE408AB4EE000A4B
:103D400028EE000A00F09EFDF2EE007AA0EE678AEF
:103D500001980028FDEEC89AF8EEE97A38EE678AF5
:103D600079DD05F1FF3EC0F1080357F82E1041FA46
:103D700003FC0CFA03F3CB1AC0F1070219EE901AF8
:103D800043FA02F26144002A47F82E3009EE901AF5
:103D900069DCB5EE408AF1EE10FA40F0C080009B7D
:103DA00005F1FF3B5B4510DC05F18043013B07EB70
:103DB00083030021944653F804294B4541EA02014C
:103DC000F9D16246002940F0F280009B013B57F890
:103DD0002330002B40F0E780049B4FF0010C53F898
:103DE00004290CF1010C002AF9D06B1CAC449E464E
:103DF000039A5119029A02EB030B0BF1804B699A5B
:103E00000BF1FF3B06EB83051EAB02EB8B0B03EBC9
:103E10008101DBED017A9FED267AF8EEE77AB8F1C1
:103E2000000F0BF1040BC1ED007A0A4601F1040109
:103E300009DB534601E072ED017AF3EC016AA3421B
:103E4000A6EEA77AF7D10EF1010EE645A5EC017AB0
:103E5000DFDD65464DE740F09C806B1E57F8232060
:103E60001212002A95DD19EE903A002D03F101039C
:103E700009EE903A40F39881396800297FD1012DED
:103E800026D03B464FF0010C53F8041F00297AD08E
:103E90000CF10103C1F580719D4247F82C1016DD2D
:103EA00057F82310BB4407EB83030AE0789211080C
:103EB00000000000000080430000803B0000C93F7C
:103EC0001968C1F1FF0143F8041B5B45F8D10121DA
:103ED00000280CDD012800F04881022807D105F1F7
:103EE000FF3C57F82C3003F03F0347F82C30022AF0
:103EF0007FF44FAFB7EE000A30EE488A00293FF456
:103F000048AF0992019000F001FD38EE408A099A0D
:103F10000198B5EE408AF1EE10FA3FF440AF0292FC
:103F2000DDE90732B0EE480A981A0195009D00F0CD
:103F3000EDFC1FED207AB4EEC70AF1EE10FADDE9D0
:103F40000132C0F259815FED247A059960EE277A3B
:103F50000831FDEEE77A0591F8EEE77A03F1010BFF
:103F6000A7EEC70AFDEEE77ABDEEC00A10EE101A02
:103F700047F8231017EE903A47F82B302EE0012334
:103F80004FF0000C86E70CF1010CAC457FF47CAFE0
:103F90009EE7F6EE007AB4EEE78AF1EE10FA80F2D0
:103FA000F2800022F5E66B1C9E469C4620E70599B0
:103FB000A1F1080057F82B1005902B46009D69B918
:103FC00003F18043023B07EB8303014653F80409E6
:103FD0000BF1FF3B08390028F8D0059105980092B5
:103FE000B7EE000A00F092FCBBF1000F009AC0F29D
:103FF00028814FEA8B0E46AB03EB0E060EF1040C44
:104000001FED537A07EB0C03311D73ED017AF8EEC7
:10401000E77ABB4267EE807A20EE070A61ED017A0B
:10402000F3D1002D1FED5B6A4FF0000420DB9348B5
:10403000DFED937AB0EE467A3146002303E09C42EE
:1040400008DBB0EC017AF1EC016A01339D42E6EE47
:10405000877AF4DA5AAB03EB8403A34543ED287A5D
:10406000A6F1040604F1010305D0002D1C46DEDA9A
:10407000DFED837AEEE7689902291CDC002900F362
:1040800095800FD132ABDFED7E7A9C443CED017A16
:10409000634577EE877AF9D10AB1F1EE677A069B2C
:1040A000C3ED007A19EE903A03F007005BB0BDEC67
:1040B000048BBDE8F08F689B032BF3D1BBF1000F9D
:1040C00000F0D4800EF5B4736B4432A913ED287A56
:1040D00001EB8B0373ED017AF0EE476A37EE277A36
:1040E000994277EEC77A83ED007A77EEA67AC3ED30
:1040F000017AEFD1BBF1010F40F3B8800BF1804B97
:104100000EF5B4730BF1FF3B0DEB030E4FEA8B0B77
:104110000BF104031EED287A0B4433A873ED017AEA
:10412000F0EE476A37EE277A984277EEC77A83ED4A
:10413000007A77EEA67AC3ED017AEFD10BF1080B86
:10414000DFED4F7A01EB0B03083133ED017A994231
:1041500077EE877AF9D1002A56D10699329A339BA5
:104160000A604B60C1ED027A9CE705F1FF3C57F80D
:104170002C3003F07F0347F82C30B8E60823079370
:10418000002302935FE519EE903A002D03F101033D
:1041900009EE903AC8BF02223FF76EAEF7EE007A02
:1041A00037EEC88A0222F4E5002191E632A9DFED5C
:1041B000347A01EB830333ED017A994277EE877A03
:1041C000F9D19DED327A8ABB069BBBF1000FC3ED9E
:1041D000007A77EE677A0BDD33A90123B1EC017A1F
:1041E00001339B4577EE877AF8DA0AB1F1EE677A08
:1041F000069BC3ED017A55E7BDEEC00A9B4610EE63
:10420000101A47F82310E9E6DDED326A9DED337AA6
:10421000069BF1EE666AB1EE477AF1EE677AC3ED7E
:10422000006A83ED017AC3ED027A3BE7069BF1EE6B
:10423000676ABBF1000F77EE677AC3ED006ACBDCEB
:10424000D4E7689B022B0DDC002B14DC7FF42AAF33
:10425000DFED0B7A002A3FF422AF1EE7039B4FEA03
:10426000830C35E5689B032B7FF41CAFDFED047AEC
:10427000002AC9D171E7DFED027AA2E7889211081E
:104280000000000008B510EE103A23F00042B2F131
:10429000465FF0EE407A0FDABDEEC07A17EE101AE4
:1042A00001BB431C134300F0A080012803D0BFEEE4
:1042B000007A87EE270A08BD50498A4212DB002B9C
:1042C000B8BFF1EE407A9FED4E7A9FED4E0AB8BF2F
:1042D000F1EE600A70EE677A37EE600ADFED4A0AA7
:1042E00070EE277A67EEA76ADFED484ADFED485A9D
:1042F0009FED485A9FED486A404926EEA67A8A42C9
:10430000E7EE245AA7EE056ADFED444A9FED445AD2
:10431000E5EE874AA6EE075ADFED425A9FED426A64
:10432000E4EE875AA5EE076ADFED404A9FED405A5A
:10433000E5EE874AA6EE075A9FED3E6ADFED3E5A4C
:10434000A4EE876AE5EE075AB0EE467AA5EEA67AA5
:1043500027EEA65AB0EE606AA7EE056ADFED374A8F
:10436000E6EE260AE5EE240A37EEA00A1FDA012857
:10437000A1D0BFEE007AC7EE006A314B10EE102AD2
:104380001A4006EE102A16EE902A76EE677A13404F
:1043900000EE103AB7EE007A70EEE70AF0EE477AD8
:1043A000E6EE007AE0EE807AA7EEA60A08BD07EEF8
:1043B000100AB8EEC77A60EE005A30EE070A9B1773
:1043C000C5EE806A03F00203C3F10103B0EE006A98
:1043D00076EEE00A00EE103A77EEE07AB8EEC00A28
:1043E000A7EEC67A20EE070A08BDFDF7FDF8B7EE86
:1043F000007AF0EE407A87EE270A08BD40A12C3FF4
:1044000068212233DA0F493F000000005FAE9BB7FE
:1044100045F4A3388453D9377AC09538C8261A3A58
:10442000B937813916696B3B48DEBE3AA427B33CE5
:104430001F37113C8988083ED10D5D3DABAAAA3ECD
:1044400000F0FFFF38B5B0EE407B17EE905A794B85
:1044500025F000449C422DED0C8B16DD764B9C42E2
:104460000EDC09D09FED577B9FED580B002D37FEDA
:10447000000BBDEC0C8B38BD10EE103A002BF1D0C8
:1044800037EE070BBDEC0C8B38BD6C4B9C4259DCF6
:10449000A3F1DE739C4249DD4FF0FF329FED4DAB3F
:1044A00027EE075B25EE056B9FED4C8B9FED4D1BBB
:1044B000A6EE0A8B9FED4D3BA8EE061B9FED4DBB74
:1044C000A1EE063B9FED4DDBA3EE06BB9FED4D9BA2
:1044D000ABEE06DB2DEE05DB9FED4C0B9FED4D2B80
:1044E000A6EE090B9FED4D4BA0EE062B9FED4DCB9D
:1044F000A2EE064B531CA4EE06CB2CEE06CB36D018
:104500003DEE0CDB4E4B03EBC20393ED000B93ED42
:10451000086B9DEE070B30EE470B002D36EE400B7F
:10452000A7DAB1EE400BBDEC0C8B38BD9FED3F6BB5
:10453000B7EE005B30EE066BB4EEC56BF1EE10FA31
:10454000AADD96E700F082F83E4B9C4218DCA3F50A
:1045500050239C4229DCB0EE007BBFEE006B30EEB6
:10456000075BA0EE076B002286EE057B96E73DEE2B
:104570000CDBADEE477BBDEC0C8BB0EE470B38BDD2
:10458000314B9C420BDAB7EE087BB7EE006B30EE96
:10459000475BA0EE076B022285EE067B7EE7BFEE4F
:1045A000006B032286EE007B78E7B7EE007B0122EA
:1045B00030EE476B30EE070B86EE007B6EE700BFF8
:1045C000AFF30080182D4454FB21F93F182D4454BB
:1045D000FB21F9BF11DA22E33AAD903FEB0D7624CF
:1045E0004B7BA93F513DD0A0660DB13F6E204CC51D
:1045F000CD45B73FFF8300922449C23F0D55555525
:104600005555D53F2F6C6A2C44B4A2BF9AFDDE529B
:104610002DDEADBF6D9A74AFF2B0B3BF711623FE3D
:10462000C671BCBFC4EB98999999C9BF9C750088A5
:104630003CE4377EFFFF0F440000F07FFFFFDB3FCD
:10464000B0921108FFFFF23F0080034051EC100BC5
:1046500010EE102A21F0004343EC102B704700BFEE
:1046600082B08DED000B01990098C1F30A52A2F2BD
:10467000FF33132B31DC002B21DB394A1A4101EACD
:10468000020C5CEA000C2DD09FED337B9DED006B9E
:1046900036EE077BB5EEC07BF1EE10FA09DD00299E
:1046A00004DA4FF4801040FA03F3194421EA0201BE
:1046B00000200B46024643EC102B02B070479FEDE2
:1046C000267B30EE077BB5EEC07BF1EE10FAF0DD15
:1046D000002928DB00200146EBE7332B06DDB3F58C
:1046E000806F1BD09DED000B02B07047A2F2134209
:1046F0004FF0FF3C2CFA02F20242F3D09FED167B02
:104700009DED006B36EE077BB5EEC07BF1EE10FA47
:10471000CFDD002910DB20EA0200CAE79DED007B17
:1047200037EE070BE0E721F000430E4A184300285C
:1047300018BF11460020BCE7142B09D04FF0010C24
:10474000C3F134030CFA03F3181828BF6144E2E7FD
:104750000131E0E7AFF300809C7500883CE4377ED0
:10476000FFFF0F000000F0BF9FED010B704700BF7F
:10477000000000000000F87F53EC102BC3F30A5137
:1047800000B59C4671BB10EE101A23F0004C5CEA99
:10479000010125D09FED2E7B394920EE077B884211
:1047A00053EC172B4CDBC3F30A519C4636390144BA
:1047B00040F2FE7E71451DDC002937DC11F1350F1A
:1047C00025DA4CF25031884214DC9FED230B9FED2B
:1047D000246BB0EE407B002B20FE060B20EE070B77
:1047E0005DF804FB40F2FF7E7145E0D130EE000B36
:1047F0005DF804FB9FED1C0B9FED1D6BB0EE407B45
:10480000002B20FE060B20EE070B5DF804FB2CF0BE
:10481000FF4C36312CF4E00C9FED177B4CEA015332
:1048200043EC102B20EE070B5DF804FB2CF0FF4C43
:104830002CF4E00C4CEA015343EC102B5DF804FB24
:104840009FED050B27EE000B5DF804FBAFF3008036
:10485000000000000000504359F3F8C21F6EA5018C
:1048600059F3F8C21F6EA5819C7500883CE4377E21
:104870009C7500883CE437FE000000000000903C7E
:10488000B03CFFFF10EE102AC2F3C7537F3B162B3C
:1048900022F0004128DC002B18DB194919410A429B
:1048A00021D0DFED187A70EE277AF5EEC07AF1EEBE
:1048B00010FA18DD002A04DA4FF4000040FA03F37E
:1048C0001A4422EA010300EE103A7047DFED0D7A38
:1048D00070EE277AF5EEC07AF1EE10FA03DD002AC9
:1048E00008DB9FED090A7047B1F1FF4FFBD330EEB3
:1048F000000A7047FFEE007A002900FE270A704781
:10490000FFFF7F00CAF249710000000082B08DED08
:10491000010A019B33F0004229D0B2F1FF4F22D2AD
:1049200013F0FF4F27D19DED017ADFED297A294B56
:1049300067EE277A9842CDED017A36DB019BC3F30F
:10494000C752193A0244FE2A19DD9FED230A9FED52
:10495000237A019BF0EE407A002B20FE070A20EE1E
:10496000270A02B0704730EE000A02B070479DED92
:10497000010A02B07047D20D0244FE2AE5DC002A8B
:104980000BDC12F1160F17DA4CF250339842DCDCD4
:104990009FED130A9FED137ADBE723F0FF4343EA11
:1049A000C25300EE103A02B070479FED0D0ADDEDE4
:1049B000017A27EE800AD8E7193223F0FF4343EA51
:1049C000C253DFED097A07EE103A27EE270ACCE74B
:1049D0000000004CB03CFFFFCAF24971CAF249F135
:1049E0006042A20D6042A28D0000003370B54FF00E
:1049F000FF0C4CF4E06C1CEA11541DBF1CEA13556B
:104A000094EA0C0F95EA0C0F00F0DEF82C4481EAD2
:104A1000030621EA4C5123EA4C5350EA013518BFF2
:104A200052EA033541F4801143F4801338D0A0FBDF
:104A300002CE4FF00005E1FB02E506F00042E0FB8C
:104A400003E54FF00006E1FB03569CF0000F18BF92
:104A50004EF0010EA4F1FF04B6F5007F64F540743A
:104A600004D25FEA4E0E6D4146EB060642EAC621CD
:104A700041EA55514FEAC52040EA5E504FEACE2E3A
:104A8000B4F1FD0C88BFBCF5E06F1ED8BEF1004F3D
:104A900008BF5FEA500E50F1000041EB045170BDB9
:104AA00006F0004646EA010140EA020081EA0301FD
:104AB000B4EB5C04C2BFD4EB0C0541EA045170BDF9
:104AC00041F480114FF0000E013C00F3AB8014F173
:104AD000360FDEBF002001F0004170BDC4F10004BC
:104AE000203C35DA0C341BDC04F11404C4F120053D
:104AF00000FA05F320FA04F001FA05F240EA020098
:104B000001F0004221F0004110EBD37021FA04F6CD
:104B100042EB06015EEA430E08BF20EAD37070BD87
:104B2000C4F10C04C4F1200500FA04F320FA05F0E6
:104B300001FA04F240EA020001F0004110EBD370E8
:104B400041F100015EEA430E08BF20EAD37070BD58
:104B5000C4F1200500FA05F24EEA020E20FA04F331
:104B600001FA05F243EA020321FA04F001F00041E0
:104B700021FA04F220EA020000EBD3705EEA430E51
:104B800008BF20EAD37070BD94F0000F0FD101F080
:104B90000046400041EB010111F4801F08BF013CB9
:104BA000F7D041EA060195F0000F18BF704703F0F7
:104BB0000046520043EB030313F4801F08BF013D7E
:104BC000F7D043EA0603704794EA0C0F0CEA13553A
:104BD00018BF95EA0C0F0CD050EA410618BF52EAF4
:104BE0004306D1D181EA030101F000414FF00000FA
:104BF00070BD50EA410606BF1046194652EA430608
:104C000019D094EA0C0F02D150EA013613D195EA7B
:104C10000C0F05D152EA03361CBF104619460AD1C3
:104C200081EA030101F0004141F0FE4141F47001CD
:104C30004FF0000070BD41F0FE4141F4780170BDBD
:104C40004FEA410212F5001215D211D56FF47873B4
:104C5000B3EB625212D94FEAC12343F0004343EA57
:104C6000505311F0004F23FA02F018BF4042704732
:104C70004FF00000704750EA013005D111F00040BC
:104C800008BF6FF0004070474FF00000704700BF52
:104C90004FEA4102B2F1E04324BFB3F5001CDCF15E
:104CA000FE5C0DD901F0004C4FEAC0024CEA507096
:104CB000B2F1004F40EB830008BF20F001007047C5
:104CC00011F0804F21D113F13872BCBF01F00040C8
:104CD000704741F480114FEA5252C2F11802C2F1FA
:104CE000200C10FA0CF320FA02F018BF40F001007B
:104CF0004FEAC1234FEAD32303FA0CFC40EA0C002D
:104D000023FA02F34FEA4303CCE77FEA625307D169
:104D100050EA01331EBF4FF0FE4040F440007047A0
:104D200001F0004040F0FE4040F40000704700BF3A
:104D3000002103F043B800BF0A22002103F0B6B9F6
:104D40000A23002203F092B90A22002103F0AEB92F
:104D50000A23002203F08AB910B5054C34B113467A
:104D60000A4601460220AFF3008010BD204610BD68
:104D700000000000014B1868704700BF042200309B
:104D800010B4044C03460A4620685DF8044B1946EB
:104D900000F010B80422003000B5054B83B0014686
:104DA00001AA186800F006F803B05DF804FB00BF24
:104DB000042200302DE9F047DFF87480064689466A
:104DC000174604F09DF9D8F8005055B199F8003015
:104DD0001C4673B14C4602E014F8013F3BB13D2B39
:104DE000FAD1304604F08EF90020BDE8F087A4EB3C
:104DF000090428680028F4D02246494601F0AEFD97
:104E000028B92B681A5D3D2A03EB040A04D055F833
:104E1000040F0028F0D1E4E7D8F80030ED1AAD1007
:104E200030463D6004F06EF90AF10100BDE8F087FC
:104E30006822003000B583B001AAFFF7BBFF03B0C2
:104E40005DF804FBF8B5D0E90067634A00230C461F
:104E500030463946FBF77CFD5F4A05463946304609
:104E60000023FBF775FD002AC0F2AC8005F52F2367
:104E700003F66C235948A0FB0250C00A4FF461614D
:104E800001FB10225649A060A1FB020149095548C7
:104E90006160C1EB0111A2EB8102D91C80FB0150C2
:104EA00008442260CA17C2EBA002C2EBC2028A1AEF
:104EB00048BF0732002BA26179DB4B4AD91782FB2E
:104EC0000302C1EBE2314948494A4A4E00FB013036
:104ED0008508A2FB053200EBD222A6FB0535464B26
:104EE000A2EBD5120509A3FB0535A2EB1512434D24
:104EF000A5FB023CA2EB0C030CEB530C404D9308BA
:104F0000A6FB03234FEA1C22A5FB0265DB09C3EBCA
:104F10005513034440F26D1000FB123303EB83057D
:104F200038480235A0FB050C4FEADC1C40F2F9566C
:104F30000CEBCC00B54200EB0010334D00F1020049
:104F4000A5FB00504FF4C87694BF02256FF0090509
:104F500006FB01216544012D98BF01315E1CB3F5AC
:104F6000997FA6EB90000BD3A3F59973A1F26C7116
:104F7000E3610023E060C4E9045123622046F8BDE8
:104F800096070BD0214E06FB02F2214EB6EB321FE4
:104F90002CBF012200223B331344E7E71B4E1D4F79
:104FA00002FB06F6B7EBB60FECD20122F3E70E498F
:104FB000A3F50E32A2F52C7281FB0201D217C2EBCF
:104FC000E13180E702F5A83205F52F2302F5C07222
:104FD00003F66B234EE700BF80510100C5B3A291D9
:104FE0008988888893244992BD066B394FC5FDFF97
:104FF0007F206B39D97CC65941D6720061F319679D
:105000001F85EB51D7802BD6CDCCCCCC295C8FC261
:105010000AD7A300285C8F02024B1844407800F0A6
:1050200008007047F0921108F03070470048704750
:1050300060230030004870476023003001F0FF011A
:10504000102A2BDB10F0070F08D010F8013B013AB3
:105050008B422DD010F0070F42B3F6D1F0B441EAE5
:10506000012141EA014122F007047FF000070023FB
:10507000F0E80256083C85EA010586EA010685FA51
:1050800047F5A3FA87F586FA47F6A5FA87F68EB9AB
:10509000EED1F0BC01F0FF0102F0070232B110F8CE
:1050A000013B013A83EA010313B1F8D100207047B4
:1050B00001387047002D06BF35460338073815F014
:1050C000010F07D1013015F4807F02BF013015F4C4
:1050D000C03F0130F0BC0138704700BF032A70B5F3
:1050E00015D940EA010C1CF0030F04460B4621D1F0
:1050F000194620460E680568B54204F1040403F120
:10510000040317D1043A032A20461946F0D8541E46
:10511000A2B100F1FF3C013901E0C3180CD01CF82A
:1051200001EF11F8012F9645A4EB0C03F5D0AEEB7F
:10513000020070BD541EECE7184670BD104670BDED
:10514000844641EA000313F003036DD1403A41D392
:1051500051F8043B40F8043B51F8043B40F8043B51
:1051600051F8043B40F8043B51F8043B40F8043B41
:1051700051F8043B40F8043B51F8043B40F8043B31
:1051800051F8043B40F8043B51F8043B40F8043B21
:1051900051F8043B40F8043B51F8043B40F8043B11
:1051A00051F8043B40F8043B51F8043B40F8043B01
:1051B00051F8043B40F8043B51F8043B40F8043BF1
:1051C00051F8043B40F8043B51F8043B40F8043BE1
:1051D000403ABDD2303211D351F8043B40F8043B81
:1051E00051F8043B40F8043B51F8043B40F8043BC1
:1051F00051F8043B40F8043B103AEDD20C3205D391
:1052000051F8043B40F8043B043AF9D2043208D088
:10521000D2071CBF11F8013B00F8013B01D30B88FA
:1052200003806046704700BF082A13D38B078DD0D8
:1052300010F003038AD0C3F10403D21ADB071CBFAA
:1052400011F8013B00F8013B80D331F8023B20F814
:10525000023B7BE7043AD9D3013A11F8013B00F84D
:10526000013BF9D20B7803704B7843708B788370D5
:10527000604670472DE9F04F012BADF21C4D0746FB
:105280008A46154640F21F814FF001090024484626
:105290004FF0FF364A4606E0A2EB0609144601200D
:1052A000221893420FD9A91915F802C0095C8C4540
:1052B000F2D300F08C804FF00109264648464C445A
:1052C00022189342EFD84FF0010E002470464FF0A1
:1052D000FF3C724606E0A2EB0C0E14460120221899
:1052E00093420FD905EB0C0115F80280095C884543
:1052F000F1D872D04FF0010EA446704674442218C3
:105300009342EFD80CF1010C0136664501D8F14605
:10531000664605AA0DF2144142F8043F8A42FBD1C9
:10532000002B00F0CB805C1E691E05EB040C0DF118
:10533000180811F8010FCA431A442A44614548F875
:105340002020F6D1324605EB090128460193FFF7EC
:10535000C5FE019B002868D1AAEB0301A3EB09035A
:10536000024602930346701E0590C6F10100CDE986
:1053700003908A4601950AE022B1039A9142029A6B
:1053800038BF11460B4453454FF0000248D807EB95
:10539000030B1BF8041058F821100029ECD1B2427D
:1053A000114638BF3146A1421DD201984D1E054419
:1053B0005818384402E00131A14214D210F801CB50
:1053C00015F801EFE645F6D0049A1344DAE7814573
:1053D00012BF01304C44012062E770450ABF241817
:1053E000013001207BE7B242059972D2019D9819E4
:1053F0003844354402E08A425ED0614610F801CD5F
:1054000015F801EDE64501F1010901F1FF3CF2D08B
:1054100001324A455BD8039A13445345029AB6D9E0
:1054200000200DF21C4DBDE8F08FAAEB030A9B1B78
:10543000B34238BF33464FF00009013307EB090090
:105440000293C6F101030193035D58F8233006F17E
:10545000FF3B4BB19944D145E2D807EB0900035D0E
:1054600058F82330002BF5D1A64213D206EB0902DF
:105470003A4405EB0B01334602E00133A34209D263
:1054800012F801CB11F801EFE645F6D0019A9144EC
:105490009944E0E7002EC4D006EB09013944AA196B
:1054A00001E0AB42BDD012F801ED11F801CDE645A7
:1054B0001346F6D0029BCDE79146A9E74FF0FF34A3
:1054C0000DF118083EE74FF00109002621E7584684
:1054D000A7E7B1469CE700BF2DE9F0470446C0B0FE
:1054E000002B69D0012B0D4690461F4600F08780A7
:1054F0008B425DD8CD1A022B00EB050660D0B3F5C8
:10550000807F00F2838000214FF4807268465D1E28
:1055100000F0FEF840460121024643781278A3EBE2
:10552000C203DBB201300DF8031001318D42F3D814
:1055300008EB07034FF0000A13F8022C18F80530A7
:10554000A3EBC203DBB21DF803900DF80350A5EBEB
:105550000909B44201D92BE063B92C44A64214F8DE
:10556000013C94F800C0ACEBC30C5FFA8CFC1DF856
:105570000C30F1D29D42A4EB0304EAD80F2D07D9D9
:10558000042208EB0A0104EB0A00FFF7A7FD60B94B
:105590002A4641462046FFF7A1FD68B1BAF1030F44
:1055A0008CBFAAF1040AA7F1050A4C44B442D4D92D
:1055B000002040B0BDE8F087204640B0BDE8F0874D
:1055C00013785578017845EA0345034613F8012F0F
:1055D0009E4242EA01421DD39542EDD0013601E0E0
:1055E0009542E6D0184613F8011FB34241EA024241
:1055F000F6D1954208BF06F1FF30D9D1D9E711782D
:105600002A4640B0BDE8F047FFF718BD40B0BDE8FE
:10561000F0472FE61E46ECE788420DD98B188342EF
:105620000AD900EB020CBAB1624613F801CD02F8B8
:1056300001CD9942F9D170470F2A0ED8034602F1E5
:10564000FF3C4AB10CF1010C013B8C4411F8012BD9
:1056500003F8012F6145F9D1704740EA01039B0728
:1056600050D1A2F1100370B501F1200C23F00F0509
:1056700001F1100E00F11004AC441B095EF8105C3F
:1056800044F8105C5EF80C5C44F80C5C5EF8085C56
:1056900044F8085C5EF8045C44F8045C0EF1100EFB
:1056A000E64504F11004E9D1013312F00C0F01EBCF
:1056B000031102F00F0400EB031327D0043C24F085
:1056C00003064FEA940C1E441C1F8E465EF8045BD2
:1056D00044F8045FB442F9D10CF1010402F0030272
:1056E00003EB840301EB840102F1FF3C4AB10CF1AE
:1056F000010C013B8C4411F8012B03F8012F61458B
:10570000F9D170BD02F1FF3C03469BE72246EBE76F
:10571000830730B548D0541E002A3FD0CAB2034692
:1057200001E0013C3AD303F8012B9D07F9D1032C8A
:105730002DD9CDB245EA05250F2C45EA054536D9C8
:10574000A4F1100222F00F0C03F1200EE6444FEA00
:10575000121C03F1100242E9045542E902551032CD
:105760007245F8D10CF1010214F00C0F03EB021298
:1057700004F00F0C13D0ACF1040323F00303043343
:10578000134442F8045B9342FBD10CF003042CB1A8
:10579000CAB21C4403F8012B9C42FBD130BD6446C5
:1057A0001346002CF4D1F9E703461446BFE71A4626
:1057B000A446E0E7F0B52DED028BB0EE408B85B04E
:1057C000154618EE902A0D9E0C9F002AB6BF2D227A
:1057D0000022B1EE408B662E0C461A7016D0462E73
:1057E00014D026F02003452B2FD0B0EE480B03AA8F
:1057F000019202AA00923B460A46022102F0F0FD05
:10580000672E2ED1EB072ED4039B17E003AB019339
:1058100002AB009322463B460321B0EE480B02F058
:10582000DFFD0378302B00EB040C30D03968B5EE87
:10583000408BF1EE10FA61441CD10B460E9A1B1AF4
:10584000136005B0BDEC028BF0BD03AA01340192D8
:1058500002AA00923B4622460221B0EE480B02F01B
:10586000BFFD472ECED0B5EE408BF1EE10FA00EB27
:105870000401E2D0039B9942E0D94FF0300C5A1C4E
:10588000039283F800C0039B8B42F8D3D6E7B5EEB2
:10589000408BF1EE10FAC9D0C4F101013960C6E7BE
:1058A000F0B5002983B002703FDB841C2B2309294B
:1058B000437030DD0DF107051F4FAC4687FB013209
:1058C000CB17C3EBA20303EB8302A1EB42020E460C
:1058D0003032632EE6460CF8012C19460CF1FF3CE1
:1058E000ECDC3031AEF10203C9B29D420CF8011C70
:1058F0001FD96346224601E013F8011B02F8011B81
:10590000AB42F9D10DF10903A3EB0E0EA644AEEBA9
:10591000000003B0F0BD3023A64619440EF8023B48
:105920006170AEEB000003B0F0BD4942841C2D2332
:10593000BDE7A646F5E700BF676666662DE9F04F4E
:105940008BB00C46DDF850A016461F460546FFF703
:105950006DFBD0F80080404600F066FF00230893FE
:10596000DAF800300490073323F0070393ED000BBF
:105970009FEDAA7BB0EEC06B0833B4EE476BF1EE3F
:1059800010FA226894F81890CAF8003084ED120BCF
:1059900000F38980B4EE400BF1EE10FA80F12F8213
:1059A00061684B1C2BD0B9F1670F64D0B9F1470F78
:1059B00061D042F4806200232260039308AB02931B
:1059C00007AB0093CDF804900DF11B032846FFF7B9
:1059D000F1FE8346B9F1650F079932D801394A467D
:1059E00004F150000791FFF75BFF089A1318012A92
:1059F0008246236140F37A810133236133E006213B
:105A0000616042F4806200232260039308AB02933A
:105A100007AB0093CDF804900DF11B032846FFF768
:105A2000C9FE09F0DF03472B8346D3D10799C81C71
:105A300080F2EC80A9F102095FFA89F9B9F1650FEA
:105A4000CCD9B9F1660F00F0F380089B8B4240F38C
:105A5000FA800029D4BFC1F102020122134423615C
:105A6000A1654FF0000A9DF81B30002B31D02D238B
:105A700084F843302DE0002900F0218142F4806257
:105A800000232260039308AB029307AB0093CDF889
:105A900004900DF11B032846FFF78CFE07998346FF
:105AA000C81CC7DBB2E0B5EEC00BF1EE10FA02D5B0
:105AB0002D2384F843305B4B5B4822F00402B9F19C
:105AC000470F94BF9B4683460323226023614FF018
:105AD000000A0097334609AA2146284600F0B0F98B
:105AE000013025D0236858052DD423695A46314604
:105AF0002846B84701301BD02368E06813F0020F36
:105B0000099B1AD0C21A002A17DD04F119094FF0B7
:105B1000000804E0E068099BC21A42450DDD01233C
:105B20004A4631462846B847013008F10108F1D10C
:105B30004FF0FF300BB0BDE8F08F9842B8BF184669
:105B40000BB0BDE8F08FB9F1650F30D994ED127B41
:105B5000B5EE407BF1EE10FA7DD1344A0123314697
:105B60002846B8470130E3D0DDE907239A4202DB3B
:105B70002368D907C1D5049B424631462846B84719
:105B80000130D5D0089B012BB6DD04F11A094FF086
:105B9000000803E0089B013B4345ADDD01234A4675
:105BA000314628469844B8470130F3D1C0E7089AF7
:105BB000012A40F3878001235A4631462846B847D8
:105BC0000130B5D0049B424631462846B8470130E3
:105BD000AED094ED127BB5EE407BF1EE10FA40F0C2
:105BE0008080089B012B78DD04F11A094FF0000832
:105BF00003E0089B013B43456FDD01234A463146E4
:105C000028469844B8470130F3D191E76368994238
:105C10003FF710AF4FF0670917E700BFFFFFFFFF27
:105C2000FFFFEF7F7448140878481408844814086C
:105C3000002960DD63682161002B00F08D80013355
:105C40000B4423610CE723682161DB077FF508AF74
:105C50004B1C236104E7079B002B54DD089BD4F801
:105C600058A05345A8BF5346002B994608DD5A4615
:105C700031462846B84701303FF45AAFD4F858A00F
:105C800029EAE9731946AAEB0303002B74DD04F13A
:105C90001A02CDF814B04FF00009A34692460C4604
:105CA00004E0DBF858301A1B4A4561DD01235246F7
:105CB000314628469944B8470130F2D138E70121EE
:105CC00061609EE6DB073FF576AF5A460123314619
:105CD0002846B84701303FF42BAF534604F1500239
:105CE00005E7089B0BF10102013BF0E72268D207B0
:105CF0007FF5B9AE80E66368002B32D12268D20707
:105D00002FD40123ABE64B4A012331462846B8473E
:105D100001303FF40DAFDDE90723134323D0049B8B
:105D2000424631462846B84701303FF401AF079B51
:105D3000002B7BDA04F11A094FF0000803E0079BFF
:105D40005B42434572DD01234A463146284698446A
:105D5000B8470130F3D1EBE62268D0077FF580AE7B
:105D60006DE702337BE62368DA077FF5C6AED6E738
:105D70005C46DDF814B09A46DDE907218A4202DB71
:105D80002368D80709D5049B424631462846B847C0
:105D900001303FF4CDAEDDE90721A1EB0A098A1AF3
:105DA0009145A8BF9146B9F1000F0BDD0BEB0A023C
:105DB0004B4631462846B84701303FF4B9AEDDE9DD
:105DC0000732D21A29EAE979A2EB0903002B7FF7FF
:105DD00093AE04F11A0A4FF0000807E0DDE907234B
:105DE0009B1AA3EB090343457FF786AE0123524676
:105DF000314628469844B8470130EFD198E610EE76
:105E0000903A002BB8BF2D2322F00402B8BF84F8CB
:105E100043302260084B094AB9F1470F94BF9346BB
:105E20009B46032323614FF0000A52E6089B5A4623
:105E30005DE600BF84481408804814087C481408B4
:105E40002DE9F84F92461F460A698B68DDF82890C5
:105E50009A42B8BF1A46CAF8002091F843300C465F
:105E6000064613B10132CAF80020226891065DD5BA
:105E7000DAF800300233CAF80030226812F0060F58
:105E800011461ED1E168CB1A002BD8BF114618DD90
:105E900004F1190B4FF0000805E0E568DAF800306E
:105EA000ED1A45450CDD01235A4639463046C847B0
:105EB000013008F10108F0D14FF0FF30BDE8F88F54
:105EC000216894F84330003B18BF01238A060AD5A5
:105ED000E1185A1C302081F84300224494F8451000
:105EE00082F84310023304F1430239463046C84772
:105EF0000130E1D0236803F00603042B1DD0A36812
:105F00002269934225DD4FF000089B1A98441A3409
:105F1000002501E045451CDA01232246394630467A
:105F2000C847013005F10105F4D1C5E712F0060FAD
:105F300012D0003B18BF0123D5E7DAF80030E16842
:105F40002269C91AA368934221EAE178DDDC0029BD
:105F5000DDDC0020BDE8F88FE168DAF80030CB1A0C
:105F6000002BD8BF114693DCABE700BF2DE9F0470B
:105F70000C4684B09046227E0C990746994604F15F
:105F80004300002A33D0A2F15803DDB2202D67D898
:105F9000202B65D8DFE813F0DE00640064006400A5
:105FA0006400640064006400640064006400A30092
:105FB0006E0064006400640064006E0064006400AD
:105FC0006400640021007F00C00064006400AE0033
:105FD00064007F0064006400E50023681A0640F155
:105FE00004810B6862691D1D0D601B681A60002327
:105FF00082462361CDF80090434603AA21463846E5
:10600000FFF71EFF013020D0236952464146384633
:10601000C847013019D02368E068039E9B0719D553
:10602000831B002B16DD04F1190A002504E0E0684B
:10603000039E831BAB420DDD012352464146384689
:10604000C847013005F10105F1D14FF0FF3004B030
:10605000BDE8F087B042B8BF304604B0BDE8F08775
:10606000012384F84220236104F1420A002384F8CA
:106070004330BFE723681A0602D45E0600F1C180F0
:106080000D682A6804350D601546002A6BDBDFF8C1
:1060900084C10A2610E023681D0640F19C800B682D
:1060A0001D1D0D601D68DFF86CC16F2A0CBF08262E
:1060B0000A26002384F843306268A260002A7FDB4E
:1060C000236823F004032360002D5BD1002A79D1DB
:1060D0008246082E65D0A0EB0A0020618AE70B6893
:1060E0000122186804330B6004F1420A84F842006C
:1060F0002261BBE70B686268181D0860D3F800A036
:1061000000215046FEF79AFF002800F08180A0EBA6
:106110000A0060602061A9E7236843F02003236040
:106120007822DFF8F4C084F845200A68151D0D6058
:106130001D0643D4590641D51588DE0744BF43F0F8
:1061400020032360002D44D1236823F02003236023
:106150001026AEE7582384F84530DFF8B8C023682E
:10616000E3E72368DCE76268A2602D21002AC5F11D
:10617000000584F8431002DB23F004032360DFF8FA
:1061800094C00A268246B5FBF6F306FB13512A4655
:106190001CF801100AF8011DB2421D46F3D2082E68
:1061A00099D12368D90796D5626823699A4292DC0F
:1061B00030230AF8013C0AF1FF3A8CE71568BCE786
:1061C000002DDFD19CF8003084F8423004F1420AFF
:1061D0007FE710266DE713F0400F0B6803F104050D
:1061E0000D600CBF1D681D885DE713F0400F0B6844
:1061F000626903F104050D601B6814BF1A801A6000
:10620000F5E60A68B2F9005004320A602A463CE713
:1062100060687FE7884814089C48140838B5124B1A
:106220001D68AA6B04461AB10023C2E9044338BDB5
:106230001820EFF0B5FD0246A86378B101200021D7
:10624000C2E90401094B0A480A499160C2E9000306
:106250000B2393810023C2E9044338BD064B074852
:10626000422102F003F800BF0422003034126DE630
:106270000E33CDABECDE0500B0481408C848140856
:106280001C4B10B51C68A26B8AB113691A4954697A
:106290001A4803FB01F100FB0411A3FB003001339A
:1062A00041EB0001C2E9043121F0004010BD18208B
:1062B000EFF076FD0246A06388B1114C114B0E48F9
:1062C000114991609FED097BC2E900430B23938143
:1062D0000E4B014682ED047BC2E9043110BD0C4B2C
:1062E0000C484E2101F0C2FFAFF300800100000016
:1062F00000000000042200302DF451582D7F954CF1
:106300000E33CDAB34126DE6ECDE05002E7F954CDE
:10631000B0481408C8481408EC46A0E8F05F4FF0F5
:1063200000007047B0E8F05FE546080008BF0120B4
:10633000704700BF10B5114C86461EF801CB14F80B
:106340000C3003F00303012B11F8013B624608BF38
:106350000CF1200214F803C00CF0030CBCF1010F87
:10636000184604D0D21A06D1002BE6D110BD203336
:10637000D01AE2D010BD104610BD00BFF192110836
:10638000830710B5044610D10268A2F1013323EA55
:10639000020313F0803F08D150F8042FA2F101331B
:1063A00023EA020313F0803FF6D003781BB110F804
:1063B000013F002BFBD100F0D9F9204610BD00BFF2
:1063C00011F0FF01034644D0820732D110B50468B2
:1063D00041EA012E4EEA0E4E8EEA0402A2F101338A
:1063E00023EA0203A4F1013222EA0402134313F068
:1063F000803F0FD150F8044F84EA0E0CA4F1013312
:10640000ACF1013223EA040322EA0C02134313F035
:10641000803FEFD0037823B936E010F8013F002B1E
:1064200032D09942F9D110BD8A4211D09A0718464C
:10643000CCD0184613F8012B002AF5D1104670472E
:106440009907184607D0184601330278002AF7D179
:1064500070478207F7D10268A2F1013323EA0203F1
:1064600013F0803F08D150F8042FA2F1013323EA42
:10647000020313F0803FF6D00378002BE8D010F829
:10648000013F002BFBD17047184610BDA2EB030063
:10649000704700BF02780B78012A28BF9A42F5D1D5
:1064A0006DE9044540EA0104CDE902676FF0000C94
:1064B0004FEA447212B380EA010414F0070F6AD164
:1064C00000F0070420F0070004F0030521F00701A5
:1064D0004FEAC505F0E8042314F0040FF1E804675F
:1064E0000CFA05F462EA040266EA04060AD063EADA
:1064F0000403624667EA0407664603E0F0E8042303
:10650000F1E8046782FA4CF582EA0604A4FA8CF4F6
:106510006CBB83FA4CF583EA0705A5FA8CF595B9AF
:1065200050E9022351E9026782FA4CF582EA060437
:10653000A4FA8CF483FA4CF583EA0705A5FA8CF5E6
:106540002543DBD09CB92DBAB5FA85F424F00704B5
:1065500027FA04F1DDE9026723FA04F303F0FF00F0
:1065600001F0FF01FDE80445A0EB0100704724BAEB
:10657000B4FA84F424F0070426FA04F1DDE9026792
:1065800022FA04F202F0FF0001F0FF01FDE80445E9
:10659000A0EB0100704714F0030F3CD110F003048E
:1065A00028D150F8082B51F8083B82FA4CF582EAC2
:1065B0000305A5FA8CF55DB950F8042C51F8043C9C
:1065C00082FA4CF582EA0305A5FA8CF5002DE8D095
:1065D0002DBAB5FA85F424F0070423FA04F122FA5F
:1065E00004F202F0FF0001F0FF01FDE80445A0EB1A
:1065F000010070474FEAC40420F0030050F8082B54
:1066000021F0030151F8083B0CFA04F462EA040299
:1066100063EA0403C9E710F003041AD0A1EB0401F4
:1066200020F00300E40750F8042B06D00FD28B783B
:106630005FFAA2F4E41A06D12BB1CB785FFAB2F478
:10664000E41A00D11BB920465DF8104B704701F1E8
:10665000040150F8042BCC0721F0030151F8043B4E
:1066600048D824D222F07F4482FA4CF594EA1325CC
:10667000A5FA8CF50AD165B951F8043B84EA020405
:10668000B4EB036F0ED150F8042BEBE74FEA132362
:1066900055E035F07F454DD10878FDE80445C0F15F
:1066A000000070474FEA126203F0FF0347E002EA7E
:1066B0001C4482FA4CF594EA1345A5FA8CF50AD1EC
:1066C00065B951F8043B84EA0204B4EB034F0CD1E2
:1066D00050F8042BEBE74FEA134330E015EA1C4572
:1066E00028D10B884FEA124229E04FEA124203EA0E
:1066F0001C4324E002F0FF0482FA4CF594EA13658F
:10670000A5FA8CF50AD165B951F8043B84EA020474
:10671000B4EB032F09D150F8042BEBE74FEA1363D6
:106720000DE015F0FF0F05D10B684FEA122223F0A0
:106730007F4304E04FF00000FDE80445704712BAC3
:106740001BBA82FA4CF482EA0304A4FA8CF5B5FA77
:1067500085F402FA04F203FA04F34FEA1260FDE84A
:106760000445A0EB13607047FFF794BE80EA010276
:10677000844612F0030F4FD111F0030F32D14DF8C0
:10678000044D11F0040F51F8043B0BD0A3F101327A
:106790009A4312F0803F04BF4CF8043B51F8043B8D
:1067A00016D100BF51F8044BA3F101329A4312F005
:1067B000803FA4F101320BD14CF8043BA24312F00C
:1067C000803F04BF51F8043B4CF8044BEAD0234609
:1067D0000CF8013B13F0FF0F4FEA3323F8D15DF8BB
:1067E000044B704711F0010F06D011F8012B0CF883
:1067F000012B002A08BF704711F0020FBFD031F8FB
:10680000022B12F0FF0F16BF2CF8022B8CF8002081
:1068100012F47F4FB3D1704711F8012B0CF8012B04
:10682000002AF9D1704700BF90F800F06DE90245E9
:1068300020F007016FF0000C10F0070491F820F031
:1068400040F049804FF000046FF00700D1E90023C9
:1068500091F840F000F1080082FA4CF2A4FA8CF2B0
:1068600083FA4CF3A2FA8CF34BBBD1E9022382FAF0
:106870004CF200F10800A4FA8CF283FA4CF3A2FA6D
:106880008CF3E3B9D1E9042382FA4CF200F1080059
:10689000A4FA8CF283FA4CF3A2FA8CF37BB9D1E917
:1068A000062301F1200182FA4CF200F10800A4FA5B
:1068B0008CF283FA4CF3A2FA8CF3002BC6D0002A98
:1068C00004BF04301A4612BAB2FA82F2FDE8024559
:1068D00000EBD2007047D1E9002304F00305C4F1B6
:1068E00000004FEAC50514F0040F91F840F00CFACF
:1068F00005F562EA05021CBF63EA050362464FF034
:106900000004A9E72AB330B5134C8646851804E085
:10691000D21A1CD1C3B1AE4517D01EF8010B235CAF
:1069200003F00303012B11F8013B14F803C00CF032
:10693000030C024608BF00F12002BCF1010F18460B
:10694000E6D12033D01AE6D030BD002030BD10464D
:1069500030BD1046704700BFF1921108A2B330B5A8
:1069600040EA0104A40784460B462AD09CF80000A4
:106970000C7884422FD1012A0DD0E64660B11EF872
:10698000010F11F8014F6FEA0E03A042134422D108
:106990001CEB0303F2D1002030BD0468194653F804
:1069A000045BA4F1013EAC4284462EEA040E00F1E1
:1069B00004000BD1043A84461946ECD01EF0803F07
:1069C000E9D1032AE9D8D1E7104670479CF80000C6
:1069D0000C78A042D1D0001B30BD00BF30B540EADA
:1069E0000104A30701D1032A0FD8844601F1FF3E19
:1069F00007E01EF8011F03F8011B541EC1B19C469D
:106A000022466346002AF4D130BD0B46844619461F
:106A100053F8045BA5F1013424EA050414F0803F27
:106A2000E4D1043A032A4CF8045B1946EFD8DDE7B9
:106A30006244002CE8D003F8011B9342FBD130BD27
:106A400010B4044C03460A4620685DF8044B19460E
:106A500000F002B80422003070B50D461446012142
:106A600062B12B4605EB020C01E0634512D01A46D9
:106A700001331478002CF8D1541B611CEFF088FA14
:106A8000064628B122462946FEF75AFB0023335515
:106A9000304670BD5C1B611CF0E700BF71B103465E
:106AA00000EB010C01E0634506D01A460133117872
:106AB0000029F8D1101A7047181A70470846704715
:106AC00030B40478A4B10D780A462B461DB90AE00B
:106AD00012F8013F3BB19C42FAD11378002B08BF5A
:106AE000002030BC704710F8014F002CECD1F4E7C7
:106AF000204630BC704700BF71B138B503460C4624
:106B0000002501E0431C054621461846FFF758FCC6
:106B10000028F7D1284638BDFFF752BC30B40478BE
:106B200094B10D7884465DB10A462B4602E012F816
:106B3000013F2BB1A342FAD11CF8014F002CF2D136
:106B4000ACEB000030BC70472046FBE72DE9F04F6E
:106B5000012BADF21C4D1D4681460F46904640F27A
:106B600045810123002419464FF0FF309C4606E082
:106B7000A3EB000C1C46012163189D4210D908EBC1
:106B8000000218F80360525C9642F1D300F0828054
:106B90004FF0010C20466146644463189D42EED8D4
:106BA000CDF808C04FF0010C002461464FF0FF36CD
:106BB000634606E0A3EB060C1C46012163189D42C8
:106BC0000FD908EB010218F803E0925D9645F1D861
:106BD00066D04FF0010C26466146644463189D421E
:106BE000EFD8013600F1010BB34502D8CDF808C04B
:106BF000B34605AB0DF2144243F8045F9342FBD158
:106C0000002D00F0F8806C1E06AE08F1FF3208EB94
:106C10000400019612F8011FD3432B4443449042D1
:106C200046F82130F6D1029B5A4608EB0301404654
:106C3000FEF754FA002840F08280029B0BF1FF32ED
:106C4000EB1A824606460592039309EB060E019A5B
:106C50001EF8043052F8233043B3BAF1000F04D0C9
:106C6000029A9342039A38BF13461E444FF0000A1B
:106C70007B1BB342E9D209EB070045F40061FFF743
:106C80000DFF07447B1BB342DFD200200DF21C4DE9
:106C9000BDE8F08F8C4512BF0131644401216BE7E0
:106CA00061450ABF64180131012187E7D3455B467E
:106CB00038BF5346A34211D2591E9A1941444A443F
:106CC00002E00133A34209D212F8010B11F801CFFF
:106CD0008445F6D0CBF101021644C6E7D345059BA7
:106CE00040F282800BEB06024A4408EB0B01CDF820
:106CF00010B002E0534516D0034612F8010D11F80A
:106D000001CD844503F1010B03F1FF30F2D05B4666
:106D1000DDF810B00AF1010A9A450BD8029BDDF8A4
:106D20000CA01E44A4E753460AF1010A9A45DDF877
:106D300010B0F3D970460DF21C4DBDE8F08FA5EBF5
:106D40000B035B4538BF5B46013304930BF1FF3304
:106D50000293CBF101030026039345F4006A09EB8B
:106D60000601019A0B5D52F823306BB11E447B1B68
:106D70009E42F4D909EB07005146FFF78FFE074406
:106D80007B1B9E42EBD980E7A34514D2029B0BEB01
:106D9000060208EB030C4A445B4602E00133A342BF
:106DA00009D212F8010B1CF801EF8645F6D0039AC0
:106DB00016441E44DBE7BBF1000F10D00BEB0600BE
:106DC000484408EB0B0201E0434508D012F801EDFE
:106DD00010F801CDE6451346F6D0049BC6E70846F9
:106DE0000DF21C4DBDE8F08F5B4693E70123029343
:106DF0004FF0000BFDE606AB4FF0FF34019312E7B6
:106E00002DE9F0410D46097890B00446002953D091
:106E10006A78002A00F08380AB78002B50D0E878A5
:106E2000002800F083802B79002B57D02846FFF7ED
:106E3000FBFC064640F400712046FFF72FFE864219
:106E40005CD8FE2E00F28780801B27184022711C20
:106E50006846FEF75DFC7EB16A1E5FFA86FC9019FB
:106E600012F8013F03F03F0340336B44A91A614419
:106E7000824203F8401CF3D1013CA35D03F03F03C1
:106E800040336B4413F8400C0444A74203D23AE069
:106E90004444A74237D314F806C00CF03F0C0CF161
:106EA00040030DEB030C2046324629461CF8408C6B
:106EB000FEF714F90028EBD1204610B0BDE8F081B0
:106EC000007842EA014200E00C4640EA0343611CBC
:106ED000A0B19A426078F7D1013CEDE722786AB11F
:106EE000296809BA01E099421ED042EA03232046EC
:106EF00014F8012F002AF6D1994215D0002420461B
:106F000010B0BDE8F081BB5DB819002BF6D04FF48E
:106F10000061FFF7C3FD0744BC42ADD9EEE710B0F6
:106F2000BDE8F041FFF74CBAC41EC5E7120442EABF
:106F3000016242EA03232178024600E02C4641EA3E
:106F40000200651C02020029D8D0B3EB002F617843
:106F5000F4D1023CB0E7014633462A46204610B041
:106F6000BDE8F041F2E500BF2DE9F04F1C462DEDE4
:106F7000108BAB4BD3F800B097B000258046584635
:106F80008A46079212950026FFF74EFC0025CDE9B0
:106F900004560246CDF844A051460F4611F8013B75
:106FA0002D2B2FD8DFE813F0A0002E002E002E008E
:106FB0002E002E002E002E002E00AE00AE00AE00E1
:106FC000AE00AE002E002E002E002E002E002E0051
:106FD0002E002E002E002E002E002E002E002E0041
:106FE0002E002E002E002E00AE002E002E002E00B1
:106FF0002E002E002E002E002E002E002E00CB0381
:107000002E00C10300210991302B7DD00021089171
:107010002F2B1C4640F2E8844FF0000938464E46BC
:107020004D4612E00130082D1190C8BF09EB8909C7
:107030000478CABF03EB4909A1F13006A9F1300970
:107040002F2C05F1010523466FDD06EB8601392C57
:1070500003EB4101E6DD59460A92FFF77FFC002869
:1070600035D1119B0A9A1946134411938C5C002D5B
:1070700040F04185302C40F0FC84C3F101029818A7
:10708000013311931C78302CF9D0A4F13103082B73
:1070900000F20B83A4F1300B119C431C0B930125D0
:1070A00027464FF0000C06EB86060BEB4606002049
:1070B000631C11936478A4F13001092900F2C7829E
:1070C00001308B46002940F06B84119CF0E70020D2
:1070D000652CAC460B90864601D0452C32D1002D54
:1070E0006ED1089B03436AD1079B9FED4B8B13B175
:1070F000079BC3F800A0B0EE480B17B0BDEC108B97
:10710000BDE8F08F119148E77B7803F0DF03582B3F
:1071100000F02A84013711973B78302BFAD0002BEE
:1071200000F0C4800121089172E759460A92FFF7E6
:1071300015FC0A9A002800F0CC80AC4600230B9383
:1071400018469E464FF0000B002D00F08B8007EE96
:10715000906A0B9BB8EE677BABEB0303BCF1000FAF
:1071600008BFAC46102D0A932B46A8BF1023092D4B
:107170008DED047B0CDD2B4A02EBC30212ED125B9A
:1071800006EE909AB8EE666BA7EE056B8DED046B7C
:107190000F2D00F3A5800A9A002A00F0DC830A9ADA
:1071A00040F34883162A40F39B840A99C5F12502CF
:1071B0008A4280F2A9840A9AEB1A134496E00025C9
:1071C000DDF844A00AF1010311939AF801402B2C39
:1071D00000F068822D2C00F01F8200230A93A4F196
:1071E0003003092B00F21382302C05D1119B01339F
:1071F00011931C78302CFAD0A4F13103082BA1D8BC
:10720000119A0C92531C1193A4F1300B54782F2C2B
:1072100011DCF8E3AFF30080000000000000000084
:107220004895110864951108013311934C782F2C5F
:10723000A2F1300B06DD0BEB8B02392C194604EB67
:107240004202F1DD0C9A9B1A082B40F3DC8344F6D2
:107250001F6B0A9B002B3FF477AFCBF1000B002D87
:107260007FF475AF089B034320D1BEF1000F7FF47C
:107270003BAF692C00F0DE8300F3F382492C00F071
:10728000D9834E2C7FF430AFC34911A802F09CFA89
:1072900000283FF429AF119B1B78282B00F0EA84CB
:1072A000BE48FDF761FAB0EE408B01E09FEDB08B78
:1072B000079A0AB1119B1360099B002B3FF41BAF87
:1072C000B1EE488BB0EE480B17B0BDEC108BBDE8AB
:1072D000F08F119B0B90991811919C5CAC46EAE6DB
:1072E0000A9AEB1A1344002B40F3D48213F00F01D7
:1072F0000AD0AB4A02EBC1029DED046B92ED007B1C
:1073000027EE067B8DED047B33F00F0240F04682C2
:107310000023089300962B4662463946404602F009
:107320001BFC002800F01A830B9BA3EB0B0B0A9BA2
:107330009FED91EB002B9FED92CB9FED93DB9FEDAB
:1073400094BBB4BF5A4600224FF0000A23EAE3730D
:107350000B920C9354468346DBF80410404602F02F
:1073600045FB0646002800F03381DBF810209DED38
:10737000048B023292000BF10C010C30FDF7E0FEA1
:10738000B0EE480B14AA13A9404602F08FFF1290EA
:10739000002800F0E8800121404602F087FC044606
:1073A000002800F01581139A002AC0F203810B9B7C
:1073B000DDF83090D718089B149DD21A2A44794BD7
:1073C000013A9A42C5F1360580F29980991A1F292F
:1073D000A5EB010500F30E81012202FA01F30D93E2
:1073E00000230E93A944089B3D44AF423A4699447A
:1073F000A8BF2A464A45A8BF4A46002A03DDAD1A5F
:10740000A9EB0209BF1A0B9B002B00F38A80002D09
:1074100000F3A0800A9B002B00F3D180B9F1000F8C
:1074200000F3DE80002F08DD21463A46404602F098
:1074300071FD0446002800F0CB8012993246404688
:1074400002F0FEFD8246002800F0C2800023C568DD
:10745000C360214602F0D2FD0028C0F2C48300F0D0
:107460007B832146504602F089FFB0EE007BB4EEEC
:10747000C70BF1EE10FA47D8002D00F0D880B7EE18
:10748000009B0598484B00224849DFF824C100EAD8
:107490000109E14500F0E180089961B1B9F1D46FCB
:1074A00009D8B4EECB9BF1EE10FA40F2648103F1FF
:1074B000D661A1EB0903B0EE480B43EC1A2B02F0A6
:1074C00065FEAAEE008B8DED048B18EE903A089ABB
:1074D00022B9364A1A40914500F0F0801299404690
:1074E00002F0C4FA3146404602F0C0FA2146404656
:1074F00002F0BCFA5146404602F0B8FA2CE70123EC
:107500000021CDE90D316DE7B6EE009B20EE099B21
:10751000002D40F08980B1EE497B059853EC172B84
:10752000B2E721461A46404602F084FC0446002891
:107530004ED00146129A404602F0CEFB002847D0BA
:107540000F901299404602F091FA0F9A1292002D74
:107550007FF760AF12992A46404602F0DBFC12909A
:1075600000287FF457AF5F4634E000BFAFF30080E0
:1075700000000000000000009535A094FFFFCF3F01
:107580009535A094FFFFDF3F35E5AF350000E03FC4
:107590000000C0FFFFFFDF41084914081849140824
:1075A0006495110802FCFFFF0000F03F0000F07F2F
:1075B0000000E07F0C9B0B9FA3EB0209FBE631462A
:1075C0000C9A404602F036FC064600287FF426AFAF
:1075D0005F46129822239FEDA68BC8F800308FE0FB
:1075E00031464A46404602F095FC064600287FF4A4
:1075F00019AFEDE7C2F17F4202F57F0202F57B424F
:107600000121E23201FA02F3CDE90D13EAE6CDF8E9
:1076100044A04FF0000B97E501230A930AF10203FF
:1076200011939AF80240DAE5B0EE497B75E7DDE99F
:107630000412002900F08680DDE90412012900F01F
:10764000E88110468C4BB7EE009B00221CE7652CAE
:107650004FF0010E3FF4B4AD3FE543EC1A2BA0F11F
:10766000547305939DED04FBB0EE4F0B02F08EFDBD
:107670008249AAEE00FB1FEE903A814A19409142DE
:107680008DED04FB73D97F4B18EE902A9A4203D1FB
:1076900018EE103A01339BD07A4A4FF0FF33CDE910
:1076A00004321BE700230A93B8E7652C00F0D28070
:1076B000452C00F0CF804FF0010ED3E551EC190BB3
:1076C0000D93F9F7CFF9F9F707F8049B1D430D9BCC
:1076D00041EC170BC3F313032B4339EE479B00F028
:1076E000A280B4EECC9BF1EE10FA05D4B4EECD9BA3
:1076F000F1EE10FA7FF7F2AE9DED048B12985F4623
:107700000146404602F0B2F93146404602F0AEF979
:107710002146404602F0AAF93946404602F0A6F951
:107720005146404602F0A2F9C2E501230993791CB3
:1077300011917B78002B3FF4D7AC0F4664E4002313
:107740000993F4E7C2F313031046002B7FF47AAFDA
:10775000B7EE007BB4EEC70BF1EE10FA00F1CF816B
:10776000B6EE009B20EE099BB1EE497BD6E603F115
:1077700054730593ABE6BCEEC99B19EE103A012B8E
:1077800038BF012309EE103AB8EE499B002D40F0B6
:107790004E81B1EE497B53EC172B88E6B2F59A7F08
:1077A00000F3DC80102A4FEA221340F37782364C34
:1077B0009DED047B00202246014613F0010F01F1EC
:1077C00001014FEA630304D092ED006B012027EE24
:1077D000067B012B02F10802EFD108B18DED047B8D
:1077E000059BA3F15473059304EBC10191ED007B5C
:1077F0009DED046B214B27EE067B17EE902A234963
:1078000013408B428DED047B00F2A880A1F580111E
:107810008B4240F2E1811B4C4FF0FF33CDE9043441
:107820000023089376E5B4EECE9BF1EE10FA7FF5D7
:1078300055AE61E71632FFF653AD0B9BA3EB0B0B76
:10784000134B03EBCB0393ED007B9DED046B86EEB6
:10785000078B2DE54FF0000CCDF82CC04FF0010E3A
:107860003FE46E2C3FF410AD3EE400BFAFF3008068
:10787000000000000000F07F0000F0BF0000F07F7B
:10788000FFFF9F7CFFFFEF7F549611080000A07C54
:10789000649511083FF43CAD5B4213F00F010AD030
:1078A000A74A02EBC1029DED046B92ED007B86EED0
:1078B000077B8DED047B1B113FF42AAD1F2B33DCBE
:1078C00013F0100218BF6A229DED047B08929D4AB6
:1078D0000021D80704D592ED006B012127EE067B2D
:1078E0005B1002F10802F4D109B18DED047B089B15
:1078F00093B1DDE90401C1F30A52C2F16B03002B1D
:107900000ADD1F2B40F3EB810020342B049040F361
:1079100019824FF05C7305939DED047BB5EE407BBF
:10792000F1EE10FA7FF4F6AC22239FED818BC8F8BC
:107930000030BDE4149B0493139B03F23342159B68
:1079400023F4801343EA02530593250742BF059BA6
:1079500043F0004305939DED048BA9E422239FEDA2
:10796000768BC8F80030A3E4099B019312AB029414
:107970000093754A13AB11A9404601F039FC10F091
:10798000070504463FF492AC062D75D1079B9FED89
:10799000688B0137002B3FF4AEAB1F60FFF7ABBB2A
:1079A0000B9B119C03440B93012805F101031A461C
:1079B00015D0284400F1FF3E03E046009E450DD05F
:1079C00001332A46082A1D4606EB8600F5D9102BFE
:1079D000DCBF09EB89094FEA4909EFE70232082DBC
:1079E0003DDC1546FFF75FBB594638460A92FEF765
:1079F000B5FF0A9A00286AD04FF0000CE1466646AF
:107A00006546FFF79BBB44F61F639B45A8BF9B469B
:107A10001FE4DDE904231846002B7FF413AE5F4614
:107A200022239FED438B1298C8F8003068E6B0EE31
:107A3000497BB0E6454911A801F0C6FE00283FF495
:107A400053AB119B4249013B11A8119301F0BCFEBD
:107A500010B9119B013311939FED378B28E4102A45
:107A6000DCBF09EB890901EB490915460020FFF746
:107A70001FBB0020FFF709BB129A3AB1352114A8A9
:107A800002F0C2FC1299404601F0F0FF013D042DC6
:107A90003FF65BAF01A353F825F000BF357902082C
:107AA000C57A0208BF7A0208B17A0208357902085D
:107AB0004FF0FF336FF00046CDE9043645E7254B24
:107AC000059342E7149B0493159B05933DE7119B97
:107AD0001946134411938C5C06468146FFF7CABAD7
:107AE000174B03EBC20393ED008B9DED047B28EE57
:107AF000078BFFF7DDBBAC460B90FFF7DCBABEEEA1
:107B0000007BB6EE009B09E50D4BC5F10F054A1B46
:107B100003EBC50503EBC20395ED008B93ED007BF2
:107B20009DED046B28EE068B28EE078BFFF7C0BB9C
:107B30000000000000000000000000000000F07FD6
:107B40006495110820941108F8931108FC48140852
:107B5000004914080000F07F5F46002D7BD0DDE96E
:107B600004BC874BCCF313019942624600F0BF80FE
:107B70000E9B002B77D0DDE90412134291461AD0F8
:107B8000B0EE480B002D00F08C8002F0FFFA089B4D
:107B90007BB1C9F30A53C3F16B03002B09DD1B054D
:107BA00003F17F51002001F5401141EC170B20EE4D
:107BB000070B38EE008B089B63B19FED6F7B28EEBF
:107BC000078B18EE103A18EE902A134304BF2223B5
:107BD000C8F80030129893E502F15473059300231E
:107BE0000893FFF797BBDDE904120B462B435F4672
:107BF000E1D1C2F313039146002BDCD122F0004304
:107C00001B0D1B05B3F1D66FD5D9DAF814301BB9AB
:107C1000DAF81030012BCEDD51460122404602F049
:107C200079F92146824602F0E9F90028C3DD089B74
:107C3000002B40F09180534B09EA0303A3F5801316
:107C40006FEA13536FEA035305934FF0FF33049326
:107C50009DED048BAFE7DDE90412C2F313030B4380
:107C6000914685D1E3E7DDE904010D9B0342A2D0F3
:107C7000894685E7444911A814AA01F0C1FD0528E9
:107C80007FF40EAB159B43F0FF4343F4E0030593F1
:107C9000149B04939DED048BFFF70ABB3B4C002122
:107CA0009EE502F073FA089B002B42D0C9F30A53F9
:107CB000C3F16B03002B09DD1B0503F17F5101F5B7
:107CC0004011284641EC170B20EE070B38EE408B95
:107CD000B5EE408BF1EE10FA7FF46FAFA0E64FF0F7
:107CE000FF3202FA03F3049A1A40049214E6089B46
:107CF0000499DBB1234B1340B3F1D46F16D81B0D9D
:107D0000C3F16B034FF0FF3000FA03F399427FF4A5
:107D10002FAF1F4B9A422BD01A4B134003F5801301
:107D20000593002304939DED048B44E74FF0FF334C
:107D3000ECE738EE408BB5EE408BF1EE10FA7FF4B5
:107D400049AF6DE64FF0FF33C2F14B0203FA02F286
:107D500002EA01030593DFE50A4B09EA0303B3F1E5
:107D6000D66F3FF76BAFB3F15C7F3FF726AF57E6B7
:107D70000131D1D12DE400BF0000000000005039D6
:107D8000FFFF0F000000F07F0C94110854961108BB
:107D9000FFFFEF7F014BFFF7E7B800BF7022003015
:107DA00010B4054C8446134620685DF8044B0A461F
:107DB0006146FFF7D9B800BF0422003010B4054C6B
:107DC000054B84460A4620685DF8044B6146FFF780
:107DD000CBB800BF042200307022003010B51C4C1C
:107DE0008446134620680A466146FFF7BDF8B4EEA4
:107DF000400BF1EE10FA19D6F7EEC06BDFED157AF5
:107E0000B0EEE67AB4EE677AF1EE10FA0BDDB0EE82
:107E1000C00B9FED0D5BB4EE450BF1EE10FA02DCEA
:107E2000236822221A60B0EE660A10BD10EE903A66
:107E3000002B094804DAF9F721FDF1EE406AF2E778
:107E4000BDE81040F9F71ABDFFFFFFFFFFFFEF7F0E
:107E500004220030FFFF7F7F1849140810B51C4C26
:107E60001C4B84460A4620686146FFF77DF8B4EE55
:107E7000400BF1EE10FA19D6F7EEC06BDFED167A73
:107E8000B0EEE67AB4EE677AF1EE10FA0BDDB0EE02
:107E9000C00B9FED0D5BB4EE450BF1EE10FA02DC6A
:107EA000236822221A60B0EE660A10BD10EE903AE6
:107EB000002B0A4804DAF9F7E1FCF1EE406AF2E738
:107EC000BDE81040F9F7DABCFFFFFFFFFFFFEF7FCF
:107ED0000422003070220030FFFF7F7F1849140811
:107EE000F0B4074610B33E468C4616F8010B01E08D
:107EF000A04216D01CF8014B002CF9D1D8B116F8CD
:107F0000015B0C4601E0002BF9D014F8013B9D42C7
:107F1000F9D14DB1002306F8013C16603846F0BC9B
:107F200070475BB13746DEE72E46F6E71768002F4D
:107F3000D9D13846F3E7F0BC106070471660384678
:107F40003B70ECE70123FFF7CBBF00BF2DE9F04FFB
:107F5000814645488E4675461EF801CB10F80C4008
:107F600014F00804F7D1BCF12D0FE34654D0BCF156
:107F70002B0F08BF9EF800B06FF0004808BF05F156
:107F8000020E1BB1102B4FD01F4604E0BBF1300F87
:107F900055D00A231F460025B8FBF7F6284607FBF5
:107FA000168A07E0864215D329D007FB00C00125B9
:107FB0001EF801BBABF1300CBCF1090F06D9ABF1D7
:107FC000410CBCF1190F08D8ABF1370C63450DDD3E
:107FD000002DE7DA4FF0FF35EAE7ABF1610CBCF1B9
:107FE000190F03D8ABF1570C6345F1DC002D0BDB07
:107FF00004B140420AB195BB1160BDE8F08FE24583
:10800000D3DA4FF0FF35D3E72223C9F800301AB393
:108010000EF1FF314046EFE79EF800B04FF0004808
:1080200005F1020E0124ACE7BBF1300FACD19EF894
:10803000000000F0DF00582807D01F46ABE79EF88D
:10804000003003F0DF03582B0BD110279EF801B04E
:108050003B460EF1020E9EE74046BDE8F08F80469B
:10806000D6E708231F4696E7F1921108012B02D0AC
:10807000242B00D86AE710B5FCF77CFE16230360BA
:10808000002010BD012A08D0242A06D884460648BC
:10809000134600680A46614658E710B5FCF76AFEC9
:1080A00016230360002010BD04220030012A08D0EE
:1080B000242A06D884460648134600680A466146C4
:1080C00044E710B5FCF756FE16230360002010BDF0
:1080D000042200302DE9F04707464B480E4635464E
:1080E00016F801CB10F80C4014F00804F7D1BCF1DD
:1080F0002D0FE64658D0BCF12B0F04BF96F800E0D8
:10810000AE1C5BB1102B54D04FF0FF38B8FBF3F826
:1081100003FB08FA6FEA0A0A994608E0BEF1300F3D
:108120005AD00A23DFF8E4804FF0050A994600256B
:10813000284607E0404515D829D009FB00C0012595
:1081400016F801EBAEF1300CBCF1090F06D9AEF117
:10815000410CBCF1190F08D8AEF1370C63450DDDA9
:10816000002DE7DA4FF0FF35EAE7AEF1610CBCF124
:10817000190F03D8AEF1570C6345F1DC002D0BDB72
:1081800004B140420AB16DB91160BDE8F087D44531
:10819000D3DD4FF0FF35D3E722233B604FF0FF30B4
:1081A000002AF2D0711EEFE796F800E00124AE1C21
:1081B000A7E7BEF1300F21D1307800F0DF0058285A
:1081C00016D14FF0100996F801E04FF00F0A023671
:1081D0006FF070484B46AAE7337803F0DF03582B63
:1081E000EFD008234FF0070A6FF0604899469EE7EA
:1081F00099466FF070484FF00F0A98E74FF00F0A5A
:108200006FF07048994692E7F1921108999999197F
:1082100060E700BF10B4044C8446134620685DF844
:10822000044B0A46614655E70422003010B4044C62
:108230008446134620685DF8044B0A46614649E7C8
:1082400004220030034BC35C03F00303012B08BF7F
:1082500020307047F1921108034BC35C03F0030315
:10826000022B08BF20387047F192110800B50B4C63
:1082700025681446EE681A4685B003460D464CB193
:1082800007490095CDE901143046064900F04AFF40
:1082900002F0ACFB04490C46F3E700BF04220030B7
:1082A0000C4914081C4914081849140808B5134649
:1082B0000022FFF7DBFF00BF2DE9F04F03690C69D7
:1082C000A34283B0C0F28780013C01F11405A300F2
:1082D00000F11408009355F8243058F82420013395
:1082E00081469A4208EB840005EB84070190B2FBBB
:1082F000F3F63BD30023AE4640469B465EF804AB04
:1083000002681FFA8AFC06FB0C334FEA134C4FEA53
:108310001A4A06FB0ACA1FFA83FCABEB0C0C1FFAC5
:108320008AF31CFA82FCC3EB124202EB2C421FFAC6
:108330008CFC4CEA0243774540F8043B4FEA224B61
:108340004FEA1A43DAD2009B58F8033073B9019B05
:10835000043B984504D307E0984504F1FF3403D269
:1083600053F80429002AF7D0C9F81040484601F014
:1083700045FE00282BDB01364046002355F8041B40
:10838000D0F800C08AB29A1A0B0C12FA8CF2C3EB26
:108390001C4303EB224392B242EA0342AF4240F84D
:1083A000042B4FEA2343E9D258F8242008EB840336
:1083B0006AB9043B984504D307E0984504F1FF34BB
:1083C00003D253F80429002AF7D0C9F810403046E8
:1083D00003B0BDE8F08F002003B0BDE8F08F00BF10
:1083E0002DE9F04F2DED028B446A8FB08DED020B1D
:1083F00057EC106B0546019107920593002C00F095
:108400007182216849B162684A60012393408B60A0
:1084100001F02CFB6B6A00221A60B7F100081A9A6F
:10842000B4BF012300231360C14BBCBF28F0004838
:10843000CDF80C8033EA080300F0A2809DED028B9A
:10844000B5EE408BF1EE10FA10D1059A01231360BE
:108450001B9B002B00F05382B6481860431E00930C
:1084600000980FB0BDEC028BBDE8F08F0CAA0DA9EF
:108470002846B0EE480B01F019FF5FEA1853044696
:1084800040F09680DDE90C130B4403F23242202ABF
:1084900040F31C83C2F1400208FA02F803F21242D0
:1084A000D64048EA060207EE102AB8EE477B581E6F
:1084B00017EE906A01230A9353EC172BA6F1F87379
:1084C0009FED953B9FED967B9FED975B06EE900AA7
:1084D00043EC122BB8EEE64BB7EE086B32EE466B70
:1084E000A6EE037BA4EE057BFDEEC76BB5EEC07B6D
:1084F000F1EE10FA16EE908A08D5B8EEE66BB4EEFF
:10850000476BF1EE10FA18BF08F1FF38B8F1160FFB
:1085100000F2DB81884B03EBC80393ED007BB4EEE4
:10852000C78BF1EE10FA5AD5091A0023B1F10109EF
:1085300008F1FF38099300F1CF8100230693B8F1C9
:10854000000F54DA069BCDF81080A3EB08030693C6
:10855000019B092BC8F1000A4FF000084FD8052BEA
:1085600040F3B282043B01930026019B9A1E032A2A
:1085700000F21B81DFE812F0C603C303BA039903BC
:10858000059A42F20F73C8F31308136058EA060302
:108590001ED11B9B002B00F09085684B0093083385
:1085A0001B9A009813600FB0BDEC028BBDE8F08FF2
:1085B00018EE906AA3F2FF30C6F3130600230A9365
:1085C00053EC182B46F07F530C9943F4401377E794
:1085D0001B9B002B40F05883594B009340E7091A2E
:1085E0000023B1F10109099300F176810693019B03
:1085F000CDF81080092BC1444FF0000AAFD90023F9
:108600000126019308964FF0FF3B07936A6ACDF865
:108610002CB000215160284601F0E8F900900028B4
:1086200000F044856A6A009B1360BBF10E0F00F2F4
:10863000D180002E00F0CE80049B002B40F3E88315
:108640003D4A03F00F0102EBC102D90592ED007B18
:108650004FEA231240F188833A4991ED086B02F00A
:108660000F02032088EE065B5AB13649D30704D5C2
:1086700091ED006B013027EE067B521001F10801ED
:10868000F4D185EE076B099B3BB1B7EE007BB4EEEE
:10869000C76BF1EE10FA00F1AE8407EE900AB8EE67
:1086A000E75BB1EE0C7BA5EE067B17EE902A51EC52
:1086B000170BA2F15071BBF1000F00F08A83049EEA
:1086C0005A46089B002B00F04784B6EE003B1A4F39
:1086D000FDEEC64B07EBC207B8EEE47B36EE477BF8
:1086E00017ED026B83EE065B41EC160B14EE900A5D
:1086F00035EE465B0099B4EEC57B3030F1EE10FAF2
:1087000001F8010B00F1AC84B7EE002BB2EE044B84
:10871000002731E0AFF3008061436F63A787D23F4A
:10872000B3C8608B288AC63FFB799F501344D33F60
:108730000000F07F85481408649511084C4914081E
:1087400058491408549611080137974242DA27EE27
:10875000047B25EE045BFDEEC76B16EE903AB8EE97
:10876000E63B303337EE437BB4EEC57BF1EE10FAD7
:1087700001F8013B00F1748432EE476BB4EEC56B37
:10878000F1EE10FAE0D5009A049602E08A4200F079
:108790005184894611F8013D392BF7D00133DBB202
:1087A0000B70049B0133049376E16A6A00265660DD
:1087B0003146284601F01AF90090002800F076842E
:1087C0006A6A009B13604FF0FF33012207960B93F8
:1087D00008929B460D9A002A55DB04990E2952DC1B
:1087E000BE4B03EBC10393ED006B079B002B15DA27
:1087F000BBF1000F12DC40F00083B1EE047B26EEEB
:10880000076BB4EEC68BF1EE10FADA465E4600F264
:108810009282079BDDF80080DF4394E288EE067BBE
:10882000BDEEC77B009917EE103ABBF1010F03F1C3
:108830003003B8EEC75B01F8013BA5EE468B00F0B4
:108840004283B2EE044B012311E088EE067BBDEEBD
:10885000C77B013317EE102A5B4502F13002B8EEF8
:10886000C75B01F8012BA5EE468B00F02C8328EEA8
:10887000048BB5EE408BF1EE10FAE6D1049B013388
:108880000493894608E1089B002B40D0019B012BF3
:1088900040F384820BF1FF339A4580F26282A3EBAE
:1088A0000A0AD0449A460023BBF1000FC0F23C8371
:1088B000069A17465A44D9440692012128460A933B
:1088C00001F0F4F90A9B064624E0091A0123B1F1EC
:1088D000010909937FF531AEC1F1010306934FF011
:1088E00000092CE61020EDF05BFA024668620028D1
:1088F00000F0EA83C0E901440460C4608DE5784B70
:10890000009300980FB0BDEC028BBDE8F08F069F7E
:10891000089E5346002F0CDDB9F1000F09DD4F45CD
:1089200006993A46A8BF4A46891A0691BF1AA9EB8A
:108930000209BAF1000F1BD0089A002A00F06182E8
:10894000002B11DD1A46314628460A9301F072FACF
:10895000224601460646284601F0BEF92146044655
:10896000284601F083F80A9BBAEB030240F0D68256
:108970000121284601F09AF9B8F1000F824600F370
:10898000B180019B012B40F3838100230A930120D6
:10899000B8F1000F40F0B280484410F01F0000F022
:1089A0009180C0F12002042A40F39383C0F11C009F
:1089B000069B0344069307448144069B002B05DD78
:1089C00021461A46284601F0A5FA0446B9F1000FDF
:1089D00005DD51464A46284601F09CFA8246099B2D
:1089E000002B40F03681BBF1000F40F31C81089B47
:1089F000002B40F09B80049B01330493DDF8008042
:108A0000012707E0214600230A22284601F052F8F8
:108A10000137044651462046FFF74EFC5F4500F102
:108A2000300008F8010BEDDBBBF1000F009AD8BF56
:108A30004FF0010B034693440027214601222846AC
:108A4000019301F067FA5146044601F0D7FA002875
:108A500040F392811BF8013C009A0BF1FF3B04E0CC
:108A60005A4500F094811BF8013D392B0BF10109A7
:108A7000F6D001338BF800305146284600F0F6FF5F
:108A800056B12FB1B74203D03946284600F0EEFF69
:108A90003146284600F0EAFF2146284600F0E6FF6E
:108AA000002389F80030DDE904231A601B9B002BAA
:108AB0003FF4D6AC0098C3F800900FB0BDEC028B29
:108AC000BDE8F08F1C2073E701264EE5C2F12002BD
:108AD00006FA02F207EE102AE7E400BF64951108D7
:108AE0008448140801464246284601F0A3F9019B38
:108AF000012B824640F3B18100230A93DAF810205B
:108B00000AEB8202106901F081F8C0F1200043E70E
:108B1000314600230A22284600F0CCFF0B9B002B95
:108B2000064640F3B782CDF810809B46002F05DD46
:108B300031463A46284601F0EDF906460A9B002BDD
:108B400040F0D581B046029B009F03F001027B1EDE
:108B50005B440893019B0A921343099351462046B4
:108B6000FFF7AAFB31468346204601F047FA42460A
:108B700051468146284601F063FAC26801460BF16E
:108B80003003002A42D1CDE90603204601F036FA2F
:108B900006990290284600F069FF029A079B1AB9CD
:108BA0000999002900F06682B9F1000FC0F26D81C9
:108BB000019949EA01090A9951EA090100F0658120
:108BC000002A00F3B581089A3B7007F1010997422A
:108BD000CB4600F0B381214600230A22284600F04C
:108BE00069FF4645044631464FF000034FF00A0244
:108BF000284612D000F05EFF4146064600230A22B6
:108C0000284600F057FF4F468046A7E728460293C4
:108C100000F02CFF029B0122C6E700F04BFF4F46FD
:108C2000064680469AE7019B022B72DC089B002BCC
:108C30007FF47CAF049B5146013320460493FFF739
:108C40003BFBDDF800B000F130030BF8013B0027DF
:108C5000F3E65146204601F0D1F90028BFF6C3AE35
:108C6000214600230A22284600F024FF049B03F13A
:108C7000FF38089B0446002B7FF44AAF0B9B002B68
:108C800040F3FF819B46B9E6AF4B0093033387E483
:108C9000DDE9020100287FF478AEC1F31302002A57
:108CA00000F0E680029B0A9371E601230893079B7C
:108CB000049A134403F1010BBBF1010FDC460B9343
:108CC000B8BF4FF0010C6B6A0021BCF1170F59605F
:108CD0007FF7A1AC01200422520002F1140767457E
:108CE000014600F10100F7D9596094E4012308938B
:108CF000079B002B3CDD0B939B469C46E3E7002340
:108D00000893D4E700230893F2E7DDF82CB0CDF800
:108D10001080BBF1000F7FF47CAD51465B4605220D
:108D2000284600F0C7FE01468246204601F066F95B
:108D300000287FF76EAD0098049F3123804600F82D
:108D4000013B013700905146284600F08FFE7B1C06
:108D5000DDF800900493CDF80080002E7FF498AEEB
:108D60009AE6AAEB03039FE50220B0EE485B7BE4A2
:108D7000012307939B4649E403D1019BDB073FF5A1
:108D800069AED9461BF8013D302BFAD074E6049B3E
:108D9000009A01330493312313706DE60A9B002B74
:108DA00000F0208102F23342069B1F4613440693D3
:108DB0009144534681E507EE900AB1EE0C5BB8EEA4
:108DC000E77BA6EE075B15EE902A51EC150BA2F19E
:108DD000507141EC150BB1EE047B36EE477BB4EEDF
:108DE000C57BF1EE10FA00F33581B1EE455BB4EED0
:108DF000C57BF1EE10FA7FF5EDAC4FF0000A564658
:108E000007E521465246284601F014F80446AFE52E
:108E100000F0EC80049B4D495A4202F00F0001EB38
:108E2000C00191ED006B121128EE066B00F03B8142
:108E3000B0EE467B464900260220D70705D591EDC6
:108E4000005B0130012627EE057B521001F108017D
:108E5000F3D1002E06FE076B15E4029B002B7FF476
:108E60004BAEDDE90201C1F31302002A40F0298173
:108E7000384A0A40002A00F0F180069B013306932D
:108E8000012309F101090A9381E5002A12DD214637
:108E900001222846019301F03DF85146044601F0B5
:108EA000ADF80028019B40F3DF80392B00F0C8802B
:108EB0000BF13103B94609F8013B049B01333746F6
:108EC00004934646D8E538EE088BB4EEC68BF1EE37
:108ED00010FA0ADCB4EE468BF1EE10FA7FF4CEAC59
:108EE00017EE103AD8077FF5C9AC009A51E47168C3
:108EF000284600F07BFD0746002800F0EF8033692C
:108F000002339A0006F10C010C30FCF719F93946CE
:108F10000122284600F0FEFF804614E6214628463E
:108F200000F088FF044623E5069AA2EB0B07C4E491
:108F3000392B00F08580B9460133BCE7049A013231
:108F400037460492464678E5584914086495110856
:108F5000549611080000F07F644FFDEEC65B07EBEE
:108F6000C20717ED023BB8EEE57B36EE477B41ECDE
:108F7000160B15EE901A23EE063B00983031012AAD
:108F800000F8011B00F08480B2EE044B009B99189E
:108F900027EE047BFDEEC76B16EE903A303300F8F7
:108FA000013B8842B8EEE65B37EE457BF0D1B6EE8A
:108FB000006B33EE065BB4EEC75BF1EE10FA3FF5E3
:108FC000E2AB36EE436BB4EEC76BF1EE10FA7FF70F
:108FD00001AC8946013919F8013C302BF9D0731CDA
:108FE000049359E50C9AC2F13602DDE60220B0EE98
:108FF000486BFFF748BBBBF1000F3FF4DCAE0B9AA8
:10900000002A7FF7E7ABB2EE044B26EE046B01308B
:1090100007EE900A049BB8EEE75BB1EE0C7BA6EE80
:10902000057B17EE907A51EC170B5E1EA7F150717D
:10903000FFF747BB049B013304933123FFF7B0BB19
:10904000049BBB4601330493392337460BF8013B9D
:10905000464601E54FF0000A56466CE60A9296E451
:10906000731C0493894617E57FF424AFDA077FF574
:1090700021AF1AE7392BE3D0B9F1000F3FF718AF52
:1090800018E7019B022B3FF740AECDF81080D1E5E9
:1090900001468CE7019B022B3FF737AEDDF82CB081
:1090A000CDF8108042E50220FFF7EDBA104B1148D1
:1090B00000224FF4D571FFF7D9F80F4B0093FFF75B
:1090C000CFB9029B0A9319E50C4B0A48EA21FFF736
:1090D000CDF83FF472ACC0F13C0069E4044B0548A4
:1090E0003A4640F2EA21FFF7C1F800BF6495110843
:1090F000904914085C4914084C491408B0481408F5
:10910000704700BF704700BF0CB400B583B004AB1C
:1091100053F8042B019301F01BFA03B05DF804EB44
:1091200002B070470EB410B583B005AB064C53F8CF
:10913000042B01930146206801F00AFA03B0BDE850
:10914000104003B0704700BF042200302DE9F04109
:109150000469B4EB611F2FDD00F1140E4E1111F004
:109160001F0C0EEB84050EEB86032BD05EF8262039
:1091700004339D4222FA0CF1CCF1200818D977462D
:109180001A6802FA08F20A4347F8042B53F8041B42
:109190009D4221FA0CF1F3D8A41BA300053B9B08C8
:1091A00001330EEB83044EF82310C9B1043417E0E9
:1091B000416174460029F9D1002303610023436112
:1091C000BDE8F0819D4288BF00F11002F4D953F848
:1091D000041B42F8041F9D42F9D8A41B0EEB840423
:1091E000A4EB0E039B1074450361E7D0BDE8F0814A
:1091F0002DE9F04FAE4C2DED028B24688BB008EEBC
:10920000100A20468946039207930494FDF70CFB4D
:10921000D9F800302118024611F801BC997830299C
:1092200040F0E5816FF00100C01A033300EB030A40
:109230001C4613F8011B3029F8D0DFF8788218F8A3
:109240000130002B00F0F7802378002718F8033056
:109250003D4626462BB116F8013F18F80330002B87
:10926000F9D1049902923046FDF778FB029A0190F9
:10927000002800F09680002D40F09680337801950C
:1092800003F0DF03502B354600F09880C9F80060EA
:10929000002F40F0B0802B1B013B072B394604DD2B
:1092A0005B10072B01F10101FADC18EE100A0592A0
:1092B00000F09CFB059A0290002800F07182029B4E
:1092C000AC4203F11406069680F0E7810027C2F154
:1092D0000103B946059310E0202F00F0978039462E
:1092E000043715F8013C18F80330554603F00F0316
:1092F0008B40A54249EA030916D915F8013C5B45A4
:1093000005F1FF3AE8D1059B5344A342E4D3184644
:10931000049909920893FDF721FBDDE90832002842
:10932000DAD11D46A542E8D846F8049B069BF61AFA
:10933000029BB6101E61484600F068FC039B760154
:109340001C68301AA04200F3B780C0F22F810027BA
:10935000039B019A9B689342C0F293810399019AFF
:109360004B68934240F384809D1AAC4200F3C48062
:10937000CA68022A00F0C681032A00F0BE81012AD1
:1093800000F0A28118EE100A029900F06FFB502540
:10939000169A0023284613600BB0BDEC028BBDE883
:1093A000F08F002D00F01181AD1BAB0001933378DD
:1093B00003F0DF03502B35467FF468AF6B782B2B1F
:1093C00000F0F2802D2B6ED06E1C002018F80310D8
:1093D0004B1E182B65D8737818F8033010390136F6
:1093E00033BB00B14942019BC9F800600B440193B3
:1093F000002F3FF450AFBAF1000F14BF002506252F
:1094000028460BB0BDEC028BBDE8F08F002146F87A
:10941000049B0427894664E701EB810103EB4103C8
:10942000A3F1100116F8013F18F80330002BD8D033
:10943000192BF1DDD5E7049901922046FDF78EFA4C
:10944000019A002876D1A15C18F80130A518002BEC
:1094500072D030292C4605D114F8013F302BFBD0B7
:1094600018F80330B3FA83F77F094FF0010AF0E6EA
:10947000012557B1039BDB68022B65D0032B67D016
:10948000012B00F0888045F01005169B029A1A60A7
:10949000079B019A1A6028460BB0BDEC028BBDE811
:1094A000F08F2E46F2E60120AB78AE1C8EE700BFAF
:1094B0004895110848941108029D061B314628461C
:1094C00000F0D0FF074678B1721E531106990127AC
:1094D00051F8231002F01F0307FA03F30B4203D0E5
:1094E000BA4200F3E4800227019B029833443146DC
:1094F0000193FFF72BFE2BE76E1E002F40F0CB8071
:10950000002E40F0CE807311069A029852F8232064
:1095100006F01F06012303FA06F61642294618BF75
:1095200047F00207FFF712FE039B5B680193641B81
:1095300002259EE72178254601F0DF01502900F041
:10954000BF80C9F8005056E7179BC3F1010317937A
:10955000179B002B97D0029BDDF818901E69002105
:109560004B464FEA860809EB860003E0984243F831
:10957000041C40D91F4653F8042BB2F1FF3FF5D02D
:109580000132022D3A6000F0C28014F01F0440F056
:10959000E180212579E7BA077FF575AF069B1B6847
:1095A0001F43FB07D7D46EE700207DE7DDE90131DB
:1095B000221A9B1A18EE100A019300F0ABFC034626
:1095C0001433029006930027C2E6B35C18F8031028
:1095D000B018064600293FF453AE16F8013F18F8BC
:1095E00003100029F9D1801B8100019148E69C1CE1
:1095F0004FF0000A21E6029B9B689E4280F28E801B
:109600003346029901EB830201330B61022D4FF0C7
:10961000010151617BD09E42B7DA002B40F3A78055
:10962000029A09EB8303516902F1180083424FEA61
:10963000510140F2AF804C46026841EAC27144F8E1
:10964000041B50F8041B83424FEA5101F4D8029ADC
:109650009B1A193B9B08013349F8231009EB83033C
:10966000002940F09B800299A3EB090292104B4520
:109670000A617FD0039B019A9B6801329342019259
:1096800087DA029918EE100A00F0F0F9169A002312
:109690001360A325B4E6012735E7069E4FF00009C5
:1096A00042E60298314600F0DDFE07462BE7B11E88
:1096B000284600F0D7FE00283FF415AF032713E734
:1096C00000230193012779E6AC427FF45BAE012CC5
:1096D00008D00298611E00F0C5FE00283FF452AE8B
:1096E000039B5B6807990B60029B069901221A6134
:1096F0000A60169A6225136082E6179A002A3FF4E0
:1097000041AEEFE7179A002A7FF43CAEEAE7039BED
:109710001B68013BA34231D02225B6E6029B596863
:1097200018EE100A013100F061F9074600283DD01B
:1097300002990B6902339A000C310C30FBF700FDE3
:10974000029918EE100A00F091F907F114093B692B
:10975000029756E7C844C4F1200458F8040C00F0FE
:1097600055FAA042BFF615AF029B1B6955E7029A56
:1097700000231361029A002353617BE7631104F015
:109780001F0459F823200123A34013420CBF2225B4
:1097900021257AE6C9F800104B4669B1043362E727
:1097A000074B0848029ADE21FEF760FD044B05488E
:1097B0003A468421FEF75AFD029B1961DAE700BFA1
:1097C00090491408A449140810B4046809E014F876
:1097D000013FA3F1410CBCF1190F98BF2033934214
:1097E00009D111F8012B002AF1D1013404600120C4
:1097F0005DF8044B704700205DF8044B704700BFD4
:109800002DE9F04F096885B04B1111F01F0102904E
:1098100002EB8303039140F08E801D1F0193029B96
:1098200001991C68002341F8043C61780134002947
:1098300000F09780DFF87091A846AC469A461E4625
:109840000EE0202900F28B80B24506DAC44501D231
:10985000072B5BDD624551D3082314F8011FA1B12A
:1098600019F801000028ECD00133082B06F101069D
:109870003ADCDCF80010090100F00F000843CCF8D6
:10988000000014F8011F0029EAD1002E69D0E0453C
:1098900001D9072B73DD624551D2111F634653F87E
:1098A000040B41F8040F9D42F9D2A5EB0C0323F001
:1098B0000303691C04330CF1010C614538BF042318
:1098C0001344002143F8041B9D42FBD2019B53F833
:1098D000043C2BB9AA4248D055F8043D002BF9D0DE
:1098E000052005B0BDE8F08F6245B6D200234CF8E4
:1098F000043C1946ACF1040C0123BDE70023ACF194
:1099000004084CF8043CB246C446A6E7C3F108017B
:109910008900DCF80030C1F1200E60468B464168BA
:1099200001FA0EF73B43036021FA0BF340F8043FC2
:109930004045F4D38EE7191D01911D466FE7039B47
:10994000002BC3D0039B0198C3F120014FF0FF33DC
:10995000CB4050F8041C0B4040F8043CB9E72929DF
:1099600009D0042005B0BDE8F08F012305202B604D
:1099700005B0BDE8F08F029901340C6085E7C3F1B2
:1099800008039B00DCF80010C3F1200764466668FA
:1099900006FA07F00143216026FA03F144F8041F98
:1099A000A045F4D877E700BF4894110810B4034CE1
:1099B000D4F8E440A4465DF8044B604770220030C0
:1099C00082B049B15AB16BB113780B601278101E96
:1099D00018BF012002B0704701A9002AF3D1104638
:1099E00002B070476FF00100F4E700BF70B5466A3F
:1099F00005460C465EB1F368A3B153F82400E8B104
:109A0000026843F824200023C0E9033370BD10200E
:109A1000ECF0C6F906466862E8B10023C0E90133FC
:109A20000360C360212204212846ECF0ADFA6B6A82
:109A3000F060DB68002BE0D1002070BD012101FA4D
:109A400004F6721D92002846ECF09EFA0028F3D02E
:109A5000C0E90146D7E7034B034832466621FEF7CB
:109A600005FC00BFB0481408F049140870B5456AF9
:109A700004460E464DB13EB1636A7268DB6853F826
:109A80002200306043F8226070BD1020ECF088F9AD
:109A90000246606220B1C0E901550560C560EAE791
:109AA000024B03488A21FEF7E1FB00BFB0481408CF
:109AB000F0491408F0B50C69064683B00D4601F173
:109AC000140E0020DEF800101FFA81FC02FB0C339C
:109AD0004FEA134C090C02FB01CC01309BB203EBA3
:109AE0000C4384424EF8043B4FEA1C43EADC3BB192
:109AF000AA68A24207DD05EB8402013453612C61A0
:109B0000284603B0F0BD6968019301313046FFF784
:109B10006DFF019B0746A0B12A69019302329200B2
:109B200005F10C010C30FBF70BFB294630463D4696
:109B3000FFF79CFF05EB8402019B536101342C610C
:109B4000DEE7034B03483A46B521FEF78FFB00BF23
:109B500090491408F04914082DE9F8430C462849A7
:109B60001F46164603F1080281FB0231092F4FEA16
:109B7000E2730546C3EB610339DD4FF0010C0021B0
:109B80004FEA4C0C634501F10101F9DC2846FFF76F
:109B90002DFF014668B3089B4361092E4FF0010376
:109BA000036112DC0A340926B7420BDDBE1B2644D2
:109BB00014F8013B0A22303B2846FFF77BFFA64200
:109BC0000146F5D10846BDE8F88304F10909C84605
:109BD000344418F8013B0A22303B2846FFF76AFF5D
:109BE000A0450146F5D1A6F108044C44DCE700216C
:109BF000CCE70A46034B0448CE21FEF737FB00BFF3
:109C0000398EE33890491408F0491408030C1B04FA
:109C1000D3B90004102310F07F4F04BF00020833B3
:109C200010F0704F04BF0001043310F0404F04BF28
:109C300080000233002805DB10F0804F03F10103A0
:109C400008BF2023184670470023E4E7036813F099
:109C50000702014607D0DA071FD4980721D55B0811
:109C60000B600120704798B2A0B11046DAB20AB971
:109C700008301B0A1A0704BF1B0904309A0704BFE7
:109C80009B080230DA0703D45B0800F1010006D01C
:109C90000B6070471B0C1020E8E700207047202065
:109CA00070479B080B600220704700BF10B50C4640
:109CB0000121FFF79BFE024618B10123C0E90434DD
:109CC00010BD034B03484FF4A071FEF7CFFA00BF5D
:109CD00090491408F04914082DE9F04F0E691569F0
:109CE000AE4285B08846144605DB2A4623463546F3
:109CF0000C4616469846A3686168AF19BB42B8BFC8
:109D00000131FFF773FE0190002800F08780019B6E
:109D100003F1140909EB870AD14505D24B4600220D
:109D200043F8042B9A45FBD808F1140808EB860B7E
:109D300004F11403D8451A4603EB85055FD22B1BAB
:109D4000153B23F0030304331534A54238BF042325
:109D5000CDE902A7AC461F46924605E0000C29D18A
:109D6000C34509F1040948D958F8040B85B2002D00
:109D7000F4D056464C46002356F8040B216882B2B4
:109D80001FFA81FE05FB02EE000C0A0C734405FB72
:109D9000002202EB13429BB243EA0243B44544F86B
:109DA000043B4FEA1243E7D849F8073058F8040C4F
:109DB000000CD5D0D9F80030544619464D46002243
:109DC0002688090C00FB06110A449BB243EA0243B1
:109DD00045F8043B54F8046B2968360C8BB200FB41
:109DE000063303EB1243A4454FEA1342E8D8C345B8
:109DF00049F8073009F10409B6D8DDE902A7002FB8
:109E000002DC05E0013F03D05AF8043D002BF9D0F5
:109E1000019B18461F6105B0BDE8F08F034B044855
:109E2000019A40F25D11FEF721FA00BF9049140833
:109E3000F04914082DE9F04112F0030382B01446F2
:109E400007462DD10E46A4101CD07A6A8AB39568B5
:109E5000002D39D0E3074FF0000806D4641011D06C
:109E6000286898B10546E307F8D531462A463846B2
:109E7000FFF732FF3146034638461E46FFF7F6FD30
:109E80006410EDD1304602B0BDE8F0812A46294683
:109E90003846FFF721FF2860C0F800800546E2E75A
:109EA000013B184A52F823200023FFF703FE064621
:109EB000C9E71020EBF074FF02467862E0B100239E
:109EC000C0E901330360C360012138460192FFF706
:109ED0008DFD019A054640B1012340F27121C0E990
:109EE0000431002390600360B4E7074B07482A461B
:109EF0004FF4A071FEF7BAF9054B04484FF4D7713F
:109F0000FEF7B4F95495110890491408F049140863
:109F1000B04814082DE9F0470D4691462F69AB680B
:109F2000496807EB62177C1C9C4280464FEA621A24
:109F300004DD5B009C4201F10101FADC4046FFF7C1
:109F400055FD064600284DD0BAF1000F00F114006F
:109F50000EDD0AF105024FEA820C034606EB82028F
:109F6000002143F8041B9342FBD1ACF114031844C5
:109F7000296905F1140319F01F0903EB810129D0A8
:109F8000C9F1200E84464FF0000A1A6802FA09F25D
:109F900042EA0A024CF8042B53F8042B994222FAA5
:109FA0000EFAF2D84B1B153B23F00303043305F1E3
:109FB0001502914238BF0423BAF1000F18BF27469B
:109FC00040F803A0404637612946FFF74FFD304671
:109FD000BDE8F087043853F8042B40F8042F994269
:109FE000F9D8EFE7034B0448324640F2D911FEF7A7
:109FF0003DF900BF90491408F04914080B698446E4
:10A000000069C01A16D10CF1140C14310CEB830248
:10A0100010B401EB830301E0944508D252F8044DDB
:10A0200053F8041D8C42F7D005D24FF0FF305DF895
:10A03000044B7047704701205DF8044B704700BF28
:10A040002DE9F84F0F691369FF1A002F0E4690464D
:10A050007AD101F11405143202EB830205EB83037C
:10A0600001E09D4273D253F8041D52F8044DA14201
:10A07000F7D064D37168FFF7B9FC8146002872D02D
:10A080003569D8F81020C76008F1140E06F11400E5
:10A0900009F1140A06F1100C0EEB820200EB8507A1
:10A0A000564600215EF8044B5CF804BFA3B211FAD7
:10A0B0008BF1CB1A210CC1EB1B4101EB23419BB26D
:10A0C00043EA0143724546F8043B4FEA2141E9D88F
:10A0D000A2EB0804153C08F11508424524F00306DC
:10A0E00006F1040638BF0426304424F0030238BFCA
:10A0F000002287425244B24416D95646044654F8C8
:10A10000043B11FA83F10A1402EB134289B241EACB
:10A110000243A74246F8043B4FEA2241EFD87A1E99
:10A12000101A20F00302524423B952F8043D013DB5
:10A13000002BFAD0C9F810504846BDE8F88F3346D6
:10A1400001274646984695E7F9DB002792E700216C
:10A15000FFF74CFC814668B101220023C9E90423C2
:10A160004846BDE8F88F074B07484A464FF4107140
:10A17000FEF77CF8034B04484A4640F23221FEF7D2
:10A1800075F800BF90491408F049140882B08DEDAD
:10A19000000B154B019A1340A3F15073002B05DD02
:10A1A0000020194641EC100B02B070475B42B3F13E
:10A1B000A07F4FEA235208DA4FF40023002043FA2D
:10A1C00002F141EC100B02B07047143A1E2ADABFBC
:10A1D0004FF0004323FA02F201220021104641EC25
:10A1E000100B02B0704700BF0000F07FF8B50469A3
:10A1F00000F1140606EB8404271F54F8045C28467B
:10A20000FFF704FDC0F120030A280B6031DDBE42D8
:10A210001BD20B3854F8081C23D0C0F1200C854009
:10A2200021FA0CF72F43A4F1080547F07F53AE4203
:10A2300043F4401336D2814054F80C0C20FA0CF051
:10A240000843024643EC102BF8BD0B3808D005FA42
:10A2500000F040F07F53002043F440130246F1E742
:10A26000014645F07F5343F440130A4643EC102B5C
:10A27000F8BDC0F10B0C25FA0CF1BE4241F07F5342
:10A2800038BF54F8081C00F1150034BF21FA0CF156
:10A29000002105FA00F043F4401340EA010243ECC8
:10A2A000102BF8BD01FA00F00246CBE72DE9F04390
:10A2B000884683B0012157EC106B1546FFF796FBDB
:10A2C000044600284FD0C7F30A59C7F31303B9F166
:10A2D000000F01D043F48013002E019324D0684670
:10A2E0000096FFF7B3FC002839D0DDE90013C0F178
:10A2F000200203FA02F20A43C34062610193002B79
:10A3000014BF02220122A3612261B9F1000F16D00D
:10A31000A9F233430344C0F13500C8F80030286087
:10A32000204603B0BDE8F08301A8FFF78FFC019B36
:10A330006361012220302261B9F1000FE8D104EB02
:10A340008203A0F23240C8F800001869FFF75EFCF3
:10A35000C0EB42102860204603B0BDE8F083009BAC
:10A360006361019BCBE7034B0348224640F20A316D
:10A37000FDF77CFF90491408F0491408F0B583B04C
:10A380000E4669460746FFF731FF01A9304655ECF6
:10A39000104BB0EE407BFFF729FF3B693169591A3A
:10A3A000DDE90023D31A03EB4113002B09DD17EE7F
:10A3B000902A02EB035545EC174B87EE000B03B0D8
:10A3C000F0BD10EE902A51EC100BC3EB033302EBFF
:10A3D000035141EC100B87EE000B03B0F0BD00BF42
:10A3E000172808DDB7EE000BB2EE047B013820EE33
:10A3F000070BFBD17047034B03EBC00090ED040B40
:10A40000704700BF549511080139491101F1010C41
:10A41000116902F1140303EB81018B4200EB8C0CF8
:10A4200016D210B5A0F1040E53F8044B4EF8044FA9
:10A430009942F9D88B1A153B23F0030304331844CF
:10A44000844504D9002340F8043B8445FBD810BD63
:10A45000844505D9002340F8043B8445FBD8704768
:10A46000704700BF03694A11934200F1140009DAF2
:10A4700000EB830302E053F8042DCAB98342FAD8F3
:10A480000020704711DD11F01F010ED010B450F8FC
:10A49000224000EB820324FA01F202FA01F18C421D
:10A4A0000CD001205DF8044B704700EB8203E5E718
:10A4B0000120704753F8042D002AF2D18342F9D8C5
:10A4C00000205DF8044B70479368013B002B9360BC
:10A4D00011DA10B49469A34209DB0A2907D0136882
:10A4E000581C1060197008465DF8044B70475DF801
:10A4F000044B00F07DB91368581C106019700846B1
:10A50000704700BF9BB1F8B5134406460F46541E72
:10A510005D1E01E0AC4208D014F8011F3A463046F7
:10A52000FFF7D2FF431CF5D1F8BD0020F8BD002095
:10A53000704700BF936810B5144613B953601846AE
:10A5400010BD00F06BFC0023C4E9013310BD00BF57
:10A550002DE9F04F88469FB015461C46814618B13C
:10A560008369002B00F0A280924B984500F0A480F4
:10A57000914B984500F0B180904B984508BFD9F8B1
:10A580000C80B8F80C30180740F19D80D8F81030D6
:10A59000002B00F0988000230B932978884E0594B7
:10A5A00020238DF8313030238DF8323001270029F7
:10A5B00074D02C460B4604E014F8013F002B00F049
:10A5C0008F80252BF8D1B4EB050B40F08C802378DD
:10A5D000002B63D000234FF0FF32CDE90723069311
:10A5E00009938DF85B301C93013404E0069A07FA56
:10A5F00003F3134306932546052214F8011B304646
:10A60000FAF71CFD831B0028F0D1069BD90644BF36
:10A6100020228DF85B2029781A0744BF2B228DF861
:10A620005B202A2970D1059A11680432002905920D
:10A63000C0F29B800991697801352E2976D0614C52
:10A6400003222046FAF7FAFC38B1069B001B40248F
:10A6500004FA00F003430693013515F8011B5A482C
:10A660008DF830100622FAF7E9FC002800F083800C
:10A67000564B002B6DD005AA0092554B424606A9B9
:10A680004846FBF75BF90390039B013306D00B9B15
:10A69000039A297813440B9300298AD1B8F80C3017
:10A6A0005B0617D40B981FB0BDE8F08F00F096FB47
:10A6B000404B98457FF45CAFD9F80480B8F80C3073
:10A6C00018073FF563AF4146484600F00DF90028F2
:10A6D0003FF461AF4FF0FF30E5E7D9F8088050E76D
:10A6E000B4EB050BDAD0AA46C5F1010503E09345AA
:10A6F00036D91AF8011F42464846FFF7E5FE0130F9
:10A7000005EB0A02F3D1C9E7A1F13002092A94D876
:10A71000099B15F8011F03EB830302EB4303A1F12F
:10A720003002092AF5D92E29099388D169782A2976
:10A730002BD1059BA9781A6807920433002A05F1EA
:10A7400002000593B8BF4FF0FF330546B8BF07932B
:10A7500075E7059B073323F007030833059396E756
:10A760000B9A23785A440B9232E7494243F0020392
:10A77000099106935FE705AA0092154B424606A988
:10A780004846FBF7F3FB03907EE7A1F1300200237C
:10A79000092A079305F101053FF651AF15F8011F8E
:10A7A00003EB830302EB4303A1F13002092AF5D93D
:10A7B000079344E7BC9611089C9611087C961108F3
:10A7C000244A14082C4A1408304A14083D59020837
:10A7D00005A5020810B4054C8446134620685DF8B0
:10A7E000044B0A466146FFF7B3BE00BF04220030A7
:10A7F000F8B50D461446064608B1836943B3254BA8
:10A800009C422AD0244B9C4229D0244B9C4208BF16
:10A81000F468A389A269A2601A0722D5236903B349
:10A8200022686169D31AEDB299422F4629DD0133BE
:10A83000A1680139A160511C2160157062699A42BA
:10A8400016D0A389DB0701D50A2D11D03846F8BDF3
:10A8500000F0C4FA0F4B9C42D4D17468D9E7B468B5
:10A86000D7E72146304600F03FF838B92369D7E7EB
:10A870002146304600F04CF90028E7D04FF0FF3772
:10A88000E4E72146304600F043F90028F6D122687B
:10A890000123CDE7BC9611089C9611087C961108FF
:10A8A00010B4044C03460A4620685DF8044B194670
:10A8B000FFF79EBF0422003010B4034CD4F8E040F0
:10A8C000A4465DF8044B60477022003049B1FF2A6E
:10A8D00002D80A70012070478A2303604FF0FF30CE
:10A8E00070470846704700BF3C4B70B51D68064670
:10A8F0000C460DB1AB69E3B1394B9C421FD0394BCB
:10A900009C424DD0384B9C4208BFEC68B4F90C30E7
:10A9100018079AB219D5216911B312F001002FD08E
:10A920000020A06060694042A06100292ED0002074
:10A9300070BD284600F052FA294B9C42DFD16C686A
:10A94000B4F90C3018079AB2E5D4D1063ED55207B7
:10A9500028D4216943F00803A3819AB20029DCD1ED
:10A9600002F42070B0F5007FD7D02146304600F0C9
:10A9700011FCB4F90C3021699AB212F00100CFD168
:10A98000950758BF6069A0600029D0D1120658BF52
:10A990000846CDD543F04003A3814FF0FF3070BD92
:10A9A000AC68B3E7616B51B104F14402914204D049
:10A9B0003046EBF0F1FAB4F90C3000226263216901
:10A9C0000022C4E9001223F02403C3E7092243F064
:10A9D000400332604FF0FF30A38170BD042200308D
:10A9E000BC9611089C9611087C96110808B50620A3
:10A9F00000F01AFD0120EAF09FFD00BF8B891A07C5
:10AA00002DE9F0410C4680463FD44A68002A58DDC3
:10AA1000E66A002E52D00022D8F80050C8F8002074
:10AA200013F4805251D10123216A4046B047431CA0
:10AA30005ED0A389E66A5F0705D56368C01A636BB9
:10AA40000BB1236CC01A216A024600234046B0476E
:10AA5000411C3CD1D8F80030002B38D01D2B01D040
:10AA6000162B4DD123690022C4E90032616BC8F86E
:10AA7000005019B304F14403994202D04046EBF070
:10AA80008BFA00206063BDE8F0810E69B6B10D68F5
:10AA90000E609A070CBF4B690023AD1B8B600BE067
:10AAA0002B463246216AA76A4046B847B0F1000CEF
:10AAB000A5EB0C05664413DD002DF1DC0020BDE89C
:10AAC000F0810A6C002AA3DCF8E7606DB3E700238D
:10AAD000636023692360A389DB04C7D56065C5E78C
:10AAE000A38943F040034FF0FF30A381BDE8F0811C
:10AAF000D8F80030002B9CD01D2B06D0162B04D08C
:10AB0000A38943F04003A381D9E7C8F80050D5E7F3
:10AB100038B50B69BBB10D46044608B18369B3B1C2
:10AB20000D4B9D4211D00D4B9D4213D00C4B9D42BD
:10AB300008BFE568B5F90C302BB129462046BDE8C1
:10AB40003840FFF75BBF002038BD6568F2E700F0D2
:10AB500045F9E5E7A568EDE7BC9611089C96110854
:10AB60007C96110838B540B303690446E3B1174B2E
:10AB70001D680DB1AB69CBB1154B9C420FD0154B85
:10AB80009C4221D0144B9C4208BFEC68B4F90C30B5
:10AB900053B121462846BDE83840FFF72FBF6C6807
:10ABA000B4F90C30002BF4D1002038BD284600F059
:10ABB00015F9074B9C42E2D1F1E7084B08491868A8
:10ABC000BDE8384000F0C2BAAC68DFE704220030CC
:10ABD000BC9611089C9611087C961108F4931108F4
:10ABE00011AB020800207047014900F0AFBA00BF66
:10ABF00011AB02080020704770B568224D1E02FBA1
:10AC000005F50E4605F17401EBF0C2F9044640B1BA
:10AC100000210C30C4E90016A06005F16802FAF7C3
:10AC200077FD204670BD00BF274B2DE9F0411E681F
:10AC3000B369074653B348364FF00408D6E90134E8
:10AC4000013B04D51EE05A1C04F168041AD0B4F983
:10AC50000C50013B002DF6D11C4B6566C4E9005534
:10AC6000C4E90253C4E90455A5610822294604F148
:10AC70005C00FAF74DFDC4E90D55C4E912552046B4
:10AC8000BDE8F08135682DB12E46D7E7304600F09B
:10AC90001FF8D0E74FF4D6713846EBF079F9044647
:10ACA00068B10560C0F804800C302946A0602546D4
:10ACB0004FF4D072FAF72CFD34602E46BEE70C2319
:10ACC00030603B60DBE700BFF49311080100FFFF39
:10ACD0002DE9F84F344B35491A68816290424FF0A4
:10ACE0000003C0E91233036504BF012383610546F5
:10ACF000FFF79AFF68602846FFF796FFA86028468E
:10AD0000FFF792FF6F68E86000240423C7E902435D
:10AD100008222146C7E90044C7E904447C66BC61B7
:10AD200007F15C00FAF7F4FCDFF88CB0AE68DFF8EE
:10AD30008CA0DFF88C90DFF88C801D4BC7F828A022
:10AD4000C7E9087BC7F82C90C7F830800822F36069
:10AD5000C6E90044C6E904447466B460B46121469F
:10AD600006F15C00FAF7D4FCC6E9086BC6E90AA94B
:10AD7000C6F83080EE680F4BF360C6E90044C6E9C0
:10AD800004447466B460B4612146082206F15C0094
:10AD9000FAF7BEFC0123C6E9086BC6E90B98C6F8B2
:10ADA00028A0AB61BDE8F88FF4931108E9AB020865
:10ADB000090001001200020099B50208C1B502089D
:10ADC00001B6020821B60208024B0349186800F0D8
:10ADD000BDB900BFF493110811AB0208836903B930
:10ADE00076E77047704700BF704700BF704700BFED
:10ADF000704700BF024B0349186800F087B900BFD5
:10AE000004220030E5AB0208024B0349186800F049
:10AE10007DB900BF04220030F5AB02089368002B17
:10AE200000F085802DE9F04FB1F90C300C46190780
:10AE3000804683B0174698B225D523691BB310F01E
:10AE400002033D682DD04FF0000ADFF8BCB2564631
:10AE5000B9465E453346524628BF5B464046002E03
:10AE600052D0216AA76AB847002856DDD9F80830C1
:10AE70001B1A8244361AC9F80830002BE9D1002089
:10AE800003B0BDE8F08F21464046FFF72DFD0028B6
:10AE900040F03681B4F90C303D6898B210F00203EE
:10AEA000D1D110F0010944D14E46009746B3820536
:10AEB000D4F808B040F18380B3455A4600F2B2801E
:10AEC00010F4906F40F0BF80206801924946FAF775
:10AED000A3FBA368019AA3EB0B012368A1601344B1
:10AEE000B24623600026009B9868A0EB0A00D1447C
:10AEF00098600028C3D0B4F90C0080B2002ED6D1DF
:10AF0000D5E900960835D1E7D5E900A60835A0E7D0
:10AF100021464046FFF7FCFD80B3B4F90C3043F006
:10AF200040034FF0FF30A38103B0BDE8F08F002055
:10AF300070471E46AA46994618461D46009756B3C6
:10AF400088B34A46D4E904132068B24228BF324687
:10AF5000884205D9A16803EB010B5A4500F3A6808E
:10AF6000934263DC216AA76A2A464046B847B0F19B
:10AF7000000BD2DDB9EB0B09CAD00120009A93680F
:10AF8000A3EB0B035D44A6EB0B069360002B3FF491
:10AF900076AF002ED4D10AF1080353E902569A463F
:10AFA0000833002EF9D032460A212846FAF746F82F
:10AFB000002800F09C800130A0EB0509C1E7206863
:10AFC0002369984216D86369B34213D86FF00042E0
:10AFD000B24228BF3246216A92FBF3F2A76A02FB13
:10AFE00003F340464A46B847B0F1000A95DDA6EBA8
:10AFF0000A0678E7B345DA4628BFB24652464946C4
:10B00000FAF70AFBA3682268A3EB0A035244A36081
:10B010002260002BEBD121464046FFF779FD002846
:10B02000E5D07AE72068B34632464EE729460192DA
:10B03000FAF7F2FA019AA3689B1AA36023681344F3
:10B040002360934696E723682169A3EB010B6369AC
:10B0500003EB430A0AEBDA7A0BF101034FEA6A0ABF
:10B0600033445345524684BF9A46524643052CD535
:10B0700011464046EAF08CFF00283BD05A46216931
:10B080000190FAF75DF8A289019B22F4906242F0E8
:10B090008002A28103EB0B002361AAEB0B03C4F82F
:10B0A00014A0A3602060B34632460EE729465A46F4
:10B0B000FAF7B2FA23685B44236021464046FFF763
:10B0C00027FD00283FF456AF27E7404600F0F0F890
:10B0D00003460028DED121694046EAF05DFFB4F95D
:10B0E0000C300C2223F08003C8F8002017E7721CF4
:10B0F000914627E70C22B4F90C30C8F800200EE77F
:10B100004FF0FF30BCE600BF00FCFF7F2DE9F041AF
:10B11000884600F148070026D7E90154013D0FD4C5
:10B12000A389012B05F1FF3506D9B4F90E3001339F
:10B13000204601D0C04706436B1C04F16804EFD1E0
:10B140003F68002FE8D13046BDE8F0812DE9F84393
:10B150000746884600F148064FF00009D6E9015439
:10B16000013D11D4A389012B05F1FF3508D9B4F9AC
:10B170000E300133214603D03846C04749EA000962
:10B180006B1C04F16804EDD13668002EE6D1484608
:10B19000BDE8F883F0B58B890C46990797B007D5C1
:10B1A00004F147030122C4E90432236017B0F0BD63
:10B1B000B4F90E10002905462DDB6A4600F05CFA52
:10B1C000002827DB019E06F470464FF48067A6F541
:10B1D0000056B6FA86F6394628467609EAF0D8FED1
:10B1E00030B3A3891A4AAA6243F08003C4E9040772
:10B1F000A3812060002ED9D0B4F90E10284600F0AB
:10B2000051FA0028D2D0A38923F0030343F00103AD
:10B21000A381CBE7A38913F0800F14BF40274FF41D
:10B220008067394628460026EAF0B2FE0028D8D1C9
:10B23000B4F90C309A05B9D423F0030304F14702A2
:10B2400043F002030121C4E90421A3812260ADE798
:10B25000E9AB020870B50C46B1F90E10002996B0A2
:10B2600016461D4613DB6A4600F006FA00280EDB80
:10B27000019901F47041A1F50051B1FA81F14FF447
:10B280008063490900202960336016B070BDB4F9AD
:10B290000C3000221B062A6004D5402300203360B6
:10B2A00016B070BD4FF480630020336016B070BDDF
:10B2B000F8B51446F9B1CAB106460D4600F01AFABF
:10B2C000A04202D32F463846F8BD21463046EAF068
:10B2D0005FFE07460028F6D022462946F9F730FFE0
:10B2E00030462946EAF058FE3846F8BD2746EAF0CF
:10B2F00053FE3846F8BDBDE8F8401146EAF048BEB6
:10B3000038B5446C0CB1002038BD80210546EAF008
:10B310003FFE0246686430B1031F7C3243F8044F9D
:10B320009342FBD1EFE74FF0FF3038BD1F29F8B54E
:10B33000054608D8466C0C4617464EB156F8240010
:10B3400046F82470F8BD162303604FF0FF30F8BDB7
:10B350008021EAF01DFE0646686440B1031F00F13B
:10B360007C05002143F8041F9D42FBD1E6E74FF026
:10B37000FF30F8BD1F2938B5054620D8426C0C4671
:10B380006AB152F8213053B1012B16D0591C10D09C
:10B390000025204642F824509847284638BD2846C4
:10B3A00000F0F8F8224601462846BDE8384000F093
:10B3B000DBB816230360012038BD002038BD1623FA
:10B3C00003604FF0FF3038BD1F292AD8426C38B5D2
:10B3D0000C46054682B152F8243002EB84024BB190
:10B3E000591C19D0012B15D000252046156098470F
:10B3F000284638BD012038BD8021EAF0C9FD02464B
:10B40000686458B1031F00217C3043F8041F984240
:10B41000FBD1E0E7032038BD022038BD4FF0FF30FC
:10B4200038BD4FF0FF30704738B5144B1F281D68EA
:10B430001FD86A6C044662B152F820304BB1012B20
:10B4400015D0591C0FD0002542F8205098472846A7
:10B4500038BD284600F09EF8224601462846BDE841
:10B46000384000F081B816232B60012038BD002041
:10B4700038BD16232B604FF0FF3038BD042200305A
:10B48000124B1F2870B51E6808D80D46716C044613
:10B4900049B151F8240041F8245070BD162333609F
:10B4A0004FF0FF3070BD80213046EAF071FD01465B
:10B4B000706440B1031F00F17C0C002243F8042F9C
:10B4C0006345FBD1E5E74FF0FF3070BD042200304B
:10B4D00038B50B4B1D686C6C0CB1002038BD802159
:10B4E0002846EAF055FD686438B1031F00F17C027C
:10B4F00043F8044F9342FBD1EFE74FF0FF3038BDE4
:10B500000422003038B5174B1F281D6826D86A6CF6
:10B51000044682B152F8243002EB84024BB1591C2C
:10B520001AD0012B16D000252046156098472846D2
:10B5300038BD012038BD80212846EAF029FD0246A9
:10B54000686458B1031F00217C3043F8041F834214
:10B55000FBD1DFE7032038BD022038BD4FF0FF30BC
:10B5600038BD00BF0422003070B50C46084D0346BC
:10B570000026204611461C462E60E9F0E1FF431CE0
:10B5800000D070BD2B68002BFBD0236070BD00BFC6
:10B59000DC2F0030E9F0CEBF10B50C46B1F90E102B
:10B5A00000F0B2F8002803DB636D0344636510BD4F
:10B5B000A38923F48053A38110BD00BF00207047EE
:10B5C0002DE9F0410C46B1F90C101F46CB0505469C
:10B5D00016460BD421F48051A1813B46B4F90E10DC
:10B5E00032462846BDE8F04100F01EB8B4F90E100E
:10B5F0000223002200F068F8B4F90C10EAE700BF5B
:10B6000010B50C46B1F90E1000F05EF8A389421C8B
:10B610000EBF23F4805343F480536065A38110BDB3
:10B62000B1F90E1000F016B838B50C46084D844636
:10B63000114620461A4600232B606446E9F06EFF4F
:10B64000431C00D038BD2B68002BFBD0236038BDD5
:10B65000DC2F003038B5074D0022044608462A602A
:10B66000E9F060FF431C00D038BD2B68002BFBD0F5
:10B67000236038BDDC2F003070B50C46084D034602
:10B680000026204611461C462E60E9F04DFF431C63
:10B6900000D070BD2B68002BFBD0236070BD00BFB5
:10B6A000DC2F003038B5074D0022044608462A60DA
:10B6B000E9F03EFF431C00D038BD2B68002BFBD0C7
:10B6C000236038BDDC2F003038B50C46084D844669
:10B6D000114620461A4600232B606446E9F01CFF01
:10B6E000431C00D038BD2B68002BFBD0236038BD35
:10B6F000DC2F003051F8040C0028A0F10400BCBF7E
:10B700000B58C018704700BF38B50C46084D84462A
:10B71000114620461A4600232B606446E9F0F8FEE5
:10B72000431C00D038BD2B68002BFBD0236038BDF4
:10B73000DC2F003010B5044620461CB154F80C3BF9
:10B74000013300D110BD0822012100F071FB54F833
:10B750000C0C54F8082C14F8041C121AB2FBF1F269
:10B7600000F066FBE8E70000C26AD0E9003112F0A1
:10B77000040F2DE9F04118BF0B46A6B00021594C2B
:10B78000042601270291CDE90003D0064CBF03F146
:10B79000200203F168020392DA690399D2099B69D6
:10B7A00002F004021B880A4303F47F4303924FF024
:10B7B000E022A3F53E41D2F8882D02F4A002B2F5B2
:10B7C000A00F04BF012202924B424B410493464D0D
:10B7D00003A82C6000F02AFA04220121434800F05B
:10B7E00027FB0422012102A800F022FB10220121E4
:10B7F000019800F01DFB0098202201210C3000F080
:10B8000017FB019804220121103000F011FB0422E3
:10B81000012103A800F00CFB01980C220121143037
:10B8200000F006FB0C220121009800F001FB029BB6
:10B83000DA071FD5009BDB6ADB064ED415A8F4F7A8
:10B84000B9FDDDF804C00DF1140E0CF120030CF16C
:10B8500060081868083353F8041C7246434503C255
:10B860009646F6D1DCF8603025938422012105A8A4
:10B8700000F0DEFA00F0C0F8FFF75CFF4FF0E023C5
:10B88000D3F8003D03F47023B3F5402F0ED0184BCE
:10B8900005A88DF81C60059314338DF82870069365
:10B8A0004FF0FF33CDE90833FFF744FF2B68A34285
:10B8B00006D0104B0422012105A8059300F0B8FA28
:10B8C00000F02AFA002882D0049B1BB1019A9369E8
:10B8D0000233936126B0BDE8F08105A8F4F764FD5A
:10B8E000C3E700BFED55CEACE02F0030DC96110869
:10B8F00028ED00E0ACCE55ED37B50E4D2A78202A64
:10B9000015D10D4C0D4823680D4918440192EAF0F9
:10B9100011F923680021019A203309482970236016
:10B92000F9F7F6FE03B0BDE83040EAF09DBE03B083
:10B9300030BD00BFD4310030FC3100302058140835
:10B94000D631003008B53420E7F04EFC144BD3F864
:10B95000902042F40022C3F89020D3F8902022F4E3
:10B960000022C3F89020D3F89020D3F8E82042F4C6
:10B970000022C3F8E820D3F8102142F40022C3F8D3
:10B9800010216D22D3F81031064BDA604FF0FF32F0
:10B990001A620D221A600122034B1A7008BD00BF03
:10B9A00000440258004C00400C320030014B186833
:10B9B000704700BFFCFF1B08014B0248C01A7047CC
:10B9C0002058140800001C0800487047205814082C
:10B9D00007490022074B5B1A9A4201D301207047A6
:10B9E00051F8040B013001D10432F5E70020704713
:10B9F0002058140800001C085E4B2DE9F74F1A6808
:10BA000002255D4B02F56A58DFF894911A7808F127
:10BA100018085A4F5A4C9044DFF888A1E9F096F87C
:10BA2000A9EB070B06460EB14E2D49D9A9EB07022B
:10BA3000B2EB080700F192804E2D00F28F80DFF804
:10BA400068C16B1C4F4E0C21DBB2ACEB06006943A6
:10BA5000B84273DD60184FF0010C665090463E44CA
:10BA600080F808C04660B2EB080213D44F2B11D007
:10BA7000454E19464548AB1C351ADBB295424FF08E
:10BA80000C0505FB01F163DD6518012602446050D9
:10BA90002E726A600C2201215343E21811724FF09A
:10BAA000FF31E15051603A4B1B782BB1394B1B6889
:10BAB0002360394B1B686360314803B0BDE8F08FE9
:10BAC000336AF06953450ABF344BF31AA3EB0A03F8
:10BAD00080B10193EAF01CFA019B58B12A460C216F
:10BAE00001354A430121EDB2A0180172F169A1505C
:10BAF0000D3141600C200121984400FB05FCD84524
:10BB000004EB0C0244F80C6006F13C0C1172C2F814
:10BB100004C005EB010205F10205D2B2EDB200FB53
:10BB200002F204EB02000172316AA1501944416033
:10BB300014D23046E9F01AF8064674E767184FF059
:10BB4000010E8044665087F808E0C7F804C08AE711
:10BB5000621801256050157256609BE74F2D01D881
:10BB60002B4697E7012384F8BC334FF0FF33C4E939
:10BB7000ED3398E7FC310030D43100302058140800
:10BB8000E0230030D82F003000000430000B0230DA
:10BB9000DC23003000320030F83100300022003069
:10BBA00000001C0800060030000B02300C4B1B7814
:10BBB00010B50BB9FFF7C6FE00230A490A48CA6947
:10BBC0009206FCD54A6A1C5CD2B2944205D101337C
:10BBD000DBB20E2BF3D1002010BD0023EFE700BF36
:10BBE0000C320030004C0040E096110838B5084B8C
:10BBF00004461B780BB9FFF7A5FEE4B2054DAC6215
:10BC0000EB695B0600D538BDEAF02EFDF8E700BF12
:10BC10000C320030004C004010B5441E14F8010FE7
:10BC200000B910BDFFF7E2FFF8E7000070B5026849
:10BC30000446EFF30581D9205369C9B2A5F0CCF9C8
:10BC4000294B1B78A3B1294B94E8030083E8030038
:10BC50002748FFF7E1FF6368B3B12648FFF7DCFF31
:10BC60002548FFF7D9FFFFF7A1FF2448FFF7D4FFCE
:10BC7000234D2B783BB124681CB12046EAF048F9EB
:10BC800020B900232B7070BD1E48E7E720461E4EEA
:10BC9000EAF052F900F2145084421FD22046EAF032
:10BCA0004BF930602046194EEAF05AF904F5E0539A
:10BCB000834217D92046EAF053F930600023144A32
:10BCC0001360144A1370FFF783FE0028D9D0EAF0FE
:10BCD000CBFC0120BDE87040E9F0B4BFA4F21453DE
:10BCE0003360DFE73360E9E7D531003004320030FC
:10BCF000F0961108F59611080697110804831208AA
:10BD0000DC2300300097110800320030F831003099
:10BD1000FC310030D4310030284B1A7870B542B174
:10BD20002748FFF779FF274B5868003818BF0120D4
:10BD300070BD254A107800283CD0244E244C33682E
:10BD40002448254D1A1D21782D1A0A44AA4205D3EC
:10BD5000224A4FF0FF31D161202222702278D2B1E5
:10BD600003F120018D4205D81F2A9FBF1B4AD361D2
:10BD700020222270202219491844E9F0DBFE3268A3
:10BD80002378002115481344202221703360F9F7ED
:10BD9000BFFCEAF069FC33689D4207D90F492022B5
:10BDA0000F48CB61E9F0C6FEEAF05EFC0020E9F046
:10BDB00049FFB8E701221A70BAE700BFD531003059
:10BDC0004C97110804320030DC230030FC31003085
:10BDD000D43100302058140800001C08D63100303F
:10BDE000E0FF1B082DE9F84307460E460024DFF864
:10BDF0003890DFF83880B44201D1BDE8F88324B12F
:10BE0000230702D14846FFF707FF3D5D01342B09A8
:10BE100005F00F0518F80300FFF7E8FE18F8050015
:10BE2000FFF7E4FEE7E700BF048312085C97110800
:10BE3000474B1B782DE9F74F07460E4690465BB1FE
:10BE4000022925D0042938D0012902D11146FFF753
:10BE5000C9FF4048FFF7E0FE3F4B1B78002B4ED058
:10BE60003E4A00253E4BA2EB030938E037F8143078
:10BE7000ADF8043024B1620702D12846FFF7CCFEAA
:10BE80000134022101A8FFF7ADFFA045EED1E0E7A4
:10BE90000024304DF9E757F82430019324B1A3076B
:10BEA00002D12846FFF7B8FE042101340DEB010052
:10BEB000FFF798FFA045EED1CBE70024254DF9E729
:10BEC000FFF71AFD022E1DD0042E2CD0012E06D114
:10BED0002378795D5A1C2270224AD1540135A84535
:10BEE0000DD0214B214C1B682278043313444B4561
:10BEF000E6D31C4B4FF0FF32DA612023237003B0EE
:10BF0000BDE8F08F2378DFF85CA05A1C22703A78E5
:10BF10000AF80320FFF7F0FC23785A1C2270002255
:10BF20000AF80320DAE74FF0000ADFF838B0227889
:10BF30003B78511C23FA0AF30AF1080A21700BF826
:10BF40000230FFF7D9FCBAF1200FF0D1C6E700BFED
:10BF5000D531003004831208DC23003000001C08B7
:10BF600020581408D6310030FC310030D431003074
:10BF7000036800221B6818477FB5039140210546DE
:10BF800092F060F9039A18B90124204604B070BDFC
:10BF9000134E039296F9DE3D002BF5D06CF026FA95
:10BFA000437A039A53B96CF021FA847A039A2CB934
:10BFB0000C4B4021284692F04DF9E6E70A4BB6F9C2
:10BFC000E01DD3F80832B3F908309942DCDD074BA5
:10BFD0004021284600240093054B92F03BF9D4E71A
:10BFE0001052003070971108107200308F971108AE
:10BFF0007D971108F0B50D46202104462DED028BEA
:10C000009DB092F01FF9002800F0C680634E96F9AB
:10C01000DE3DBBB106F50052B6F9E03DD2F808228C
:10C02000B2F90C1003F10A02914203DD40F28D32A5
:10C03000934207DC5A4B2A462021204692F00AF907
:10C040000020A5E096F9CD3D022B05D1554B2A469F
:10C050002021204692F0FEF8B6F8A43D41F6583271
:10C06000A3F57A739BB293420CD806F61463DFED06
:10C070004E6A93ED007AB4EEE67AF1EE10FA03D848
:10C080004A4BD8E74A4BD6E706F61863D3ED007A59
:10C09000F4EEE67AF1EE10FAF2D9464FD7F89C307A
:10C0A000D3ED096AF4EEC76AF1EE10FAE8D493ED25
:10C0B0000B7AB4EEE77AF1EE10FAE1D4B6F9DA3D94
:10C0C000002B01DC3C4BB6E7A7F5405393F8102852
:10C0D0000D2A06D80123934013F4215F01D0374B7A
:10C0E000A9E737480FF0DCFE012806D1D7F8A800F1
:10C0F00099F07CFE48B1012810D0324B93F881159D
:10C1000011F010012AD0304B95E7304B0093304BA3
:10C110002A462021204692F09DF891E7294B93F87A
:10C120002032CBB119212B4859F02EFCA0B106F6D4
:10C13000B8531921274893ED008A59F055FCDFEDDB
:10C14000267AB8EEC88A20EE270AB4EEC08AF1EE4D
:10C1500010FAD2DD214BD9E7214BD7E7602204A8A2
:10C160000391F9F7D5FA642303AA1E49D7F8A4006E
:10C1700099F0DCF818B903AB00931B4BC8E76423B4
:10C1800003AA1A49D7F89C0095F00CFF0028F2D0BA
:10C190001DB0BDEC028BF0BD0120F9E7105200305C
:10C1A00098971108AB971108000000B4E3971108A5
:10C1B000D397110810920030FD97110812981108BA
:10C1C00054A6003010720030A39811085798110837
:10C1D00032981108984300300000C8427698110840
:10C1E00067981108B8981108BC981108CE981108E2
:10C1F00008B516F02BF80121BDE8084015F090B8FD
:10C200002DE9F043DFF850910546ADB00E46D9F860
:10C21000680503681B699847804616F017F80021E7
:10C220000746602214A81391F9F772FA642313AA3F
:10C230004146384615F050FA044648B913AB3B4A1C
:10C240003146284692F02AFA20462DB0BDE8F08308
:10C2500037487AF0C1FDB8F1000F03D195F91E30CF
:10C26000012B0AD1334812F0FBFF80B9324A314624
:10C27000284692F013FA0024E6E710F0060FE3D008
:10C28000A9F5804012F0ECFF08B92C4AEFE703A9AA
:10C29000384615F037F828B19DF80D305B0601D50A
:10C2A000274AE4E7DFF8B4800023D8ED007AF5EE02
:10C2B000C07AF1EE10FAC7DD0DF120090893099359
:10C2C00005AA0A9307AB04A93846019306ABCDF83B
:10C2D000009015F021FC1B4B48460B931A4B0D9315
:10C2E0001A4B0F931A4B119334F0AEFF059B0422A7
:10C2F000D8ED007A0E93049B8DED0C0A1093069BEB
:10C3000012930BAB93ED017AB4EEE77AF1EE10FAEB
:10C3100004D5013A03F10803F4D195E71B683146CF
:10C320000C4A284692F0BAF9A5E700BFD498110844
:10C33000CC5C003010320030DD981108F498110800
:10C340001A991108D7EF11089CB313086AD1130882
:10C350004604120828991108107200300C60003051
:10C3600008B5064B93F881359B0704D5044A92F033
:10C3700095F9002008BD0120FCE700BF10720030D5
:10C380003899110870B50C4C05460E46D4F868056E
:10C3900003685B69984710B10124204670BDA4F57D
:10C3A000804012F06FFF04460028F5D1034A314661
:10C3B000284692F073F9F0E710720030489911089E
:10C3C0002DE9F046454D9BB081468A46D5F88C351F
:10C3D00093F8D56066B9424B1B68986A03685B6B3B
:10C3E0009847044640B93F4A5146484692F056F9AC
:10C3F00030461BB0BDE8F0866BF0F8FF20216DF0F1
:10C4000045F958B16BF0F2FF1F216DF03FF980B391
:10C410000024354A5146484692F040F995F8563581
:10C4200043B195F858352BB10024304A514648465F
:10C4300092F034F95146484693F0D0F90021602239
:10C44000884202A8019108BF0C46F9F761F9D5F8B6
:10C450008C0501AA642103681B689847054680B9CA
:10C460002C4601AB224A5146484692F017F926461F
:10C47000BEE76BF0BBFFA5216DF008F90028C7D11E
:10C48000CCE7002CF3D0D9F808303BB9D9F800300C
:10C49000514648469B6B98470446E8E75146484654
:10C4A000FFF7A8FD074651464846FFF759FF3840B9
:10C4B0005146C4B24846FFF75FFD51460440484626
:10C4C000FFF760FF51460440484692F02BF9514671
:10C4D0000440484693F09AF90440C8E710720030CF
:10C4E000A8A800305C991108739911088D9911085A
:10C4F000A599110808B5FFF763FF034A82F84805BC
:10C50000024A907108BD00BF10720030ADAA003021
:10C51000F7B506460F4691F0D1FE0446A0B30221BE
:10C52000304691F08FFE054670B315F08FFE4FF444
:10C530008071044614F0F4FE48BB20464FF40071AD
:10C5400014F0EEFE04460023019315F07FFE01A9CE
:10C5500014F07EFCECB1DDED017A0F4BF1EE677A61
:10C5600093ED1A7A77EEC77AB7EE007AF0EEE77AB3
:10C57000F4EEC77AF1EE10FA06DD0024074B3A46D6
:10C580000221304691F066FE204603B0F0BD002443
:10C59000D9E72C46F8E700BF10920030B099110897
:10C5A000F8B504460F4692F06FF910210546204673
:10C5B00091F048FE58B12046FFF71AFE064630B902
:10C5C0003546044B3A461021204691F043FE28465A
:10C5D000F8BD00BFC499110870B505460E4691F02C
:10C5E000B3FD044678B18021284691F02BFE50B16E
:10C5F000074B93F84D3B43B10024064B3246802154
:10C60000284691F027FE204670BD0446FBE700BF98
:10C6100010720030D899110838B50D4D0446D5F880
:10C62000A80099F0E3FB012810D0D5F8A80099F0F4
:10C63000DDFB022804D02046BDE8384091F086BDDD
:10C6400004480FF02DFC0128F5D138BD0020FCE78F
:10C650001092003054A60030F0B50F4D85B006465C
:10C660000F46D5F800326A460093D5F8043201939C
:10C67000D5F808320293D5F80C32039393F03CF8C6
:10C6800004463946304691F03FFE2040C0B285F85E
:10C69000470505B0F0BD00BF107200302DE9F8432A
:10C6A000DFF8AC90064626480F467AF095FB044624
:10C6B000D9F86805DFF89C8003681B699847054630
:10C6C00030B914F0060F03D1D9F89C35022B09D1EB
:10C6D0003946304691F004FF054618B9002488F821
:10C6E00007400AE039463046FFF78AFD0446002835
:10C6F000F4D02DB9012388F807302046BDE8F8832F
:10C700000821304691F09EFD0028F3D00D4825F019
:10C710001BFC0028EED00C4BB02193F8E42301FB66
:10C72000023203F50053B2F8EE21B3F9CE3D9A423E
:10C73000E0DD064B3A460821304691F08BFDCDE70F
:10C74000CC5C00303033003010320030EC991108EE
:10C7500010720030ADAA003070B588B005460E46A4
:10C7600091F0C4FF044688B32021284691F06AFD69
:10C7700060B31B4B93F85C2142B393F838319B07AD
:10C7800024D507AA06A9174876F0F6FCF0B19DED6E
:10C79000077ADFED157AB4EEE77AF1EE10FA15D8E4
:10C7A000B7EEC77A0024202128468DED027BDDED0F
:10C7B000067AFDEEE77A08A3D3E90023CDED007AEF
:10C7C000CDE90423094B324691F044FD204608B0E0
:10C7D00070BD00BFAFF30080000000403333E33F83
:10C7E000109200307C6000309A99193FFC99110832
:10C7F0002DE9F3410F46044615F028FD804614F05C
:10C8000043FD054640B9524A0121204691F046FFBA
:10C81000284602B0BDE8F0814E4E3946D6F868058C
:10C8200003689B699847054658B9D6F868050368B8
:10C83000DB6C9847484A03460121204691F02EFFC1
:10C84000E6E7A368002BE3D01021204691F0FAFC24
:10C8500020B3D8ED967A98ED950A20EE270AF5F7E1
:10C860003BFBDFED3E7AA6F5005320EE270ADFED15
:10C870003C7AB3F9A43D20EE270A07EE903AF8EE91
:10C88000E77AB4EEE70AF1EE10FA07DD354B012244
:10C890001021204691F0DEFC0025B9E7202120463A
:10C8A00091F0D0FC38B196F88135DB0603D52E4BDC
:10C8B00001222021EDE74021204691F0C3FCE8B1A0
:10C8C000012F14D0232F12D0042F10D0274800F0AE
:10C8D000ADFBB5EEC00AF1EE10FA1DDD244B0122CE
:10C8E000402120460093234B91F0B4FCD4E7D6F8C6
:10C8F000680503689B6C98470028E7D01E4B1B68AF
:10C90000D86A0368DB6998470128014619D11B4A98
:10C91000204691F0C3FEBFE7D6F8680503685B695F
:10C92000984730B1D6F80832B3F90A30002BE5DD6C
:10C93000D4E7D6F8680503681B6898470B28DDD153
:10C94000F0E73946204602B0BDE8F04192F05ABA0D
:10C95000289A110810720030399A1108E02E6542A9
:10C960000000C8424D9A1108A398110810320030F7
:10C970008F971108559A1108A8A80030619A1108DC
:10C9800070B505460E46FFF73BFC084B04463146A2
:10C99000D8712846FFF7F6FC00283146284608BF24
:10C9A000002492F02FFD204070BD00BFADAA0030E2
:10C9B0002DE9F341524F3B78002B40F09E80514CC3
:10C9C0000126D4F88C553E7095F8D55025B13B70B2
:10C9D000284602B0BDE8F08192F0DAFF054630B992
:10C9E000494A3870137843F001031370F0E75EF0A2
:10C9F000B5FC31465DF07EFCA4F5804007F010FAEE
:10CA0000424B1E710B26013E54F018FC54F034FBCF
:10CA100016F0FF06F7D13E4801F072FA15F016FC49
:10CA200004F2B452D0F81812116090F88832DA0784
:10CA30004DD414F0C7FE5EF091FC3C215EF01EFA6E
:10CA400004F2745300221A600021314801F002FB05
:10CA50002F4812F005FC01462E489FF01FFF2E4B79
:10CA600001212E4E1B68D86A03681B689847D4F8CA
:10CA70008C050368DB6A98470121D4F88C059CF08B
:10CA80004DF95EF06BFC8046D4F8680503681B68BE
:10CA9000984796F8382D014640465DF007FE4FF066
:10CAA0000008A6F5005006F5804607F0ABF95AF0ED
:10CAB00029FA59F055FD87F80080A4F0F9FA01230E
:10CAC000C6F8B40084F8593584F85D8580E79B0783
:10CAD000BAD431460E4805F071FA0023019315F0DF
:10CAE000B5FB01A914F0B4F9DDED017A04F2745339
:10CAF000F1EE677AC3ED007AA6E7002568E700BF8C
:10CB00000D32003010720030CCAA0030ADAA0030D7
:10CB100010320030A8720030A8A800301052003047
:10CB20002DE9F0433F4C87B007460D46D4F88C35CD
:10CB3000164693F8D530002B71D05AB1012901D097
:10CB4000232907D194F84B3523B90025284607B08F
:10CB5000BDE8F083002D56D029463246384692F083
:10CB6000D7FF05460028F0D015F070FB07461DF0F2
:10CB700093FF8046384614F03BF8D8B198F9283036
:10CB8000022B17D100264FF00009F1B203AA384654
:10CB9000CDF80C900191CDF81090CDF8149014F0D0
:10CBA00037FC019918B103AA40461DF021FC01365B
:10CBB000032EEAD101211C4807F09EFB01211A48EF
:10CBC00007F0F2FA0021D4F88C059CF0A7F817487A
:10CBD00036F052FF5EF0C2FB00215DF08BFB144B80
:10CBE00000211B68D86A03681B689847D4F8681549
:10CBF0000023104884F859350B1A383059425941EE
:10CC0000A0F08EF8A2E7D4F8680503685B6998473E
:10CC10000028A1D194F84B35002B9DD195E7012533
:10CC200094E700BF1072003010320030F89E0030E0
:10CC3000A8A8003008A200300020704710B5064CAC
:10CC4000D4F8680503685B6A984718B1D4F88C3546
:10CC500093F8D50010BD00BF1072003030B52DED37
:10CC6000028B87B0B0EE408A0C46FFF7E7FF05461F
:10CC7000E8B1B4EE488A2268636803A9D4ED027A69
:10CC8000F1EE10FA9FED0C0AF1EE677A039204932D
:10CC90004FF000024FF00103084850FE080ACDEDA6
:10CCA000057ACDE9002368BF13460DF0CDF928467B
:10CCB00007B0BDEC028B30BD00000000F4A40030D2
:10CCC00007B50191FFF7BAFF30B10199044803B0ED
:10CCD0005DF804EB00F0D2BB03B05DF804FB00BFCD
:10CCE0001032003001487AF039BA00BFCC5C003015
:10CCF00000F5804008B590F849358B4209D080F89E
:10CD0000491531B15EF02AFB0F21BDE808405EF005
:10CD1000B5B808BD70B500F5804605460C46D6F896
:10CD20009C358B4212D0012911D0022916D059B955
:10CD30005EF014FB1B215EF0A1F80D4A05F586405C
:10CD40000621743063F0C8FDC6F89C4570BD5EF0E6
:10CD500005FB1A215EF092F8064AEFE7012101F087
:10CD600079F95EF0FBFA1D215EF088F8024AE5E7EA
:10CD7000DC9A1108F19A1108EC9A110800F580422A
:10CD800010B592F881350C4603F00101A14209D09B
:10CD900064F3000382F88135DB0704D406F026FC37
:10CDA000024B9C7210BD06F003FEF9E7ADAA0030FD
:10CDB00000F5804090F8813561F3410380F88135BA
:10CDC000014B1973704700BFADAA003010B504467F
:10CDD0006BF00CFB20216CF059FC003804F580440A
:10CDE00018BF012084F8560510BD000070B5044638
:10CDF0005AF088F8436F04F5C045D5F8A420C2F86E
:10CE00006832D5F89C20936604F5E04292F89526A6
:10CE10004AB904F58044D4F88C25D360D5F89C0039
:10CE200003689B6D9847D5F89C000368BDE8704087
:10CE3000DB6D184770B500F5804504462DED028B7B
:10CE4000D5F88C3582B093F8D530002B00F0818076
:10CE500095F84B35002B7CD100F5C04696F8183C70
:10CE6000002B76D1D5F8680503685B6998470028E0
:10CE70006FD13A4BD3F8680503681B6898470B28B5
:10CE800067D0D6F8A4309FED367AD3EDC57AF0EEB0
:10CE9000E77AF4EEC77AF1EE10FA5AD515F0D6F922
:10CEA00095F8442301A914F0BDFF002851D0D5F80E
:10CEB0008C05443060F0E4FC0346B7EE001A9B207A
:10CEC000DFED280A93ED000A2EF006FCB5EEC00A4D
:10CED000F1EE10FA3DDDDDED017A9FED237AF0EE03
:10CEE000E77AF4EEC77AF1EE10FA32D504F5805401
:10CEF000D6F89C0004F5F36393ED848A0368D3F8B5
:10CF00009C309847DFED197A9FED197AA0EE678A79
:10CF1000B0EEC88AB4EEC78AF1EE10FA19D504F55E
:10CF2000F364D4ED857AFDEEE77A17EE903A002BA4
:10CF3000B8BF5B4207EE903AF8EEE77AF4EEC77AB4
:10CF4000F1EE10FA05D59FED0B0AD5F88C059DF092
:10CF500063FA02B0BDEC028B70BD00BF10720030EE
:10CF600000000034000000009A99193FD4023739BC
:10CF7000C2B8B23D0AD7233C00F5804008B5D0F8CE
:10CF80008C0503685B699847F6EE007A20EE270A65
:10CF9000B5EEC00AF1EE10FA48BF9FED010A08BDD8
:10CFA0000000000038B500F5C0450446B7EE001A91
:10CFB0007C2004F58044DFED110A2DED028BD5F8BD
:10CFC0009C3093ED370A2EF087FBD4F88C05B0EE39
:10CFD000408AD5F8A450036805F5BA755B6998478F
:10CFE00038EE400ADFED067A2846BDEC028B20EED3
:10CFF000270ABDE8384086F0BFBE00BF0000000031
:10D0000000007A4400F58043B3F9483143B900F594
:10D010000050B0F9DA0D0028B8BF404280B2704726
:10D0200083EAE370A0EBE370F8E7000038B52DED7C
:10D03000028B04466BF0DAF90368DB68984720B985
:10D040009FED310ABDEC028B38BD304B04F5005525
:10D05000DFED2F8A5920D3F80832B0EE681ADFEDE1
:10D060002A0AB3F90A3000EE103AB8EEC00A2EF0E0
:10D0700033FB4FF4C8720021B5F9E20DB0EE408ADF
:10D080002EF092FBA5F8E20D204611F09DFAB5F9BD
:10D09000E23D07EE900AB8EEE77A07EE903AF8EE36
:10D0A000E77A77EE676AB4EEE68AF1EE10FA11D508
:10D0B000204638EE668AFFF7A5FF07EE900AB8EE25
:10D0C000E70ADFED147A20EE270A20EE088A88EEC0
:10D0D000260AB7E777EE877AB4EEE78AF1EE10FA20
:10D0E000AEDDB5F9DA3D38EE678A9FED0A7A78EE63
:10D0F000E77A00EE103AB8EEC00A20EE070A20EEFA
:10D10000088A88EE270A9DE70000000010720030B0
:10D1100000007A440AD7233C7047000070470000A3
:10D1200000207047002070470020704700207047A3
:10D130000020704700207047002070470020704793
:10D14000002070477047000000F5375030307047BE
:10D150000048704750CC110800F58040D0F86805B1
:10D1600003681B68184700000348086031211170EC
:10D1700008221A60704700BFEC9E110800F5C040FD
:10D180009FED0A7AD0F8B0300120D3ED0C7AF4EE9E
:10D19000C77AF1EE10FABEBFD3ED027A9FED047AA2
:10D1A00067EE877AC1ED007A704700BF0000003457
:10D1B0000AD7233C00F58040D0F8680503681B6F50
:10D1C0001847000000F5C04393F8B93F002B14BF87
:10D1D0001B2003200B1A58425841704700F580402D
:10D1E00090F88105C0F380007047000000F5804092
:10D1F000D0F8680503681B6E1847000000F58040F2
:10D20000D0F8680503689B6D1847000000F5804062
:10D21000D0F8680503685B6D1847000000F580438F
